:100000000C94AC050C94F2050C94F2050C94F205DA
:100010000C94F2050C94F2050C94F2050C94F20584
:100020000C94F2050C94DA180C94F2050C94F20579
:100030000C94FC310C94F2050C94F2050C94F2052E
:100040000C94F2050C94F2050C94EC140C94F2054B
:100050000C94890B0C94F2050C94530B0C94F20540
:100060000C94E21B0C94F2050C945D2D0C94F2059B
:100070000C948E770C94F2050C94FF71071C0C1CE9
:10008000111C1A1C311C481C581C681C851CA91EFC
:10009000481C5B1D6C1D9B1DB91DD61D301E8B1E83
:1000A0009F204621B12133226B220E23D5233624F3
:1000B000B024E124392567259425F92543268D268A
:1000C000F026EB277C2DB02DF32D632E7B2EBB2E3F
:1000D000822F493049304930493049304930493020
:1000E0004930493049304930FE2F003005301D304D
:1000F0001F301066EB667067B166C467F2674D66C5
:10010000E0660A0D3D3D3D3D3D3D3D3D3D3D3D3DB6
:100110003D3D3D3D3D3D3D3D3D3D3D3D3D3D3D3D0F
:100120003D3D3D3D3D3D3D000A0D426174743A0048
:100130002025642043656C6C732000204C6F772071
:100140007761726E696E673A2025642E2564000A15
:100150000D466F756E6420424C2D4374726C3A20CC
:10016000002564000A0D0A0D2121204D49535349F1
:100170004E4720424C2D4354524C3A2025642021B6
:1001800021000A0D43616C6962726174696E6720B7
:1001900070726573737572652073656E736F722EFE
:1001A0002E004F4B0A0D000A0D466C696768742DCE
:1001B00074696D65202575206D696E20546F7461BA
:1001C0006C3A2575206D696E00416E676C654E69ED
:1001D000636B20202020202020416E676C65526FC9
:1001E0006C6C202020202020204163634E69636BCB
:1001F000202020202020202020416363526F6C6C3F
:100200002020202020202020205961774779726FFC
:10021000202020202020202020416C7469747564E7
:1002200065205B302E316D5D204163635A202020B4
:100230002020202020202020204761732020202003
:10024000202020202020202020436F6D70617373B8
:100250002056616C7565202020566F6C746167654F
:10026000205B302E31565D202052656365697665CE
:1002700072204C6576656C20204779726F20436F41
:100280006D70617373202020204D6F746F72203168
:100290002020202020202020204D6F746F722032DB
:1002A0002020202020202020204D6F746F722033CA
:1002B0002020202020202020204D6F746F722034B9
:1002C0002020202020202020203136202020202007
:1002D00020202020202020202031372020202020F6
:1002E00020202020202020202031382020202020E5
:1002F00020202020202020202031392020202020D4
:10030000202020202020202020536572766F20207E
:10031000202020202020202020486F7665726761F1
:1003200073202020202020202043757272656E7477
:10033000205B302E31415D20204361706163697420
:1003400079205B6D41685D2020486569676874208D
:10035000536574706F696E74203235202020202020
:100360002020202020202020203236202020202065
:10037000202020202020202020436F6D7061737387
:1003800020536574706F696E744932432D457272E3
:100390006F7220202020202020424C204C696D6963
:1003A0007420202020202020204750535F4E696376
:1003B0006B20202020202020204750535F526F6C5C
:1003C0006C202020202020202021212120494E4364
:1003D0004F4D50415449424C4520212121002E00CF
:1003E0000A0D20444143206F722049324320455278
:1003F000524F522120436865636B204932432C20C1
:1004000033567265662C2044414320616E6420425D
:100410004C2D4374726C005B25695D005B25695D42
:10042000002B204D696B726F4B6F70746572202BBF
:100430000048573A5625642E25642053573A2564C0
:100440002E256425632056340053657474696E67E5
:100450003A2564202573004D6978657220457272D3
:100460006F72210048617264776172652045727213
:100470006F7220313A2564202121004D6973736920
:100480006E6720424C2D4374726C3A256421210022
:1004900021204E432D4552523A20253264202120FE
:1004A00000493243204552524F52212121004865D4
:1004B000696768743A202025356900536574706F48
:1004C000696E743A2535690050726573737572658B
:1004D0003A253569004F66667365743A20202535E4
:1004E00069006163742E2062656172696E67004EF7
:1004F00069636B3A20202020202025356900526F47
:100500006C6C3A20202020202025356900436F6D37
:10051000706173733A202020253569004B25693AB4
:1005200025346920204B25693A25346920004E691D
:100530003A2534692020526F3A25346920004773E8
:100540003A253469202047693A2534692000503122
:100550003A253469202050323A253469200050333E
:100560003A253469202050343A25346920004779EF
:10057000726F202D2053656E736F72004E69636B2E
:100580002025346920282533692E25782900526FCB
:100590006C6C2025346920282533692E25782900A4
:1005A00059617720202534692028253369290041A5
:1005B0004343202D2053656E736F72004E69636B49
:1005C0002025346920282533692900526F6C6C205E
:1005D000253469202825336929005A202020202528
:1005E000346920282533692900566F6C746167656A
:1005F0003A2020202533692E253169560043757233
:1006000072656E743A2020202533692E25316941A8
:1006100000506F7765723A202020202025346957DA
:10062000004469736368617267653A202535696DB6
:1006300041680052656365697665720052432D51C9
:1006400075616C6974793A202534690052432D43F1
:1006500068616E6E656C733A25346900436F6D7026
:10066000617373004D61676E65743A2020202535F3
:1006700069004779726F3A202020202025356900D3
:10068000536574706F696E743A2025356900506F38
:10069000746925693A202025336900506F746925F3
:1006A000693A202025336900536572766F20200057
:1006B000536574706F696E74202025336900506F24
:1006C000736974696F6E3A202533690052616E67F1
:1006D000653A2533692D25336900424C2D437472E8
:1006E0006C204572726F72732000253364202533AD
:1006F0006420253364202533642000424C20546557
:100700006D706572617475726500253364202533E0
:100710006420253364202533642000424C20437537
:100720007272656E740028696E20302E3141290086
:100730002533642025336420253364202533642049
:1007400000424C2D4374726C20666F756E642000FD
:1007500020256320202025632020202563202020C1
:1007600025632000202563202020256320202025CC
:1007700063202020256320002025632020202D20B9
:1007800020202D2020202D2000313000313100315B
:100790003200466C696768742D54696D65202000CD
:1007A000546F74616C3A2535756D696E00416374E0
:1007B0003A20202535756D696E0028726573657461
:1007C00029000A0D47656E65726174696E67206461
:1007D000656661756C7420506172616D65746572D7
:1007E00020536574202564000A0D5573696E6720D7
:1007F000506172616D657465722053657420256463
:10080000000A0D47656E65726174696E67206465E4
:100810006661756C74204D69786572205461626CF4
:1008200065000A0D4D697865722D436F6E666967C4
:100830003A202725732720282575204D6F746F7265
:100840007329000A0D414343206E6F742063616C6D
:1008500069627261746564210D0A0000008F001ED8
:1008600001AD013B02CA025803E603740402058F7E
:10087000051B06A7063307BE074808D2085B09E335
:10088000096B0AF20A780BFD0B810C040D860D072B
:100890000E870E060F840F00107B10F5106E11E509
:1008A000115B12CF124213B31323149214FE146A75
:1008B00015D3153B16A11605176717C817271883F8
:1008C00018DE1837198E19E319361A871AD61A2323
:1008D0001B6E1BB61BFD1B411C831CC31C001D3C57
:1008E0001D751DAB1DE01D121E421E6F1E9A1EC3FC
:1008F0001EE91E0D1F2E1F4D1F691F841F9B1FB059
:100900001FC31FD31FE11FEC1FF51FFB1FFF1F009D
:1009100020040100002C6D000201011B6E01030286
:1009200002AF6E02040303576F030004040C6F252B
:1009300032692E2531695600253364256320253020
:1009400033646D25630053746174757300455252AE
:100950004F523A202532642000253469202532691F
:100960003A25303269002534696D256300253369E5
:100970002025336920253369202533690025336913
:100980002025336920253369202533690054656D9E
:100990007065726174757265732020202000256374
:1009A000432020202020002532692E253169562041
:1009B0002533692E253169410025346957202536B4
:1009C000696D4168004D61676E65743A253369252C
:1009D0002520253369256300496E636C692E3A250D
:1009E00033692563202825692920002532756D2F5C
:1009F00073205361743A2564200020203344004E54
:100A00006F4678004447505300486F6D653A253370
:100A1000646D202533642563202563004E6F204ECE
:100A20006176694374726C21000A0D7777772E4DD9
:100A3000696B726F4B6F707465722E6465202863EA
:100A40002920486953797374656D7320476D624836
:100A5000000A0D74686520757365206F66207468E0
:100A6000697320736F667477617265206973206F94
:100A70006E6C79207065726D6974746564200A0DFE
:100A80006F6E206F726967696E616C204D696B7261
:100A90006F4B6F707465722D486172647761726517
:100AA000005573657200486F54542056340041431A
:100AB000542044534C004A657469005370656B744C
:100AC00072756D0050504D000A0D52656365697670
:100AD00065723A2000756E6B6E6F776E2E205573BF
:100AE000696E672050504D2E2E2E006E6F7420734D
:100AF0007570706F727465642062792068617264C9
:100B00007761726521000A0D202D204C4942204E4C
:100B10004F5420434F4D50415449424C45202121D0
:100B20002121000A0D466C69676874436F6E747208
:100B30006F6C0A0D48617264776172653A25642EA4
:100B400025640A0D536F6674776172653A562564A1
:100B50002E2564256320000011241FBECFEFD0E1B5
:100B6000DEBFCDBF11E0A0E0B1E0E6EBF5EF02C0E3
:100B700005900D92AE3AB107D9F719E0AEEAB1E0AF
:100B800001C01D92A530B107E1F76AEAE2E0F0E0AA
:100B900081E2809357007491AE014F5F5F4F20EF69
:100BA00037EFDA019FE0F9012F5F3F4F84918D937A
:100BB000915097FFF8CF773911F40000FECFFA017A
:100BC0009EE0819168276095915097FFFACF8889C0
:100BD000681721F0773911F40000FECF0E94BE069D
:100BE0000C94DA7A0C94000082E091E09F938F934A
:100BF00082E092E19F938F93E0918E03F0918F03B7
:100C000009950F900F900F900F90089580913306E3
:100C1000E82FFF27EE0FFF1FE859F84F80819181E1
:100C20008D5E9F4F14F010920301808191818A5B49
:100C30009F4FCCF4809103018823A9F481E0809335
:100C400003018091C2038F5F8093C203853038F027
:100C500088EE93E09093E4018093E301089566E9C0
:100C600070E00E94FA3308951F93CF93DF93182FFB
:100C7000882389F088E291E09F938F9382E092E14C
:100C80009F938F93E0918E03F0918F0309950F90BE
:100C90000F900F900F9080915606823308F044C059
:100CA00084EF91E00E94DF15EC01112329F0CE01C1
:100CB0000E94E8158823D9F3C2E0D0E026E530E0B1
:100CC00080912201909123018217930730F02196A1
:100CD000255D3F4FC730D10598F38091560699277F
:100CE000C89F9001C99F300DD89F300D11242093CB
:100CF00001011123D9F068EC70E08C2F0E94FA33C7
:100D0000DF93CF9380E391E09F938F9382E092E112
:100D10009F938F93E0918E03F0918F0309958DB788
:100D20009EB706968DBF02C080930101112311F179
:100D3000809101016AE00E942D7A892F99279F9363
:100D40008F93809101010E942D7A99279F938F9311
:100D50008BE391E09F938F9382E092E19F938F9337
:100D6000E0918E03F0918F0309952DB73EB7285F70
:100D70003F4F2DBFDF91CF911F910895CFEFD0E16D
:100D8000DEBFCDBF88249924C1E07C2E14B815B8ED
:100D90008AE08AB98FE58BB9B7EEEB2EB3E0FB2E74
:100DA0002EEC3FEFE20EF31EF7FEFACF189B06C0C3
:100DB000199B02C08DE005C08BE003C0199B04C0E5
:100DC00084E18093020107C08AE0809302018EE3F0
:100DD0008AB987E48BB981E887B93E9A8FEF88B9E1
:100DE0008BE184B981E085B9469A84B7877F84BF57
:100DF000809160008861809360001092600084ECB4
:100E000099E09093E4018093E30110928F02109295
:100E10008E0210926D0710926C0710929102109240
:100E200090021092930210929202209102012431BA
:100E300028F084EC94E0A0E0B0E004C08BE095E002
:100E4000A0E0B0E080933E0190933F01A093400169
:100E5000B09341012A3011F0243110F0289801C0DC
:100E6000289A2C3010F0293111F4299A01C02998C0
:100E70000E9448160E9419160E940A120E94C3314D
:100E80000E945B1A81E00E94112D0E94B6640E94AC
:100E90004F7085E00E944976809102018C3010F0FD
:100EA000893111F4299A01C0299878940E94322C32
:100EB00080913002826080933002109233020E944F
:100EC000A13F84EF91E00E94DF157C018091300208
:100ED00080FD05C0C7010E94E8158823B9F38FE49F
:100EE00091E09F938F93A2E0AA2EA2E1BA2EBF9227
:100EF000AF92E0918E03F0918F03099580EA9FE015
:100F00000E94DF157C01C0E0D0E00F900F900F90A1
:100F10000F900AE017E0FEEBCF2EF6E0DF2E0E94E6
:100F2000A13F8091300280FD05C0C7010E94E815F5
:100F30008823B9F3F60180811816ACF40BC00E9427
:100F4000A13F8091300280FD05C0C7010E94E815D5
:100F50008823B9F3C7010E94E815882321F4F8011A
:100F60008081882364F7F801808187FF19C021966A
:100F7000DF93CF93219781E691E09F938F93BF9268
:100F8000AF92E0918E03F0918F0309958091AF01AC
:100F90008F5F8093AF012DB73EB72A5F3F4F2DBFC4
:100FA000219684E090E0C80ED91E085F1F4FCC3018
:100FB000D10508F4B4CFC0E0D0E007E017E0EEEBD5
:100FC000EE2EE6E0FE2EF801838187FD1DC0F701BD
:100FD00080811816CCF42196DF93CF93219784E675
:100FE00091E09F938F9382E092E19F938F93E091A2
:100FF0008E03F0918F03099582E08093E1012DB774
:101000003EB72A5F3F4F2DBFF801838180788383ED
:10101000219624E030E0E20EF31E085F1F4FCC3033
:10102000D10588F20E94F405909131068091AF01BC
:10103000981728F48091A80380618093A80382E820
:1010400091E09F938F93C2E0D2E1DF93CF93E09141
:101050008E03F0918F03099588EE93E00E94DF15CF
:101060007C010E94991A0F900F900F900F90C7016A
:101070000E94E8158823D9F382EA91E09F938F9329
:10108000DF93CF93E0918E03F0918F03099580E079
:101090000E94DE34809102010F900F900F900F900C
:1010A0008A3011F0843110F0289801C0289A80ED20
:1010B00097E09093E4018093E30185E58093C40376
:1010C0008EE090E00E94562A9927182F00278FE083
:1010D00090E00E94562A080F111D1093B50100934D
:1010E000B4018AE090E00E94562A9927182F002721
:1010F0008BE090E00E94562A080F111D1093B30157
:101100000093B2010F5F1F4F39F08091B4019091AD
:10111000B5018F5F9F4F41F41092B5011092B40159
:101120001092B3011092B2018091B2019091B3017B
:101130009F938F938091B4019091B5019F938F936A
:1011400087EA91E09F938F93DF93CF93E0918E0393
:10115000F0918F0309950E94162088E893E19093FF
:10116000390180933801C1E0C093C3038C2F0E94E2
:101170003406809159060E949C750E94F40580ED0A
:1011800097E00E94DF157C018AEF90E00E94DF1556
:1011900083E080938B051092AE018091A2062DB75B
:1011A0003EB7285F3F4F2DBF84FF02C0C093B601FA
:1011B00012BC11BC8091B801882311F04798FECF72
:1011C0008091E701882309F45DC28091140188238E
:1011D00009F458C21092E7018091C203882319F0E4
:1011E0000E94060602C00E9419430E94A13F20915E
:1011F00002012A3011F0243110F0289801C0289AF9
:1012000080918202882331F0809182028150809304
:1012100082020EC080916F00806280936F001092F6
:101220006907109268078091A80388608093A803DB
:101230008091380190913901019790933901809301
:1012400038018091380190913901892B21F08091EA
:1012500031028823C9F18091380190913901892B9D
:10126000D9F40E943B2D85E090E090933901809362
:1012700038018091C5059091C60501969093C605E9
:101280008093C5058091A80381608093A803809115
:101290008C05826080938C0580910A0190910B01EE
:1012A0008F5F9F4FC1F4809181028823A1F088EA6B
:1012B00091E69093E4018093E30180E890E09093BD
:1012C0000B0180930A0107C02A3011F0243110F07D
:1012D000289801C0289A0E9416778091E7018823F8
:1012E00009F0CEC180911001882311F00E94A2164E
:1012F0000E9454120E94D90DC7010E94E81588234C
:1013000009F4BAC184E190E0E80EF91E0E9460166B
:1013100080913102882349F08091A80382608093F4
:10132000A80380918C0582600FC08091E3019091A9
:10133000E401892B59F48091380190913901079784
:1013400028F080918C058D7F80938C058091B6016B
:10135000882361F080918202873940F01092B601B3
:1013600088E893E19093E4018093E3018091050183
:10137000882321F08150809305012EC08093CE03F5
:10138000109255021092540210925302109252027F
:101390001092510210925002809182028823E1F44F
:1013A00080910A0190910B018F5F9F4FA9F42091CA
:1013B000B601223089F088E99AE39093E4018093A2
:1013C000E30180E09CE090930B0180930A012223CB
:1013D00019F082E08093B60180919D01893C70F004
:1013E000815080939D018091A8038B7F8093A803F7
:1013F0008091AB0381608093AB0351C080916E08F4
:101400008823F9F08091A80384608093A80389E081
:101410008093600380910A0190910B018F5F9F4F31
:1014200081F480918102882361F088E99AE39093A6
:10143000E4018093E30180E098EA90930B018093AC
:101440000A0110925203109251031092500310920D
:101450004F0310924E03109261088FEF8093D608CD
:101460001092A00810929F081092A2081092A10852
:101470008FEF9FEF90939E0880939D0810927102CA
:1014800010927202109273021092740210927502FE
:101490008091AB038E7F8093AB0310929D0180916E
:1014A0000101282F33278091220190912301821777
:1014B0009307FCF4809149028062809349028091F5
:1014C0000A0190910B018F5F9F4FF1F480912201EF
:1014D000909123010B97C4F080E797E19093E4018A
:1014E0008093E30180E093E090930B0180930A01E5
:1014F0000BC08091E3019091E401892B29F4809144
:1015000049028F7D8093490212BC11BC8091B701C2
:101510008F5F8093B701813309F065C01092B701E6
:101520008091490281FF0AC08091B0019091B10180
:1015300001969093B1018093B00104C05AEA852EC0
:1015400055E0952E80914A0290914B028050944034
:1015500008F049C02091D4053091D5054091D605B9
:101560005091D70580911A0190911B01A0911C0107
:10157000B0911D01281739074A075B0764F4809171
:10158000D4059091D505A091D605B091D7050596C3
:10159000A11DB11D20C02091D4053091D5054091E9
:1015A000D6055091D70580911A0190911B01A09109
:1015B0001C01B0911D0182179307A407B5079CF485
:1015C0008091D4059091D505A091D605B091D7050D
:1015D0000597A109B1098093D4059093D505A093EF
:1015E000D605B093D7050894811C911C82E7881614
:1015F0008BE0980609F040C0882499242091B4011A
:101600003091B5012F5F3F4F3093B5012093B40166
:101610008091B2019091B30101969093B3018093B0
:10162000B201832F9927682F8EE090E00E945E2AF6
:101630008091B4019091B5019070682F8FE090E097
:101640000E945E2A8091B2019091B301892F99275F
:10165000682F8AE090E00E945E2A8091B20190910A
:10166000B3019070682F8BE090E00E945E2A84E1C5
:1016700090E00E94DF157C010E94C1690E946670A3
:1016800071107A94772039F40E948569882319F0C3
:101690008CE0782E8FCD8091E201882309F08ACDED
:1016A0000E94D76487CD1F920F920FB60F9211241C
:1016B0008F939F93EF93FF93809107018823E1F429
:1016C0008091D2019091D30101969093D3018093A0
:1016D000D201FC01E155FB4FE081ED3019F08C3D6A
:1016E000910539F41092D3011092D20181E08093D8
:1016F0000701E093C60004C01092D3011092D201FA
:10170000FF91EF919F918F910F900FBE0F901F90BF
:1017100018951F920F920FB60F9211242F933F939B
:101720004F935F936F937F938F939F93AF93BF93E9
:10173000CF93EF93FF9390E08091B801813029F42B
:101740008091C6008093CE00CCC08091B8018230D9
:1017500029F48091C6008093D103C3C08091C60054
:101760008093CA015091D8015C3D10F09093D9014B
:101770008091CA018D3009F065C08091D901823015
:1017800009F060C09093D901852F99278F529C4F03
:10179000FC01329740812091D4013091D501241B66
:1017A0003109DC0111978C91281B3109C9019F7007
:1017B0009093D5018093D40146E0969587954A95FC
:1017C000E1F7982F935C9093D6012F733070235CD0
:1017D0002093D7018081981729F48C91281711F450
:1017E00091E006C090E08091C7018F5F8093C701B0
:1017F000C091C901CC2309F074C0992309F471C0C8
:1018000081E08093C901580F5093C6015150E52FD4
:10181000FF27EF52FC4F8DE080838091D303823508
:1018200009F05FC00E94162088E190E02CE00FB61E
:10183000F894A895809360000FBE20936000C09339
:10184000E1014FC02091D901822F99278130910564
:10185000F9F0823091051CF4892B21F040C00297E9
:1018600011F13DC08091CA01833239F48091C901E0
:10187000882319F481E08093D9018091CA01809373
:10188000D10381E08093D8018091CA01992722C0B9
:101890002F5F2093D901E52FFF27EF52FC4F809156
:1018A000CA01808309C0E52FFF27EF52FC4F8091CA
:1018B000CA0180835C3D20F45F5F5093D80102C071
:1018C0001092D9012091CA018091D4019091D50143
:1018D000820F911D9093D5018093D40102C0109284
:1018E000D901FF91EF91CF91BF91AF919F918F91CE
:1018F0007F916F915F914F913F912F910F900FBE0C
:101900000F901F901895AC01A0E0B0E09D01A817C2
:10191000B90748F4EFEAF4E08191280F311D1196E0
:10192000A417B507C8F33F70FD01E155FB4FC9018E
:1019300056E0969587955A95E1F7835C80831196DA
:10194000FD01E155FB4F2F733070822F835C808344
:10195000A055BB4F8DE08C93109207018091AF048E
:101960008093C6000895A0E0B0E0E9EBFCE00C94A1
:10197000A67A2C859D850E85BB2483E28093AF04D7
:101980009F599093B0042093B10433E0E32EF12CDF
:10199000002309F49EC0CF84D888BE016D5E7F4FBE
:1019A000A989BA890150109709F493C01097B9F02A
:1019B000F601EB0DF11DB3949081119791F4002382
:1019C00049F1FB016E5F7F4FDB01C080D1806E5F0C
:1019D0007F4F0D90BC91A02DBB24015002C090E020
:1019E00019C01097B9F0F601EB0DF11DB3944081C9
:1019F000119791F4002341F1FB016E5F7F4FDB01F2
:101A0000C080D1806E5F7F4F0D90BC91A02DBB2414
:101A1000015002C040E018C01097B1F0F601EB0D84
:101A2000F11DB3941081119781F4002371F0FB0133
:101A30003296DB01CD90DC90BF016E5F7F4FA081BD
:101A4000B181BB24015001C010E0F701E155FB4F0B
:101A5000892F86958695835C80830894E11CF11C10
:101A6000F701E155FB4F892F99278370907024E08F
:101A7000880F991F2A95E1F755279A0194E036952A
:101A800027959A95E1F7822B835C80830894E11C6B
:101A9000F11CF701E155FB4F4F705070440F551F7B
:101AA000440F551F812F992726E0969587952A95F3
:101AB000E1F7842B835C80830894E11CF11CF7011F
:101AC000E155FB4F1F73135C10830894E11CF11C5C
:101AD0006ACFC7010E94830CE9E00C94C27AA3E0AC
:101AE0007A2F4091C6014650442309F458C0E72F8D
:101AF000FF27EF52FC4F80818D537F5FE72FFF2739
:101B0000EF52FC4F20812D537F5FE72FFF27EF52CD
:101B1000FC4F30813D537F5FE72FFF27EF52FC4F93
:101B200060816D537F5F9927880F991F880F991FD8
:101B3000522F52955F70582B822F99278F7090707B
:101B4000F4E0880F991FFA95E1F7232F2695269543
:101B5000282B832F992783709070E6E0880F991FB8
:101B6000EA95E1F7682B41504F3FC9F0EA2FFF2774
:101B7000EF52FC4F5083AF5F41504F3F81F0EA2F4F
:101B8000FF27EF52FC4F2083AF5F41504F3F39F0AA
:101B9000EA2FFF27EF52FC4F6083AF5FA5CF84EDA4
:101BA00093E09093C5018093C401A350A093C30117
:101BB0000895A2E0B0E0EFEDFDE00C94AC7A8091E6
:101BC000C901882309F41AC40E946F0D8091D203C1
:101BD000823609F0E6C28091D303992780379105B8
:101BE00009F4ABC081379105C4F48A36910509F434
:101BF00043C28B36910544F48B34910571F18636DE
:101C0000910509F470C1CDC28D36910509F469C002
:101C10008E36910509F44DC0C4C28437910541F157
:101C2000853791054CF48137910509F48DC08337D0
:101C3000910509F4E0C0B5C28737910509F4DEC10A
:101C4000883791052CF48537910509F49AC1A9C20A
:101C50008937910509F47FC1A4C2E091C401F091D4
:101C6000C5018081918190938D0180938C0199C2EF
:101C70008091C601A091C401B091C501853140F0A9
:101C800080E1ECEAF3E00D9001928A95E1F70DC056
:101C90008D919D910D90BC91A02D8093AC0390935C
:101CA000AD03A093AE03B093AF0380EF8093C10167
:101CB00047C0809107018823E1F38DE490E09F9372
:101CC0008F9381EB96E09F938F9381E08F938F9317
:101CD0008EE48F930E94B30C8DB79EB707968DBF8D
:101CE00060C2A091C401B091C5011C91113081F472
:101CF0008DE4E1EBF6E00D9001928A95E1F70E9408
:101D00006D2B19838091A8038F7E8093A80301C057
:101D10001982809107018823E1F381E090E09F938D
:101D20008F93CE0101969F938F9381E08F938F9332
:101D30008DE48F930E94B30C09C181E08093CC01A4
:101D40008FEF809305012DC280918102882309F0D5
:101D500028C2E091C401F091C501E0818E2F8A5024
:101D60008A3058F48983882311F481E003C08630D7
:101D700010F085E0898361E00EC08E2F84518A3097
:101D800070F48983882311F481E003C0863010F059
:101D900085E0898360E089810E94EF2B12C0E9838E
:101DA000EF3F19F40E94D02B89838981882311F495
:101DB00081E003C0863010F085E0898389810E942C
:101DC000742A809107018823E1F38EE790E09F93C6
:101DD0008F9382E396E09F938F9381E090E09F93AF
:101DE0008F93CE0101969F938F9382E08F9381E032
:101DF0008F9381E539C12091C4013091C501D9018A
:101E00008C918150853008F045C0F90181818F3572
:101E100009F040C0809181028823E1F52F5F3F4F98
:101E20008EE7E2E3F6E0D9010D9001928A95E1F7A1
:101E3000F90182910E94DF2A809173069927AA27CF
:101E4000BB27BC01CD0124EC39E040E050E00E940A
:101E50000E7ADC01CB018093840190938501A093DD
:101E60008601B0938701809174069927AA27BB2722
:101E7000BC01CD010E940E7ADC01CB018093800170
:101E800090938101A0938201B09383010E94D02B93
:101E9000898301C01982809107018823E1F381E0E1
:101EA00090E09F938F93CE0101969F938F9381E053
:101EB0008F938F9383E58F930E94B30C8DB79EB75A
:101EC00007968DBF80918102882329F46EE670E029
:101ED00089810E94FA3380E00E943406809159067D
:101EE0000E949C755EC180918102882309F059C1CE
:101EF000E091C401F091C501E0818E2F81508530C1
:101F000018F48E2F0E94742A0E94D02B898380910E
:101F100007018823E1F381E090E09F938F93CE0146
:101F200001969F938F9381E08F938F9386E48F9395
:101F30000E94B30C6EE670E089810E94FA3380E063
:101F40000E943406809159060E949C75ADB7BEB7B9
:101F50001796ADBF26C119822981A091C401B09105
:101F6000C501E8E6F7E08D91992787FD909593A349
:101F700082A3822F8F5F8983282F32968C3098F32B
:101F800010C1E091C401F091C50180810E94193116
:101F90008A83882319F481E0898301C019828091A2
:101FA00007018823E1F388E090E09F938F938FEF00
:101FB00096E09F938F9321E030E03F932F938091A1
:101FC000C4019091C5019F938F933F932F93CE01AE
:101FD00002969F938F933F932F93CE01820F931F6F
:101FE0009F938F9384E08F9381E08F9385E58F9308
:101FF0000E94B30CEDB7FEB773963CC08091C3014D
:10200000893008F4CEC02091C4013091C5012F5F02
:102010003F4F88E0AFEFB6E0F90101900D928A954D
:10202000E1F7D9018E910E946C308A83882319F4DC
:1020300081E0898301C01982809107018823E1F33F
:1020400021E030E03F932F93CE0102969F938F9330
:102050003F932F93CE01820F931F9F938F9382E024
:102060008F9381E08F9387E58F930E94B30CEDB738
:10207000FEB73B96EDBF95C080918102882309F0A1
:1020800090C00E9453758983823019F0843009F022
:1020900088C020E430E0F8948091C1008F73809371
:1020A000C1008091C9008F738093C9008091C100E5
:1020B000877E8093C1008091C900877E8093C9008C
:1020C0008091C80087FF03C08091CE00F9CF809136
:1020D000C00087FF03C08091C600F9CFE091C40122
:1020E000F091C501E081E13021F482E08093B801F4
:1020F0002EC0E43611F421E830E081E08093B8018D
:10210000832F99278093CD002093CC008091CD0020
:102110008093C5008091CC008093C4008091CA0058
:102120008F7D8093CA008091CA008F7E8093CA0001
:102130008091C9008B7F8093C9008091CA00846020
:102140008093CA008091CA0082608093CA00809107
:10215000CA00877F8093CA008091C200877F8093E6
:10216000C2008091C9008E7F8093C9008091C10018
:1021700088618093C1008091C90088618093C90003
:102180008091C10080688093C1008091C9008068FF
:102190008093C90010926E0010926F001092700030
:1021A00078948091D30399278436910509F4BBC0B4
:1021B00085369105ACF48136910509F46FC08236FD
:1021C00091052CF48B34910509F45DC00FC1823662
:1021D000910509F470C08336910509F47FC006C1EA
:1021E0008C36910509F4EDC08D3691054CF4873697
:1021F000910509F4F8C08836910509F4B2C0F6C01B
:102200008437910529F08637910509F4E8C0EEC0BE
:102210008091C601A091C401B091C501803140F008
:1022200080E1ECEAF3E00D9001928A95E1F70DC0B0
:102230008D919D910D90BC91A02D8093AC039093B6
:10224000AD03A093AE03B093AF0380910701882341
:10225000E1F31F92809104018F9384E58F930E9494
:10226000B30C8AEF8093C1018FEF8093050180EA60
:102270009FE00E94DF159093BA018093B9010F90FF
:102280000F900F90B3C0E091C401F091C50180811F
:10229000918190938D0180938C01A8C0E091C4013D
:1022A000F091C501808180930601803298F08FE122
:1022B000809306010FC0A091C401B091C5018BE0CD
:1022C000E4ECF3E00D9001928A95E1F78091CD0363
:1022D0008093CD058FEF8093050188C08091BD016B
:1022E0009091BE01892B89F4E091C401F091C50160
:1022F000E081EE2351F08AE0E89FC00111240E94A2
:10230000DF1590939F0380939E03E091C401F091A9
:10231000C50190818AE0989FC00111249093BE016D
:102320008093BD0115C08FEF80930501E091C4013A
:10233000F091C50190818AE0989FC001112490938B
:10234000C0018093BF01892B19F081E08093CE01F9
:1023500080EA9FE00E94DF159093BA018093B90153
:1023600045C08FEF80930501E091C401F091C50154
:10237000908197FD08C082E08093CB011092BC0150
:102380001092BB011AC0909580912902892B8093ED
:10239000290291818AE0989FC00111249093BC0189
:1023A0008093BB0184E08093CB0180EA9FE00E9490
:1023B000DF159093BA018093B90181E08093CF013A
:1023C00015C08FEF80930501E091C401F091C50124
:1023D000808180932A0281E08093D00107C081E050
:1023E0008093CD0103C081E08093D1011092C90197
:1023F0001092C5011092C4011092C301E3E0CE5FB8
:102400000C94C87A982F8091C00085FFFCCF9093E0
:10241000C60008950F931F9388E18093C1008091B7
:10242000C00082608093C0008091C100806880936A
:10243000C1008091C10080648093C10000E010E081
:102440000093C5008AE290E08093C4008091BF01B0
:102450009091C0010E94DF159093A1038093A00387
:102460008CED90E00E94DF159093D0038093CF0312
:1024700082E08093A2031092A30385E08093A603D9
:102480008BE08093A4031092A5031092AA0380917D
:1024900002018093A9031093C5010093C401109217
:1024A000C3011F910F910895A0E1B0E0EAE5F2E1C8
:1024B0000C94AB7A80910701882309F489C280913A
:1024C000B9019091BA010E94E815882361F0109239
:1024D000BC011092BB011092C0011092BF0110927A
:1024E000BE011092BD018091BB019091BC01892B6E
:1024F00041F08091AD049091AE040E94E8158823CC
:1025000029F48091CF01882309F460C080910701EC
:10251000882309F45BC08091CB0101EE15E0843083
:10252000A8F00E942C2080E590E09F938F931F934A
:102530000F9381E08F938F9388E48F930E94B30C65
:102540002DB73EB7295F3F4F2DBF34C010922B02ED
:1025500089EC93E09F938F938FE190E29F938F9309
:10256000E0918E03F0918F03099584E190E09F93B1
:102570008F931F930F9381E090E09F938F938BEC49
:1025800091E09F938F9382E08F9381E08F9388E413
:102590008F930E94B30C8091CB01982F8F5F809313
:1025A000CB012DB73EB7215F3F4F2DBF943010F0C8
:1025B0001092CB018091BB019091BC010E94DF156C
:1025C0009093AE048093AD041092CF018091D0011E
:1025D000882351F180910701882331F10E942C203A
:1025E00080E590E09F938F9381EE95E09F938F938A
:1025F00021E030E03F932F9384E291E09F938F930B
:102600003F932F938AE292E09F938F9383E08F937F
:1026100081E08F938CE48F930E94B30C1092D001D1
:102620008DB79EB70F968DBF8091CD018823D1F0D5
:10263000809107018823B1F08AE090E09F938F9307
:1026400082EA93E09F938F9381E08F938F9386E547
:102650008F930E94B30C1092CD012DB73EB7295F26
:102660003F4F2DBF8091D1018823D9F08091070180
:102670008823B9F08BE090E09F938F9384EC93E0F4
:102680009F938F9381E08F93809104018F9387E4D0
:102690008F930E94B30C1092D1018DB79EB707960D
:1026A0008DBF8091BF019091C001892B41F0809135
:1026B000A0039091A1030E94E815882321F4809142
:1026C000CE01882341F180910701882321F10E94E6
:1026D000043382E490E09F938F938BE895E09F937F
:1026E0008F9381E08F938F9384E48F930E94B30C38
:1026F0001092CE012DB73EB7295F3F4F2DBF80917D
:10270000BF019091C001009731F00E94DF159093B6
:10271000A1038093A0038091BD019091BE01892BFC
:1027200009F497C080919E0390919F030E94E81541
:10273000882309F48EC080910701882309F489C099
:102740008091740890917508909391038093900301
:1027500080917608909177089093930380939203E9
:1027600020915608309157084091580850915908C7
:10277000DA01C90163E0880F991FAA1FBB1F6A9580
:10278000D1F7820F931FA41FB51F820F931FA41FA1
:10279000B51F20913E0130913F0140914001509181
:1027A0004101BC01CD010E94827A309395032093B0
:1027B00094038091A4029091A502A091A602B091E9
:1027C000A70249E0B595A795979587954A95D1F7C2
:1027D000809396038091A0029091A102A091A20201
:1027E000B091A30239E0B595A795979587953A954D
:1027F000D1F7809397038091AC029091AD02A091A4
:10280000AE02B091AF0229E0B595A795979587954F
:102810002A95D1F7809398038EE090E09F938F9351
:1028200080E993E09F938F9381E08F938F9383E46C
:102830008F930E94B30C8091BD019091BE010E94C4
:10284000DF1590939F0380939E038DB79EB70796E5
:102850008DBF809106018F3F79F1992704E0880FA1
:10286000991F0A95E1F787539E4F40E150E0BC0164
:10287000CE0101960E94617880E190E09F938F9352
:10288000CE0101969F938F9381E090E09F938F9369
:1028900086E091E09F938F9382E08F9381E08F9306
:1028A00081E48F930E94B30C8FEF809306012DB7C4
:1028B0003EB7255F3F4F2DBF8091CD058823C9F0DE
:1028C000809107018823A9F081E090E09F938F9386
:1028D0008DEC95E09F938F9381E08F938F9382E4AB
:1028E0008F930E94B30C1092CD058DB79EB70796BB
:1028F0008DBF8091CC018823D1F08091070188237E
:10290000B1F086E490E09F938F9388E697E09F93E1
:102910008F9381E08F938F9380E58F930E94B30C08
:102920001092CC012DB73EB7295F3F4F2DBF80914C
:10293000CF039091D0030E94E815882309F448C082
:1029400080910701882309F443C080917408909115
:1029500075089093BD038093BC0380917608909195
:1029600077089093BF038093BE0380915E028093AB
:10297000C00380915D028093C10388E090E09F9343
:102980008F938CEB93E09F938F9381E08F9383E001
:102990008F938BE68F930E94B30C8091C2032DB767
:1029A0003EB7295F3F4F2DBF853018F086E08093FA
:1029B000C20380919D01882319F483E690E002C050
:1029C00087EE93E00E94DF159093D0038093CF03AE
:1029D000E4E0C05F0C94C77A1F920F920FB60F927B
:1029E00011242F933F935F936F937F938F939F93C4
:1029F000AF93BF93EF93FF9320E08091E201882390
:102A000029F08091E20181508093E201809173036B
:102A1000882319F08150809373038091EA018150DB
:102A20008093EA018F3F09F05BC089E08093EA015F
:102A30008091E8019091E90101969093E9018093DA
:102A4000E801809111018F5F8170809311018823CB
:102A500019F481E08093E701349903C081E0809309
:102A6000E0018091E3019091E401892B21F18091B3
:102A7000E3019091E4010B9750F08091E301909174
:102A8000E4010A979093E4018093E30104C010925B
:102A9000E4011092E3018091E3019091E40120911F
:102AA0000A0130910B0182239323892B11F021E03D
:102AB00008C020E006C08FEF9FEF90930B0180933A
:102AC0000A0180910201222331F08A3011F45A9ACE
:102AD00007C0479A05C08A3011F45A9801C0479838
:102AE0008091E001882309F45AC020919D0122239E
:102AF00009F055C08091460883FF51C086B19927DF
:102B0000FC01E071F07084FF13C08091E5019091A9
:102B1000E60101969093E6018093E5018091E5013D
:102B20009091E601895E9340D0F12093E00137C097
:102B30008091E5019091E601892B69F18091E50191
:102B40009091E6018A56914030F58091E50190918F
:102B5000E60169E270E00E94397A8091E501909186
:102B6000E601860F971F9093E6018093E50180911F
:102B7000E5019091E6010B9750F08091E50190916D
:102B8000E6010A9790938D0180938C0104C0F09325
:102B90008D01E0938C011092E6011092E501FF9106
:102BA000EF91BF91AF919F918F917F916F915F91C5
:102BB0003F912F910F900FBE0F901F90189520916D
:102BC000E8013091E901280F391FC90101960895E4
:102BD0002091E8013091E901821B930B892F9927FD
:102BE0008695807490700895CF93DF930E94DF15CF
:102BF000EC01CE010E94E8158823D9F3DF91CF9133
:102C00000895CF93DF930E94DF15EC0109C08091F6
:102C10001401882329F0909314018FEC80937A009B
:102C2000CE010E94E815982F882389F3DF91CF9178
:102C300008959FB7F8945F983E9A469A8091B000A5
:102C40008F708093B0008091B00083608093B0005B
:102C50008091B1008B738093B1008091B1008B6043
:102C60008093B1001092B2008FEF8093B3008091F7
:102C7000B00080688093B000809170008A7F80935C
:102C80007000809170008260809370009FBF0895F3
:102C90008AE090E00E94DF159093CF058093CE05E7
:102CA00082E085BD83EB84BD8FEF88BD84EB87BD5B
:102CB00086E086BD80916E00816080936E000895ED
:102CC0008091A10620916B0182FF30C09091620635
:102CD0008CE3989FB00111249091610680E5989F44
:102CE000A0011124922F905897FD9D5F9595959581
:102CF00086E09802C0011124209108013091090159
:102D0000281B390B30930901209308014217530700
:102D10002CF05093090140930801089526173707B6
:102D200084F070930901609308010895822F992718
:102D300036E0880F991F3A95E1F790930901809347
:102D400008010895EF92FF920F931F93CF93DF93A3
:102D500080916906E82FFF27EC5BFE4F9681C081CA
:102D600080911001813009F027C180915E02843684
:102D700008F047C0892F992787FD9095A92FB92F73
:102D80002091DC023091DD024091DE025091DF02A1
:102D9000BC01CD010E940E7A97FF04C061587F4F9D
:102DA0008F4F9F4F7B018C0187E015950795F79416
:102DB000E7948A95D1F78C2F992787FD9095A92FB5
:102DC000B92F2091D4023091D5024091D602509172
:102DD000D702BC01CD010E940E7A97FF04C0615852
:102DE0007F4F8F4F9F4FB7E0959587957795679564
:102DF000BA95D1F7F801E701C61BD70BE80BF90B21
:102E000004C0C0E0D0E0E0E0F0E020915903309150
:102E10005A03C901A3E0880F991FAA95E1F7821B05
:102E2000930BAA2797FDA095BA2FC81BD90BEA0BC5
:102E3000FB0B809169019927AA27BB27BC01CD0113
:102E40009E01AF010E940E7A97FF04C061507E4F31
:102E50008F4F9F4FFC01EB0179E0F595E795D795F2
:102E6000C7957A95D1F71091A106609108017091EC
:102E7000090112FF05C070930F0160930E0118C085
:102E800040910E0150910F0180916806282F332741
:102E9000CB01841B950BB9010E944D7A80910E01E4
:102EA00090910F01860F971F90930F0180930E0151
:102EB00010FF14C080910E0190910F0197FD0F96A5
:102EC00064E0959587956A95E1F7AA2797FDA09507
:102ED000BA2FC80FD91FEA1FFB1F15C080910E0122
:102EE00090910F0197FD0F9654E0959587955A950F
:102EF000E1F7AA2797FDA095BA2F8C1B9D0BAE0B6F
:102F0000BF0BFD01EC0120919C06222321F1332708
:102F10008091DC019091DD01829FA001839F500D83
:102F2000929F500D1124CA01AA2797FDA095BA2F90
:102F30008C0F9D1FAE1FBF1F2F5F3F4F442737FDD4
:102F40004095542FBC01CD010E94827A3093DD015F
:102F50002093DC0104C0D093DD01C093DC0180919B
:102F60006106282F3327220F331F220F331F809132
:102F7000DC019091DD01821793077CF0809162065D
:102F8000282F3327220F331F220F331F8091DC019C
:102F90009091DD012817390724F43093DD01209347
:102FA000DC0180910201843108F4FDC080911001A0
:102FB0008F5F80931001F9C0892F992787FD909525
:102FC000A92FB92F2091D4023091D5024091D60279
:102FD0005091D702BC01CD010E940E7A97FF04C028
:102FE00061587F4F8F4F9F4F7B018C0187E0159574
:102FF0000795F794E7948A95D1F78C2F992787FD49
:103000009095A92FB92F2091DC023091DD024091DB
:10301000DE025091DF02BC01CD010E940E7A9B01BD
:10302000AC0197FF04C021583F4F4F4F5F4FC7E09F
:103030005595479537952795CA95D1F72E0D3F1D84
:10304000401F511F809168019927AA27BB27BC0107
:10305000CD010E940E7A97FF04C061507E4F8F4FC2
:103060009F4FFC01EB01B9E0F595E795D795C79522
:10307000BA95D1F780916A019927A6E0880F991F28
:10308000AA95E1F740910C0150910D01209168063D
:103090003327841B950BB9010E944D7A80910C0156
:1030A00090910D01860F971F90930D0180930C0155
:1030B0008091A10681FF14C080910C0190910D01B7
:1030C00097FD0F9674E0959587957A95E1F7AA2775
:1030D00097FDA095BA2FC80FD91FEA1FFB1F15C077
:1030E00080910C0190910D0197FD0F9664E09595EC
:1030F00087956A95E1F7AA2797FDA095BA2F8C1BB3
:103100009D0BAE0BBF0BFD01EC0120919D06222310
:1031100021F133278091DA019091DB01829FA00198
:10312000839F500D929F500D1124CA01AA2797FD2D
:10313000A095BA2F8C0F9D1FAE1FBF1F2F5F3F4F53
:10314000442737FD4095542FBC01CD010E94827A5F
:103150003093DB012093DA0104C0D093DB01C093EC
:10316000DA0180916506282F3327220F331F220FA3
:10317000331F8091DA019091DB01821793077CF075
:1031800080916606282F3327220F331F220F331F0B
:103190008091DA019091DB012817390724F43093EC
:1031A000DB012093DA0110921001E6E0CDB7DEB723
:1031B0000C94C57A1F920F920FB60F9211242F9381
:1031C0003F934F935F938F939F93EF93FF938091E0
:1031D00002019091EB01843108F04CC0992309F071
:1031E00029C18091B00086FF24C08091B0008F7B00
:1031F0008093B0008091DC019091DD0187559E4F56
:103200009093DF018093DE0125E08D3D920718F059
:103210008CED95E005C08757914030F487E791E049
:103220009093DF018093DE018091DE019091DF01B8
:10323000C2C08091B00080648093B0008091670626
:10324000282F33278DED96E0289FA001299F500D50
:10325000389F500D1124CA012091EC013091ED01ED
:10326000821B930B9093DF018093DE0181E08093BA
:103270001001DDC0992309F0DDC08091B00086FF08
:103280009FC08091B0008F7B8093B000E091EE01F1
:1032900020916706EE23D9F433278DED96E0289F21
:1032A000A001299F500D389F500D1124CA01209173
:1032B000EC013091ED01821B930B9093DF01809321
:1032C000DE011092ED011092EC01469AB0C02E176B
:1032D00038F48AE090E09093DF018093DE01A7C08C
:1032E00089EA93E09093DF018093DE018E2F992786
:1032F00083309105D9F08430910534F48130910503
:1033000049F0029761F020C08430910591F0059753
:1033100099F01AC08091DC019091DD0104C0809188
:10332000DA019091DB0187559E4F1DC080912108E5
:1033300005C08091FA0702C080912A089927880F5A
:10334000991F880F991FEFCFFF27EE0FFF1FE85936
:10335000F84F20813181220F331F8091DE0190913F
:10336000DF01820F931F9093DF018093DE01809134
:10337000DE019091DF0155E08D3D950718F08CED51
:1033800095E005C08757914030F487E791E090932E
:10339000DF018093DE012091DE013091DF012C5BA3
:1033A00030403093DF012093DE018091EC01909159
:1033B000ED01820F931F9093ED018093EC0137C0D4
:1033C0008091B00080648093B0008CEB90E090938B
:1033D000DF018093DE018091EC019091ED01845436
:1033E0009F4F9093ED018093EC018091E101882340
:1033F00021F080918202882321F48091E1018230C2
:1034000011F4469801C0469A8091EE018F5F809337
:10341000EE01282F3327809167069927019682179E
:1034200093072CF481E0809310011092EE0181E06B
:103430008093EB012091DE013091DF0141E02F37D5
:10344000340730F08FEF8093B3002F5F30400FC010
:103450002F3F3105C9F0C0F0A9014F5F50404F37F1
:10346000510550F480E88093B300205830403093E9
:10347000DF012093DE0112C08FEF8093B3005093E1
:10348000DF014093DE010AC08091DE018093B3002A
:103490001092DF011092DE011092EB01FF91EF918B
:1034A0009F918F915F914F913F912F910F900FBE00
:1034B0000F901F90189510927C008FEC80937A00EB
:1034C0000895809141026091120170911301209141
:1034D000FB01882379F0CB01AA27BB27332727FDDF
:1034E0003095432F532FBC01CD010E940E7ADC0191
:1034F000CB0116C084E0660F771F8A95E1F7CB01F8
:10350000AA27BB27332727FD3095432F532FBC0114
:10351000CD010E940E7ADC01CB010497A109B1090B
:103520008093F3019093F401A093F501B093F60119
:103530000895CF93DF931092FB010E94611A83E0FC
:1035400090E00E94562AC82FDD27C03FD10508F41D
:103550002A96C7BD8C2F809588BD86E990E00E9491
:10356000011680911801909119018152934010F039
:10357000C0EFD0E0C630D10510F1C7BD8C2F8095CB
:1035800088BD84E690E00E9401168EED93E09F9343
:103590008F9382E092E19F938F93E0918E03F0915D
:1035A0008F03099580911801909119010F900F9048
:1035B0000F900F908152934010F42197DBCFC0936E
:1035C000DE056C2F83E090E00E945E2A80913F062A
:1035D00080FF0AC08091DE058A508C3D28F08091E2
:1035E000A70380648093A7038CE291E00E940116F8
:1035F000DF91CF910895EF92FF921F93CF9310E048
:1036000080ED97E00E94DF157C01CCE8133019F4BF
:10361000CB3008F0C9E010E080910A0290910B02D3
:103620008C5F934024F48091170181500AC08091EF
:103630000A0290910B028750944034F08091170158
:103640008F5F8093170101C011E080910802909173
:1036500009028C5F934024F48091160181500AC0C6
:1036600080910802909109028750944034F0809133
:1036700016018F5F8093160101C01F5F80910602C3
:10368000909107028C5F934024F480911501815042
:103690000AC0809106029091070287509440C4F0BE
:1036A000809115018F5F8093150113C080EE93E028
:1036B0009F938F9382E092E19F938F93E0918E038B
:1036C000F0918F0309950F900F900F900F905FC0AE
:1036D0001F5F82E180933602809130028E7F80935B
:1036E000300285EA8093BC00809117018A3040F453
:1036F0008091A70381608093A7038AE080931701DC
:1037000080911701863F40F08091A70381608093EC
:10371000A70385EF80931701809116018A3040F44A
:103720008091A70382608093A7038AE080931601AB
:1037300080911601863F40F08091A70382608093BC
:10374000A70385EF80931601809115018A3040F41C
:103750008091A70384608093A7038AE0809315017A
:1037600080911501863F40F08091A703846080938B
:10377000A70385EF8093150180913602882339F0E5
:10378000C7010E94E815882309F090CFF5CF109269
:1037900014018FEC80937A00809114018823E1F367
:1037A000CA3020F48AE090E00E940116C15009F06E
:1037B0002DCF86E490E00E940116CF911F91FF90DB
:1037C000EF9008951F920F920FB60F9211242F932E
:1037D0003F934F935F936F937F938F939F93AF9399
:1037E000BF93CF93DF93EF93FF9380911302282F22
:1037F0003327442755278F5F80931302F901223125
:10380000310508F0F0C3E25CFF4F0C94D47A80914C
:1038100078009091790046C080917800909179006D
:1038200054C1809178009091790090931702809311
:1038300016027FC18091E6029091E7022091780004
:1038400030917900821B930B9093D1058093D00522
:103850008091D0059091D105909321028093200210
:1038600086C180917800909179002091E802309192
:10387000E902821B930B9093DD058093DC05809118
:10388000DC059091DD059093230280932202ADC365
:1038900080911A0290911B0220917800309179005A
:1038A000820F931F90931B0280931A0281E09EC3A4
:1038B000809118029091190220917800309179003E
:1038C000820F931F909319028093180284E08EC395
:1038D00080912201909123019C01220F331F280F18
:1038E000391F809178009091790063E070E00E9428
:1038F000397A260F371F36952795369527953093B9
:1039000023012093220185E071C38091780090917A
:1039100079009093D3058093D2058091D205909140
:10392000D3054091E2025091E302841B950B209154
:10393000E102332727FD3095821B930B9093010200
:103940008093000280914102882309F06DC080912C
:1039500000029091010202977CF122E04E3E520754
:103960000CF062C020911402309115022B5F3F4F82
:1039700030931502209314022550304080914A0262
:1039800090914B02845F914030F4215F3F4F309320
:10399000150220931402809114029091150285362D
:1039A00091050CF441C04F5F5F4F5093E302409389
:1039B000E2028456904034C080910002909101024E
:1039C0008F5F9F4F8CF562E0473256076CF1209174
:1039D0001402309115022550304030931502209387
:1039E00014022B5F3F4F80914A0290914B02845FFB
:1039F000914030F42F503040309315022093140240
:103A000080911402909115022FEF8C39920764F483
:103A1000415050405093E3024093E2028C599F4F33
:103A200090931502809314028091000290910102FC
:103A30009C01442737FD4095542F80919C02909122
:103A40009D02A0919E02B0919F02820F931FA41F1E
:103A5000B51F80939C0290939D02A0939E02B09309
:103A60009F0220919C0230919D0240919E025091B4
:103A70009F0257FF04C021503C4F4F4F5F4F7AE0E9
:103A800055954795379527957A95D1F780919C0262
:103A900090919D02A0919E02B0919F02821B930B78
:103AA000A40BB50B80939C0290939D02A0939E0261
:103AB000B0939F022EC1809118029091190220911B
:103AC000780030917900820F931F909319028093B0
:103AD0001802109212028CC2809102018A3071F495
:103AE0008091780090917900209116023091170210
:103AF000820F931F01969695879517C040911602E5
:103B000050911702843158F020917800309179005B
:103B1000240F351F8FEF97E0821B930B06C0809117
:103B2000780090917900840F951F909307028093FD
:103B3000060286E05BC28091E6029091E702209146
:103B4000780030917900821B930B9093D10580937C
:103B5000D0058091D0059091D1052091200230911F
:103B60002102820F931F909305028093040287E045
:103B70003DC280917800909179002091E8023091C7
:103B8000E902821B930B9093DD058093DC05809105
:103B9000DC059091DD052091220230912302820FF5
:103BA000931F90930302809302021FC220911A0276
:103BB00030911B028091780090917900280F391F75
:103BC00030931B0220931A02809102018A3019F46B
:103BD000220F331F04C0220F331F220F331F3093D5
:103BE0001B0220931A0220911A0230911B02C90174
:103BF00037FD079643E0959587954A95E1F79093B1
:103C00000B0280930A0280911C0290911D02820F88
:103C1000931F97FD01969595879590931D0280932C
:103C20001C022091F2023091F302821B930B9093BD
:103C30002101809320012091100230911102809186
:103C4000200190912101280F391F37FF02C02F5FFB
:103C50003F4F35952795309311022093100226CEC1
:103C6000209118023091190280917800909179008A
:103C7000280F391F309319022093180280910201F6
:103C80008A3019F4220F331F04C0220F331F220F72
:103C9000331F30931902209318022091180230919B
:103CA0001902C90137FD0796F3E095958795FA95B6
:103CB000E1F7909309028093080280911E0290918F
:103CC0001F02820F931F97FD0196959587959093FC
:103CD0001F0280931E022091F0023091F102821B9C
:103CE000930B90931F0180931E0120910E0230913F
:103CF0000F0280911E0190911F01280F391F37FF7D
:103D000002C02F5F3F4F3595279530930F022093C8
:103D10000E0283E06BC180917C0290917D02A091A4
:103D20007E02B0917F028093EF019093F001A09307
:103D3000F101B093F2011092130281E0809314011B
:103D40008091F7019091F80101969093F80180938A
:103D5000F7018091780090917900909319018093F8
:103D600018018091180190911901AA27BB27C091D1
:103D70002402D0912502E0912602F0912702C80F7B
:103D8000D91FEA1FFB1FC0932402D0932502E093A2
:103D90002602F0932702809128028F5F80932802E9
:103DA000803108F422C180911A0190911B01A091E9
:103DB0001C01B0911D019C01AD0163E0220F331F76
:103DC000441F551F6A95D1F7281B390B4A0B5B0B13
:103DD0002C0F3D1F4E1F5F1F8091F3019091F40146
:103DE000A091F501B091F601281B390B4A0B5B0B32
:103DF00057FF04C0295F3F4F4F4F5F4F93E05595EA
:103E00004795379527959A95D1F720931A013093C6
:103E10001B0140931C0150931D01C091D405D0910A
:103E2000D505E091D605F091D70580911A019091C2
:103E30001B01A0911C01B0911D01C81BD90BEA0BFD
:103E4000FB0BC0937C02D0937D02E0937E02F09343
:103E50007F022091FC013091FD014091FE015091C3
:103E6000FF0157FF04C0215F3F4F4F4F5F4F84E07A
:103E700055954795379527958A95D1F78091FC01FF
:103E80009091FD01A091FE01B091FF01821B930B67
:103E9000A40BB50B8093FC019093FD01A093FE0150
:103EA000B093FF018091FC019091FD01A091FE0172
:103EB000B091FF018C0F9D1FAE1FBF1F8093FC01AF
:103EC0009093FD01A093FE01B093FF018091FC014E
:103ED0009091FD01A091FE01B091FF01B7FF03C0D9
:103EE0000F96A11DB11DC4E0B595A795979587952F
:103EF000CA95D1F720917C0230917D02281B390BA5
:103F000064E0213036071CF020E034E006C08CEF7E
:103F10002030380714F420E03CEF8091F9019091B3
:103F2000FA018091F9019091FA0197FF03C09095F1
:103F300081959F4FA901F3E0440F551FFA95E1F7D2
:103F40008D5B9240C4F08091F9019091FA019C013F
:103F5000E4E0220F331FEA95E1F7281B390B240F09
:103F6000351F37FF02C0215F3F4F74E0359527951D
:103F70007A95E1F717C08091F9019091FA019C01BF
:103F800065E0220F331F6A95E1F7281B390B240FD8
:103F9000351F37FF02C0215E3F4F45E0359527951D
:103FA0004A95E1F73093FA012093F90180912402B8
:103FB00090912502A0912602B0912702B7FF03C07D
:103FC0000196A11DB11DB595A795979587958093ED
:103FD000240290932502A0932602B093270288E042
:103FE0008093280202C01092130282E08093120292
:103FF0008091120280937C0080911302882319F033
:104000008FEC80937A00FF91EF91DF91CF91BF9178
:10401000AF919F918F917F916F915F914F913F9160
:104020002F910F900FBE0F901F90189590E2E1EE28
:10403000F5E08FE49193815087FFFCCF0895909134
:104040002B02903540F4E92FFF27EF51FA4F808380
:104050009F5F90932B020895AF92BF92CF92DF9211
:10406000FF920F931F93CF93DF932091290220FF9C
:104070000AC080912A02882311F0815002C08091E9
:10408000240180932A0221FF0CC090912A02809182
:104090002401981719F410922A0203C09F5F90938D
:1040A0002A02822F992780FF04C081FF02C010924C
:1040B0002A020E94162080912A02282F33270FE11E
:1040C00010E2C0918E03D0918F038A3098F481E181
:1040D00080932B023F932F9387E194E09F938F93DC
:1040E0001F930F93FE0109952DB73EB72A5F3F4FEF
:1040F0002DBF11C080E180932B023F932F938CE161
:1041000094E09F938F931F930F93FE0109958DB7B2
:104110009EB706968DBF20912A02822F9927AA2743
:10412000BB27FC01429708F0B6C7E05BFF4F0FE1E9
:1041300010E2C0918E03D0918F030C94D47A109228
:104140002B0281E294E09F938F935FE1C52E50E2B2
:10415000D52E1F930F93FE01099584E180932B02C6
:104160000F900F900F900F9086E690E09F938F93A3
:104170001F921F9282E090E09F938F9380910201A3
:104180006AE00E942D7A892F99279F938F938091BF
:1041900002010E942D7A99279F938F9381E394E0E7
:1041A0009F938F931F930F93E0918E03F0918F0352
:1041B000099588E280932B02EDB7FEB73E96EDBFDE
:1041C00082EB96E09F938F938091000199279F93B4
:1041D0008F9389E494E09F938F931F930F93E091C3
:1041E0008E03F0918F0309958091A8032DB73EB7F8
:1041F000285F3F4F2DBF84FF0AC08CE380932B02C2
:1042000087E594E09F938F931F930F93DAC6909165
:10421000A703992351F08CE380932B02892F9927D0
:104220009F938F9384E694E010C19091310299237B
:1042300071F08CE380932B02892F99279F938F93A2
:104240008BE794E09F938F93DF92CF9208C4909175
:104250006003992371F08CE380932B02892F9927B7
:104260009F938F9380E994E09F938F93DF92CF92F7
:104270006DC38091380190913901069708F014C7F9
:104280008CE380932B0281EA94E097C610922B0274
:1042900080917C0290917D02A0917E02B0917F027C
:1042A000BC01CD0125E030E040E050E00E94827A80
:1042B0003F932F938EEA94E09F938F931F930F93D6
:1042C000FE01099584E180932B028DB79EB7069677
:1042D0008DBF8091780290917902A0917A02B0917D
:1042E0007B02BC01CD0125E030E040E050E00E94BF
:1042F000827A3F932F938BEB94E09F938F931F933E
:104300000F93E0918E03F0918F03099588E28093DB
:104310002B02EDB7FEB73696EDBF80911801909154
:1043200019019F938F9388EC94E09F938F931F9331
:104330000F93E0918E03F0918F0309958CE38093A6
:104340002B022DB73EB72A5F3F4F2DBF87B5992768
:104350009F938F9385ED94E09F938F931F930F937B
:1043600078C010922B0282EE94E09F938F934FE1DE
:10437000C42E40E2D42E1F930F93FE01099584E1D1
:1043800080932B020F900F900F900F908091DC0282
:104390009091DD02A091DE02B091DF02B7FF04C070
:1043A00081509C4FAF4FBF4F3AE0B595A795979579
:1043B00087953A95D1F7BF93AF939F938F938FEEE5
:1043C00094E09F938F93DF92CF92E0918E03F091D0
:1043D0008F03099588E280932B02EDB7FEB73896DC
:1043E000EDBF8091D4029091D502A091D602B091F8
:1043F000D702B7FF04C081509C4FAF4FBF4F2AE098
:10440000B595A795979587952A95D1F7BF93AF93C3
:104410009F938F938EEF94E09F938F93DF92CF9231
:10442000E0918E03F0918F0309958CE380932B022A
:104430002DB73EB7285F3F4F2DBF80910208909166
:1044400003089F938F938DE095E09F938F93DF9266
:10445000CF92E0918E03F0918F0309958DB79EB7AF
:1044600006968DBF21C691E0F92EC1E0D0E00AE6A4
:1044700017E09F2D969584E1989FC00111248093A9
:104480002B02F801828193819F938F932196DF9372
:10449000CF932197808191819F938F93DF93CF93C7
:1044A0008CE195E09F938F938FE190E29F938F93A0
:1044B000E0918E03F0918F0309952DB73EB7245FED
:1044C0003F4F2DBF32E0F30E22960C5F1F4F88E066
:1044D0008F1578F6E9C510922B0280913406E82FEB
:1044E000FF27EE0FFF1FE859F84F808191819F93BE
:1044F0008F9380913306E82FFF27EE0FFF1FE859B7
:10450000F84F808191819F938F938EE295E09F93E6
:104510008F931F930F93FE01099584E180932B02E3
:10452000EDB7FEB73896EDBF80913606E82FFF272E
:10453000EE0FFF1FE859F84F808191819F938F9371
:1045400080913506E82FFF27EE0FFF1FE859F84F3F
:104550008081918181589F4F9F938F938EE395E047
:104560009F938F931F930F93E0918E03F0918F038E
:10457000099588E280932B022DB73EB7285F3F4F05
:104580002DBF80913806E82FFF27EE0FFF1FE85957
:10459000F84F8081918181589F4F9F938F93809195
:1045A0003706E82FFF27EE0FFF1FE859F84F8081ED
:1045B000918181589F4F9F938F938EE495E09F93B5
:1045C0008F931F930F93E0918E03F0918F030995C2
:1045D0008CE380932B028DB79EB708968DBF809198
:1045E0003A06E82FFF27EE0FFF1FE859F84F8081AA
:1045F000918181589F4F9F938F9380913906E82F27
:10460000FF27EE0FFF1FE859F84F808191818158F5
:104610009F4F9F938F938EE595E023C110922B02BD
:104620008EE695E09F938F938FE1C82E80E2D82E7F
:104630001F930F93FE01099584E180932B020F9045
:104640000F900F900F908091F2029091F3029C01D5
:1046500097FF02C0215F3F4F207F821B930B97FD86
:104660000196959587959F938F938091F2029091F3
:10467000F30297FD0F96B4E095958795BA95E1F70B
:104680009F938F932091F2023091F30237FF02C083
:10469000295F3F4FA3E035952795AA95E1F78091D3
:1046A0000A0290910B02821B930B9F938F938CE7CE
:1046B00095E09F938F93DF92CF92E0918E03F091DC
:1046C0008F03099588E280932B022DB73EB7265FB2
:1046D0003F4F2DBF8091F0029091F1029C0197FF16
:1046E00002C0215F3F4F207F821B930B97FD0196F5
:1046F000959587959F938F938091F0029091F10209
:1047000097FD0F96E4E095958795EA95E1F79F93DD
:104710008F932091F0023091F10237FF02C0295FA0
:104720003F4F73E0359527957A95E1F78091080220
:1047300090910902821B930B9F938F938EE895E0D3
:104740009F938F93DF92CF92E0918E03F0918F032E
:1047500009958CE380932B028DB79EB70A968DBF87
:104760008091EE029091EF0297FD019695958795C5
:104770009F938F938091EE029091EF022091060219
:1047800030910702821B930B9F938F9380EA95E0F1
:104790009F938F93DF92CF92E0918E03F0918F03DE
:1047A0000995EDB7FEB7389662C110922B028FEAD9
:1047B00095E09F938F931F930F93FE01099584E1DA
:1047C00080932B020F900F900F900F908091E80232
:1047D0009091E9029F938F9380910202909103023E
:1047E0009F938F938CEB95E09F938F931F930F93E1
:1047F000E0918E03F0918F03099588E280932B025C
:104800002DB73EB7285F3F4F2DBF8091E6029091B4
:10481000E7029F938F9380910402909105029F93EA
:104820008F938BEC95E09F938F931F930F93E09161
:104830008E03F0918F0309958CE380932B028DB743
:104840009EB708968DBF8091E2029091E3029F93FC
:104850008F9380910002909101029F938F938AED34
:1048600095E09F938F931F930F9396CF10922B02F7
:1048700080912201909123016AE070E00E944D7ABC
:104880009F938F9380912201909123016AE070E0C1
:104890000E944D7A7F936F9389EE95E09F938F935B
:1048A0001F930F93FE01099584E180932B022DB78E
:1048B0003EB7285F3F4F2DBF8091DB089091DC0809
:1048C0006AE070E00E94397A9F938F938091DB08B1
:1048D0009091DC086AE070E00E94397A7F936F93D0
:1048E0008DEF95E09F938F931F930F93E0918E032D
:1048F000F0918F03099588E280932B028DB79EB7C4
:1049000008968DBF8091DD089091DE089F938F936C
:1049100081E196E09F938F931F930F93E0918E0315
:10492000F0918F0309958CE380932B02EDB7FEB7CE
:104930003696EDBF8091DF089091E0089F938F93AA
:1049400081E296E09F938F931F930F93E0918E03E4
:10495000F0918F0309952DB73EB72A5F3F4F47C1AE
:1049600010922B0283E396E09F938F931F930F93F4
:10497000FE01099588E280932B020F900F900F9013
:104980000F908091820299279F938F938CE396E0FA
:104990009F938F931F930F93E0918E03F0918F035A
:1049A00009958CE380932B028DB79EB706968DBF39
:1049B00080916707992701979F938F938CE496E0E6
:1049C0004AC010922B028CE596E09F938F931F9321
:1049D0000F93FE01099584E180932B020F900F90B5
:1049E0000F900F9080918C0190918D019F938F93E8
:1049F00084E696E09F938F931F930F93E0918E032D
:104A0000F0918F03099588E280932B022DB73EB772
:104A10002A5F3F4F2DBF80910208909103089F931A
:104A20008F9382E796E09F938F931F930F93E0916C
:104A30008E03F0918F0309958CE380932B028DB741
:104A40009EB706968DBF80919A0290919B029F938C
:104A50008F9380E896E09F938F931F930F93E0913D
:104A60008E03F0918F030995EDB7FEB73696EDBF33
:104A70001BC353E8C52E52E0D52E20E030E0E901FB
:104A800043E0F42EC0932B02F60181916F01992728
:104A90009F938F9389010F5F1F4F1F930F938EE892
:104AA00096E09F938F938FE190E29F938F93E09195
:104AB0008E03F0918F0309952DB73EB7285F3F4FC6
:104AC0002DBFFA9464969801F7FEDCCFEDC227E87B
:104AD000C22E22E0D22EC0E0D0E08E0193E0F92E6B
:104AE00000932B02F60181916F0199279F938F9379
:104AF0002596DF93CF938BE996E09F938F938FE179
:104B000090E29F938F93E0918E03F0918F0309952C
:104B10002DB73EB7285F3F4F2DBFFA940C5E1F4F55
:104B20002497F7FEDDCFC0C210922B0288EA96E0F0
:104B30009F938F938FE1C82E80E2D82E1F930F93FF
:104B4000FE01099584E180932B020F900F900F9046
:104B50000F9080916B0199279F938F9380EB96E044
:104B60009F938F931F930F93E0918E03F0918F0388
:104B7000099588E280932B028DB79EB706968DBF6C
:104B80008091DC019091DD0197FD039695958795C5
:104B9000959587959F938F938EEB96E09F938F9338
:104BA000DF92CF92E0918E03F0918F0309958CE311
:104BB00080932B02EDB7FEB73696EDBF809162066B
:104BC00099279F938F938091610699279F938F9345
:104BD0008CEC96E09F938F93DF92CF92E0918E03BF
:104BE000F0918F0309952DB73EB7285F3F4F2DBF3A
:104BF0005BC210922B028AED96E09F938F93AFE1F8
:104C0000CA2EA0E2DA2E1F930F93FE0109950F9092
:104C10000F900F900F90C7E0D7E000E010E0F2E0B7
:104C2000FF2E802F8C5E80932B028B8D99278F77A0
:104C300090709F938F938B8999278F7790709F9314
:104C40008F938B8599278F7790709F938F938B810C
:104C500099278F7790709F938F938AEE96E09F931A
:104C60008F93DF92CF92E0918E03F0918F0309959D
:104C70008DB79EB70C968DBFFA940C5E1F4FA09611
:104C8000F7FECFCF11C210922B028BEF96E09F93CD
:104C90008F93EFE1CE2EE0E2DE2E1F930F93FE0105
:104CA00009950F900F900F900F90C7E0D7E000E0AC
:104CB00010E072E0F72E802F8C5E80932B028F8D98
:104CC000992787FD90959F938F938F89992787FDCB
:104CD00090959F938F938F85992787FD90959F93AC
:104CE0008F938F81992787FD90959F938F938AE06B
:104CF00097E09F938F93DF92CF92E0918E03F09194
:104D00008F030995EDB7FEB73C96EDBFFA940C5EA4
:104D10001F4FA096F7FECFCFC7C110922B028BE199
:104D200097E09F938F936FE1A62E60E2B62E1F93BC
:104D30000F93FE01099587E480932B020F900F904B
:104D40000F900F9086E297E09F938F931F930F939E
:104D5000E0918E03F0918F030995FF240F900F903F
:104D60000F900F9054E0C52ED12CC7E0D7E000E0A3
:104D700010E0802F8C5E80932B028D8D99279F935E
:104D80008F938D8999279F938F938D8599279F93D3
:104D90008F938D8199279F938F9380E397E09F93C3
:104DA0008F93BF92AF92E0918E03F0918F0309959C
:104DB0008091310699272DB73EB7245F3F4F2DBF15
:104DC000C816D9060CF070C1F3940C5E1F4FA09664
:104DD00084E090E0C80ED91E92E09F1550F664C1A1
:104DE00010922B0281E497E09F938F934FE1C42EA2
:104DF00040E2D42E1F930F93FE01099584E1809326
:104E00002B020F900F900F900F9080912207881F18
:104E10008827881F97E0899FC00111248D969F9352
:104E20008F9380911A07881F8827881F96E0899F93
:104E3000C00111248D969F938F9380911207881F34
:104E40008827881F95E0899FC00111248D969F9324
:104E50008F9380910A07881F8827881F9927880FBA
:104E6000991F880F991F8D969F938F9380E597E0E8
:104E70009F938F931F930F93E0918E03F0918F0375
:104E8000099588E280932B02EDB7FEB73C96EDBF03
:104E900080914207881F8827881F9BE0899FC00157
:104EA00011248D969F938F9380913A07881F8827AE
:104EB000881F9AE0899FC00111248D969F938F933C
:104EC00080913207881F8827881F99E0899FC00139
:104ED00011248D969F938F9380912A07881F88278E
:104EE000881F992723E0880F991F2A95E1F78D964F
:104EF0009F938F9384E697E09F938F931F930F93D5
:104F0000E0918E03F0918F0309958CE380932B023F
:104F10002DB73EB7245F3F4F2DBF80914A07881FB2
:104F20008827881F9CE0899FC00111248D969F933C
:104F30008F9388E797E09F938F931F930F93E09150
:104F40008E03F0918F03099580915207EDB7FEB75C
:104F50003696EDBF87FF12C080E480932B0289E86C
:104F600097E09F938F931F930F93E0918E03F0919F
:104F70008F0309950F900F900F900F9080915A0713
:104F800087FF12C084E480932B028CE897E09F9304
:104F90008F93DF92CF92E0918E03F0918F0309956A
:104FA0000F900F900F900F908091620787FF7CC049
:104FB00088E480932B028FE897E09F938F93DF9292
:104FC000CF92E0918E03F0918F0309950F900F908F
:104FD0000F900F9069C010922B0282E997E09F9387
:104FE0008F931F930F93FE01099584E180932B0209
:104FF0000F900F900F900F908091B2019091B3019C
:105000009F938F9380EA97E09F938F931F930F93C3
:10501000E0918E03F0918F03099588E280932B0233
:105020002DB73EB72A5F3F4F2DBF8091B4019091BD
:10503000B5019F938F938DEA97E09F938F931F9372
:105040000F93E0918E03F0918F03099589E480938B
:105050002B028DB79EB706968DBF8AEB97E09F9384
:105060008F931F930F93E0918E03F0918F03099517
:10507000809129020F900F900F900F9083FF14C022
:105080001092B5011092B40160E070E08EE090E003
:105090000E946F2A09C080912401281719F4215019
:1050A0002093240110922A0210922902DF91CF91BD
:1050B0001F910F91FF90DF90CF90BF90AF90089518
:1050C000F999FECF92BD81BDF89A80B599270895D0
:1050D000F999FECF1FBA92BD81BD60BD0FB6F8949D
:1050E000FA9AF99A0FBE08954AEA20E030E02617AE
:1050F000370740F4FC018191480F2F5F3F4F26177F
:105100003707C8F3842F99270895EAEA40E050E072
:105110004617570778F49C01F999FECF32BD21BD9F
:10512000F89A80B5E80F4F5F5F4F2F5F3F4F4617EC
:10513000570790F38E2F9927089581E080933506C5
:1051400082E08093340683E08093330684E080938A
:10515000360685E08093370686E08093380687E040
:105160008093390688E080933A0689E080933B0675
:105170008AE080933C068BE080933D068CE0809330
:105180003E0608958FE5809332068CE0E4EAF6E06F
:1051900011928A95E9F780910201843150F08AE0FA
:1051A00080935206109276068BE180934E068EE431
:1051B0000AC083E08093520680E2809376068EE1F7
:1051C00080934E0685E5809373068093740680E293
:1051D000809375061092A0068AE680933F0682E7C8
:1051E0008093A20680E58093A30666E0609359064B
:1051F000109296061092930658E050934C0646EE95
:1052000040934D0680E480934F069EE190934006C4
:1052100085E0809342062FE0209343069093410659
:10522000109245065093460684E1809347061092FB
:105230004806109299062093440610929E068CE030
:1052400080939F0610925B0610925C0610925D069A
:1052500010925E06109278061092790610927A06E5
:1052600010927B0690E890935F0632E330936006DD
:10527000E2E0E093A10688E1809361064093620634
:1052800083E0809367064DE740936A0640936B0680
:1052900040936C069093630675E57093640686E40C
:1052A000809365068CED809366068CE38093680698
:1052B000109269069AEA90937C068CEC80937E06A5
:1052C000109280069093810698E290937D069093C9
:1052D0007F061092820630936D062AE520936E06B3
:1052E00030936F066093830684E6809384068093F0
:1052F00085062093860688E78093870690938B0621
:105300008BE4809388067093890680938A06609365
:105310008C0650938D0630938E068AE280938F061A
:1053200085EF809390068CE880939106E093920637
:10533000109294061092950681E28093560681E4BD
:10534000809357062093580610929706109298065D
:1053500086E980939A064093700684E380937106F1
:1053600010929B0610929C0610929D0608950E9432
:10537000C2288AE08093490680E180934A0626E0AD
:1053800020934B069AE59093500688E78093510648
:1053900090935306809354062093550680E28093A1
:1053A0005A068CE3809372068BE48093770686E43A
:1053B00091E6A3E7B4E78093A4069093A506A09393
:1053C000A606B093A7066EE770E082E396E00E941F
:1053D00074288093B0060895CF93DF930E94C2286B
:1053E00088E08093490630E130934A0626E0209316
:1053F0004B0694E69093500688E78093510690936D
:105400005306809354062093550630935A0686E43B
:105410008093720680937706A4EAB6E085E0E5E221
:10542000F1E0ED01019009928A95E1F76EE770E0F5
:10543000CD01825790400E9474288093B006DF917E
:10544000CF9108950E94C22826E0209349068AE061
:1054500080934A0684E080934B0694E6909350062E
:1054600088E78093510690935306809354062093C7
:10547000550680E180935A0686E4809372068093F5
:10548000770685E491E6A3E7B9E78093A4069093B5
:10549000A506A093A606B093A7066EE770E082E388
:1054A00096E00E9474288093B0060895F999FECF83
:1054B00092BD81BDF89A80B599270895F999FECFDC
:1054C0001FBA92BD81BD60BD0FB6F894FA9AF99AE1
:1054D0000FBE089560E678E20E949C78089548E641
:1054E00058E20E94D6780895EF92FF920F931F938F
:1054F000CF93C82F8150853008F0C3E08FE7C89F55
:105500008001112485EEE82E8FEFF82EE00EF11EBB
:105510006EE770E0C7010E948528682F98012D5919
:105520003F4F8FB39927AC014270507081FDF9CF86
:1055300032BD21BDF89A80B5861711F0CA0121C08D
:105540008FB399279C012270307081FDF9CFF2BC96
:10555000E1BCF89A80B58F3511F0C90112C08FE710
:10556000C89FC00111244B9720E638E24FE750E076
:10557000BC0182E396E00E9477780E94B26981E0E4
:1055800090E0CF911F910F91FF90EF900895282FF9
:10559000863010F025E003C0882309F421E0209331
:1055A0000001F999FECF1FBA82E090E092BD81BD63
:1055B00020BD0FB6F894FA9AF99A0FBE0895CF93CA
:1055C000C82F809132068F3509F04FC0C63010F0D9
:1055D000C5E003C0CC2309F448C00E940077809145
:1055E000A30682FF07C080915706843618F080E535
:1055F000809357066EE770E082E396E00E9474287D
:105600008093B0068FE7C89FC001112428E638E2D6
:105610004FE750E062E376E04B970E94B47828E6CB
:1056200038E24CE050E063E376E080E590E00E94F1
:10563000B4786CE070E083E396E00E947428282F31
:10564000F999FECF1FBA8CE590E092BD81BD20BDD7
:105650000FB6F894FA9AF99A0FBE8C2F0E94C72AB7
:105660000E94B26981E090E002C080E090E0CF91BA
:1056700008956DE470E088EE93E00E948528482F3D
:105680008FB399279C012270307081FDF9CF85E39B
:1056900094E092BD81BDF89A80B5841779F48FB3F8
:1056A00099279C012270307081FDF9CF88EE93E03C
:1056B00092BD81BDF89A80B5813011F0C90108957D
:1056C00020E638E24EE450E068EE73E081EB96E0CD
:1056D0000E94777881E090E008958091B106813052
:1056E000A9F46DE470E081EB96E00E947428809349
:1056F000FE0628E638E24EE450E061EB76E088EE04
:1057000093E00E94B47881E090E0089580E090E01A
:105710000895CF93DF9381E08093B106E1EBF6E04B
:105720008FE0158616861786108A8150349687FF7B
:10573000F8CF80E48093BE068093BF061092C00627
:105740008093C1068093C20690EC9093C30610929A
:10575000C4068093C5068093C6061092C706909330
:10576000C8069093C9068093CA061092CB06809310
:10577000CC069093CD06A2EBB6E08CE0EBE2F1E034
:10578000ED01019009928A95E1F76DE470E0CD0199
:1057900001970E9474288093FE06DF91CF910895AF
:1057A000F999FECF82E090E092BD81BDF89A80B574
:1057B000282F863078F023E0322FF999FECF1FBAD8
:1057C00082E090E092BD81BD30BD0FB6F894FA9AA8
:1057D000F99A0FBE20930001822F992708951F93F5
:1057E000CF93C82F162F863010F0C5E003C0882352
:1057F00009F4C1E08C2F99278230910541F0833064
:10580000910544F4019731F40E94B72905C00E9424
:10581000EC2902C00E94222A1123E1F06CE070E022
:1058200080E590E00E948528282FF999FECF8CE52D
:1058300090E092BD81BDF89A80B5821759F420E6B8
:1058400038E24CE050E060E570E083E396E00E94CF
:10585000777802C00E949D288C2F0E94DF2ACF916A
:105860001F910895DF92EF92FF920F931F93CF93B2
:10587000FF24DF2CEF2C81E090E00E94562A8F3528
:1058800011F031E0E32E6CE070E080E590E00E94E2
:105890008528C82FF999FECF8CE590E092BD81BD97
:1058A000F89A80B58C1711F421E0D22EC1E001E006
:1058B00010E0EE2029F48C2F0E94742A8823B9F579
:1058C00091E0F92E1F930F9382EC97E09F938F93B3
:1058D00082E092E19F938F93E0918E03F0918F038A
:1058E00009952DB73EB72A5F3F4F2DBF01301105F7
:1058F00021F00230110521F006C00E94B72905C031
:105900000E94EC2902C00E94222ADD2059F020E6E4
:1059100038E24CE050E060E570E083E396E00E94FE
:10592000777802C00E949D288C2F0E94DF2ACF5FCB
:105930000F5F1F4FC63008F4BCCFFF2019F083E083
:105940000E94C72A0E94D02BC82F0E94742A8C2F35
:1059500099279F938F9388EE97E09F938F9302E010
:1059600012E11F930F93E0918E03F0918F0309953D
:1059700081E090E00E94562A2DB73EB72A5F3F4F44
:105980002DBF8F3F21F00E94392B882399F481E0AD
:1059900098E09F938F931F930F93E0918E03F09164
:1059A0008F0309950E94892B0E946D2B0F900F90F9
:1059B0000F900F90EE2029F06FE581E090E00E94BB
:1059C0005E2A1092310690E0EEEBF6E0CFE08081A7
:1059D000349618160CF49F5FC150C7FFF8CF909310
:1059E0003106892F99279F938F9382EB96E09F939F
:1059F0008F9382E298E09F938F931F930F93E09190
:105A00008E03F0918F0309950E94F4058DB79EB720
:105A100008968DBFCF911F910F91FF90EF90DF906F
:105A20000895982F2FB7F8943998389A88B18360E1
:105A300088B98091B9008C7F8093B9008AE2809305
:105A4000B800109236021092340210923302992359
:105A500079F0E7E0F7E08BE0108211821282138286
:105A600014821582168217828150389687FFF4CFF0
:105A700078942FBF08951092360284E98093BC0079
:105A800080E88093BC001092BD001092BA00109282
:105A9000BB001092B9001092B8001092320280E060
:105AA0000E94112D1092BB0085E88093BC0080916C
:105AB000300282608093300208951F920F920FB6D9
:105AC0000F9211242F933F934F935F938F939F9344
:105AD000EF93FF9380913602282F332744275527D1
:105AE0008F5F80933602F9012731310508F0D1C26A
:105AF000EE59FF4F0C94D47A81E08093320209C0B2
:105B0000809134028C3090F4809134028F5F8093C6
:105B1000340280913402E82FFF27EE0FFF1FEE0FB3
:105B2000FF1FEF54F94F8585181654F78091340202
:105B30008C3070F010922F0210922E0210923402CC
:105B400085E08093360280913302880F8D5A04C01D
:105B500080913402880F8E5A8093BB0085E88EC2F4
:105B600080913402E82FFF2783E0EE0FFF1F8A9514
:105B7000E1F7E95FF84F81818093BB0085E880936E
:105B8000BC0080913402E82FFF27EE0FFF1FEE0FBD
:105B9000FF1FEE0FFF1FE95FF84F808180FF91C06C
:105BA00080913402E82FFF27EE0FFF1FEE0FFF1F3B
:105BB000EE0FFF1FE95FF84F8281882329F0809163
:105BC0003106873008F47BC280912E0290912F021B
:105BD000892B09F074C280912C0290912D02892B9F
:105BE00009F06DC26EC08091340221E030E002C045
:105BF000220F331F8A95E2F780912C0290912D029B
:105C000028233923232B79F080913402E82FFF27B2
:105C1000EE0FFF1FEE0FFF1FEE0FFF1FE95FF84FA4
:105C200080E184830DC080913402E82FFF27EE0FBE
:105C3000FF1FEE0FFF1FEE0FFF1FE95FF84F1482EB
:105C400080913402E82FFF2753E0EE0FFF1F5A9593
:105C5000E1F7E95FF84F8481282F332743E0220FD3
:105C6000331F4A95E1F780913402E82FFF2733E094
:105C7000EE0FFF1F3A95E1F7E95FF84F82818770D9
:105C8000822B8093BB0085E88093BC002091340276
:105C900081E090E002C0880F991F2A95E2F72091D9
:105CA0002E0230912F0282239323892B51F08FEF04
:105CB00096E090933A028093390288E080933B0209
:105CC000FEC184E098C1E0913902F0913A028191DD
:105CD0008093BB0085E88093BC00F0933A02E09388
:105CE000390280913B02815080933B02882309F462
:105CF000E6C183E080C18091B900803349F580918D
:105D00003702882329F4809134028F5F8093370211
:105D100080913402E82FFF2793E0EE0FFF1F9A9542
:105D2000E1F7E95FF84F838199278F7790708F377C
:105D3000910574F480913402E82FFF2783E0EE0F81
:105D4000FF1F8A95E1F7E95FF84F83818F5F8383B7
:105D50001092360284E98093BC008AE090E0909330
:105D6000390180933801809134028F5F809334022F
:105D7000109236027DC18091B9008034C9F18091C2
:105D80003302E82FFF27EE0FFF1FEE0FFF1FEE0F6E
:105D9000FF1FE95FF84F83818F7783838091330200
:105DA0008F5F80933302809133028C30A0F0109289
:105DB000330210922D0210922C02809138028F5FD4
:105DC000809338028C3038F0109238028091300283
:105DD0008D7F809330028091300281608093300209
:105DE0001092360284E98093BC001092320283C084
:105DF00080913302E82FFF27EE0FFF1FEE0FFF1FEA
:105E0000EE0FFF1FE95FF84F8381806883838091E5
:105E10003302E82FFF27EE0FFF1FEE0FFF1FEE0FDD
:105E2000FF1FE95FF84F808180FF3FC08091330200
:105E3000E82FFF27EE0FFF1FEE0FFF1FEE0FFF1FD4
:105E4000E95FF84F848199270097C9F0409709F0DE
:105E500049C08FEF96E090933A028093390288E030
:105E600080933B0280913302E82FFF2753E0EE0F2F
:105E7000FF1F5A95E1F7E95FF84F148233C0809114
:105E80003302992743E0880F991F4A95E1F7845F11
:105E9000984F90933A028093390290913302809107
:105EA00038029817E1F483E01BC0809133029927F0
:105EB00033E0880F991F3A95E1F7845F984F9093EC
:105EC0003A02809339028091300281FD06C09091A0
:105ED000330280913802981711F482E001C081E00A
:105EE00080933B0280913B02813011F485E801C030
:105EF00085EC8093BC008091370280933102109230
:105F00003702DDC0E0913902F0913A028091BB0086
:105F100080838091390290913A02019690933A02DF
:105F20008093390280913B02815080933B02823002
:105F300010F085EC5DC0813011F485E859C0809186
:105F4000300281FF2DC08091490280FD1DC08091EB
:105F50003302E82FFF2723E0EE0FFF1F2A95E1F71A
:105F6000E95FF84F86818A3F79F480913302E82F08
:105F7000FF2793E0EE0FFF1F9A95E1F7E95FF84FD7
:105F80008081816080830CC080913302E82FFF27DD
:105F900083E0EE0FFF1F8A95E1F7E95FF84F10826B
:105FA000809133028F5F80933302809133028C3073
:105FB000A0F01092330210922D0210922C028091C8
:105FC00038028F5F809338028C3038F0109238029C
:105FD000809130028D7F809330021092360284E9E6
:105FE0008093BC008091300281608093300265C054
:105FF0008093BC0086E08093360261C088E9ACCD16
:1060000080913502880F805FA7CD80913502992756
:106010008130910561F0823091051CF4892B21F0CB
:106020004EC0029739F04BC08091170195CD8091F9
:10603000160192CD809115018FCD80E88DCD109203
:10604000360284E98093BC00109232028AE090E02C
:10605000909339018093380180913502823088F421
:10606000809135028F5F8093350282E18093360202
:10607000809130028E7F8093300285EA8093BC004D
:106080001EC01092350280913002816080933002F0
:1060900016C01092360284E98093BC0080913002D1
:1060A0008160809330028AE090E090933901809380
:1060B0003801109234021092330210923202FF9192
:1060C000EF919F918F915F914F913F912F910F9001
:1060D0000FBE0F901F9018951F93CF93DF93182F2B
:1060E00080918102882321F48091C101882319F0D5
:1060F00081E090E09AC01D3008F095C01123B1F006
:10610000E12FFF2723E0EE0FFF1F2A95E1F7E95F5C
:10611000F84F35978081359688230CF084C03897E6
:10612000808180FD03C083E090E07FC08091FF0606
:1061300099278B709070029719F084E090E075C0F9
:1061400067E070E08FEF96E00E9474289091060758
:10615000891719F085E090E068C080ED97E00E9413
:10616000DF15EC018091300280FD05C0CE010E9458
:10617000E8158823B9F3112319F48FEF90E00BC0D1
:10618000212F33272150304081E090E002C0880F5A
:10619000991F2A95E2F790932F0280932E02A1E097
:1061A000B0E0E7E0F7E040E050E06BE0CD01042E26
:1061B00002C0880F991F0A94E2F720912E023091B5
:1061C0002F0282239323892B11F0118212826150B6
:1061D0004F5F5F4F389667FFE9CF109234021092FD
:1061E0003602809130028E7F8093300285EA809360
:1061F000BC008091300280FD05C0CE010E94E815F0
:106200008823B9F380912E0290912F02892B29F0D7
:10621000CE010E94E815882311F380912E029091FF
:106220002F02009711F082E090E0DF91CF911F9153
:1062300008950F931F93CF93DF93982F809181023E
:10624000882321F48091C101882319F081E090E036
:1062500095C09D30A0F4992319F486E090E08EC09B
:10626000C92FDD27FE0133E0EE0FFF1F3A95E1F75E
:10627000E95FF84F35978081359687FD03C082E04E
:1062800090E07CC03897808180FD03C083E090E07F
:1062900075C080ED97E00E94DF158C01809130027F
:1062A00080FD05C0C8010E94E8158823B9F3219735
:1062B00021E030E0C90102C0880F991FCA95E2F7BA
:1062C00090932D0280932C02D901E7E0F7E040E0A3
:1062D00050E06BE0CD01042E02C0880F991F0A9494
:1062E000E2F720912C0230912D0282239323892BF7
:1062F00011F01182128261504F5F5F4F389667FF35
:10630000E9CF109233021092FF0610920607109206
:106310003602809130028E7F8093300285EA80932E
:10632000BC008091300280FD05C0C8010E94E815C4
:106330008823B9F380912C0290912D02892B29F0AA
:10634000C8010E94E815882311F38091FF06992760
:106350008B709070029719F084E090E00FC067E0B6
:1063600070E08FEF96E00E947428909106078917DD
:1063700019F085E090E002C080E090E0DF91CF91DD
:106380001F910F910895CF93DF9380E021E83FEFB5
:10639000CEEAD7E0E8E6F7E0DF01853020F4119699
:1063A0001C921E9202C03183208319821882229689
:1063B0008F5F12963296833280F38FE790E090934E
:1063C000A7078093A60781E89FEF9093A507809386
:1063D000A4071092A9071092A8071092EF0210923A
:1063E000EE021092F1021092F0021092F30210925B
:1063F000F202DF91CF9108951F920F920FB60F9284
:1064000011240F931F932F933F934F935F936F9399
:106410007F938F939F93AF93BF93CF93DF93EF932C
:10642000FF93409186005091870080913D029091AA
:106430003E02481B590B80918600909187009093F3
:106440003E0280933D02CA018D549440A0913F02C8
:10645000B0914002835F9A4178F480913F0280932B
:106460006707149714F010923C0181E090E090933C
:10647000400280933F02B3C0A131B1050CF0AFC020
:10648000CA018B5F9040845B914008F085C0809189
:106490003A0190913B01481B590BE0919B06EE237A
:1064A00051F0FF27EE0FFF1FE859F84F80819181CF
:1064B00084369105ECF4FD01EA0FFB1FE859F84F13
:1064C00080819181FA01E81BF90BCF01F7FF03C02E
:1064D000909581959F4F06975CF480918202883C4D
:1064E00020F480918202865F01C088EC8093820252
:1064F000FD01EA0FFB1FE859F84F808191819C0153
:10650000220F331F280F391F240F351F37FF02C0FA
:106510002D5F3F4FE901D595C795D595C795CA0120
:1065200001968C179D0714F4219706C041505040E6
:10653000C417D5070CF4219680918202833CD8F0D1
:106540008D010A0F1B1FF801E859F84F80819181D6
:106550009E01281B390BC90163E070E00E944D7A4F
:10656000CB01880F991F860F971F0255184FF8010E
:106570009183808307C0AA0FBB1FA255B84F119605
:106580001C921E92E0913F02F0914002EE0FFF1F1D
:10659000E859F84FD183C08320913F0230914002E7
:1065A0002F5F3F4F3093400220933F0280910201C2
:1065B0008431A8F42530310511F45D9A01C05D984D
:1065C00080913F02909140028630910511F45C9ACF
:1065D00001C05C98079711F45B9A01C05B98FF912A
:1065E000EF91DF91CF91BF91AF919F918F917F916B
:1065F0006F915F914F913F912F911F910F910F904C
:106600000FBE0F901F901895809174089091750897
:1066100090938E0580938D058091760890917708F0
:106620009093900580938F0580914A0890914B0834
:1066300097FD0396959587959595879590939205E7
:106640008093910580915A0890915B0897FD03967D
:106650009595879595958795909394058093930547
:106660008091EE029091EF02209106023091070294
:10667000821B930B909396058093950580917C02E5
:1066800090917D02A0917E02B0917F02BC01CD016C
:106690002AE030E040E050E00E94827A3093980592
:1066A000209397058091D2059091D30590939A05F8
:1066B0008093990580918C0190918D0190939E0516
:1066C00080939D0580912201909123019093A005D4
:1066D00080939F058091820299279093A2058093D1
:1066E000A10580910208909103089093A4058093DE
:1066F000A3058091080799279093A6058093A50587
:106700008091100799279093A8058093A705809101
:10671000180799279093AA058093A90580912007CF
:1067200099279093AC058093AB058091DC01909103
:10673000DD019093B6058093B50580916602909136
:1067400067029093B8058093B7058091DB0890911C
:10675000DC089093BA058093B9058091DF08909189
:10676000E0089093BC058093BB05809178029091DE
:106770007902A0917A02B0917B02BC01CD012AE09E
:1067800030E040E050E00E94827A3093BE052093D2
:10679000BD0580919A0290919B029093C4058093CD
:1067A000C3058091E10899279093C8058093C70598
:1067B00080915103909152039093CA058093C9052B
:1067C00080914F03909150039093CC058093CB051B
:1067D0008091A703882321F48091A803882321F0C6
:1067E00080918C05816003C080918C058E7F8093A1
:1067F0008C050895EF92FF921F93CF93DF93182F8C
:106800007B0180918102882391F5809102018C3077
:1068100010F0893111F4299801C0299A11501F3FB5
:10682000E9F0F092E401E092E301E7018091E301F5
:106830009091E401892B11F4209781F38091E70175
:106840008823A1F31092E7018091E3019091E40184
:10685000892B09F421970E941677E8CF80910201D5
:106860008C3010F0893111F4299A01C02998DF91F8
:10687000CF911F91FF90EF900895CF93DF93809178
:1068800002018D3011F40E94FB1A10927A0080915F
:106890000A0290910B0290930D0880930C0880914E
:1068A0000802909109029093FE078093FD07809162
:1068B0000602909107029093500880934F08209110
:1068C000020230910302C901880F991F880F991F96
:1068D000820F931F820F931F90934B0880934A0857
:1068E0002091040230910502C901880F991F880F79
:1068F000991F820F931F820F931F90935B088093C1
:106900005A088FEC80937A00A3E8B2E0C7E3D6E0A0
:1069100097E08991E82FFF27EE0FFF1FE859F84F06
:106920000190F081E02DE158FF4F1E161F061CF06C
:10693000E0E0F0E005C0EF3FF10514F0EFEFF0E02C
:106940008C91282F3327E217F30714F4815004C0E9
:106950002E173F0714F48F5F8C939150119697FF79
:10696000D8CF809173069927AA27BB27BC01CD01F8
:1069700024EC39E040E050E00E940E7ADC01CB01CB
:106980008093840190938501A0938601B093870141
:10699000809174069927AA27BB27BC01CD010E94CC
:1069A0000E7ADC01CB018093800190938101A0934A
:1069B0008201B0938301DF91CF910895A0E0B0E010
:1069C000E4EEF4E30C94A27AD82E91E0792EEE2432
:1069D000FF2457014701E7011092A703F092E90253
:1069E000E092E802F092E702E092E602F092E3021F
:1069F000E092E2021092E102F092F302E092F202DF
:106A0000F092F102E092F002F092EF02E092EE02D8
:106A100010926601109265011092FB010E943D34B4
:106A200084E690E00E9401160E943D3480913F066A
:106A300080FF14C08091180190911901875B9340E9
:106A400058F480911801909119018E5E924020F0C7
:106A50008091FB01882311F00E94991A009118017E
:106A60001091190187B5865F87BD87B5809588BD70
:106A70008FE1C82E8AE090E00E9401168091060204
:106A800090910702E80EF91E80910A0290910B0284
:106A9000A80EB91E8091080290910902880E991ED5
:106AA0008091D2059091D305C80FD91FCA94C7FE13
:106AB000E1CF8091180190911901825F934080F499
:106AC0008091180190911901459750F0809118011B
:106AD00090911901081B190B1093130100931201D7
:106AE00087B58A5087BD87B5809588BD9501205FA1
:106AF0003F4F36952795369527953093F30220938F
:106B0000F202C40140969695879596958795909345
:106B1000F1028093F00240E150E0E40EF51EA5E0A2
:106B2000F694E794AA95E1F7F092EF02E092EE0274
:106B3000C40FD51FF5E0D695C795FA95E1F7D09328
:106B4000E302C093E2029093ED028093EC02309353
:106B5000EB022093EA0252E0D516C9F580914A086B
:106B600090914B0897FF03C0909581959F4F6CE0E3
:106B700070E00E944D7A9B017093E9026093E802F5
:106B800080915A0890915B0897FF03C0909581957A
:106B90009F4F6CE070E00E944D7A7093E702609323
:106BA000E602B90184E090E00E946F2A6091E6025B
:106BB0007091E70286E090E00E946F2A6091E20205
:106BC0007091E30288E090E00E946F2A4FC084E059
:106BD00090E00E946A2A9093E9028093E80286E09E
:106BE00090E00E946A2A9C019093E7028093E6025B
:106BF0008091E8029091E9028150984018F4215068
:106C00003840A0F183E498E09F938F9382E092E173
:106C10009F938F93E0918E03F0918F03099580915C
:106C20004A0890914B0897FF03C0909581959F4F1C
:106C30006CE070E00E944D7A7093E9026093E80284
:106C400080915A0890915B0897FF03C090958195B9
:106C50009F4F6CE070E00E944D7A7093E702609362
:106C6000E60277240F900F900F900F9012BC11BC8A
:106C700010920D0810920C081092FE071092FD075A
:106C80001092500810924F0888EC90E00E94011674
:106C900080910202909103029C01220F331F220F68
:106CA000331F280F391F280F391F30934B082093AB
:106CB0004A0880910402909105028C01000F111F77
:106CC000000F111F080F191F080F191F10935B08E1
:106CD00000935A0880914E06C82EDD24EE24FF242E
:106CE000442737FD4095542FC701B6010E940E7A04
:106CF0004B015C016093DC027093DD028093DE0245
:106D00009093DF029801442737FD4095542FC70127
:106D1000B6010E940E7ADC01CB018093D4029093DD
:106D2000D502A093D602B093D7028092BC02909273
:106D3000BD02A092BE02B092BF028093B4029093B3
:106D4000B502A093B602B093B7021092AC021092B3
:106D5000AD021092AE021092AF0200918C01109120
:106D60008D0110939B0200939A0284E690E0909329
:106D700089018093880182E390E09093E4018093FD
:106D8000E301809173069927AA27BB27BC01CD0197
:106D900024EC39E040E050E00E940E7ADC01CB01A7
:106DA0008856954CAF4FBF4F8093840190938501D7
:106DB000A0938601B0938701809174069927AA2732
:106DC000BB27BC01CD010E940E7ADC01CB018856A5
:106DD000954CAF4FBF4F8093800190938101A0935A
:106DE0008201B09383011092430110924201C801C5
:106DF000AA2797FDA095BA2F20913E0130913F011F
:106E00004091400150914101BC01CD010E940E7A98
:106E1000DC01CB018093560890935708A093580843
:106E2000B093590810929702109296020E94B2698C
:106E3000809149028460809349028FEF8093D60845
:106E40001092D70880E28093D808C3E8D2E0A7E385
:106E5000B6E067E0C62E8D91E82FFF27EE0FFF1FEB
:106E6000E859F84F8081918181588993CA94C7FE6F
:106E7000F2CF84E6809382028091E101882311F0B1
:106E8000579A17C08091A106992780FF05C082FFFD
:106E900003C080EE9EE202C080E091E19093090180
:106EA0008093080181E0809310010E94A2160E9445
:106EB000A21688E090E00E946A2A9093E3028093F1
:106EC000E20212BC11BC8091F2029091F302805652
:106ED0009940815C9B4228F08091A7038160809358
:106EE000A7038091F0029091F10280569940815C55
:106EF0009B4228F08091A70382608093A703809132
:106F0000EE029091EF028C5291408957954028F003
:106F10008091A70384608093A7038091E8029091F9
:106F2000E9028C529140835C914028F08091A70344
:106F300088608093A7038091E6029091E7028C52CB
:106F40009140835C914028F08091A70380618093F9
:106F5000A7038091E2029091E30280509240835512
:106F6000914028F08091A70380628093A7038091CD
:106F7000A7038111772486E480937B0180911A0115
:106F800090911B01A0911C01B0911D018093D4052B
:106F90009093D505A093D605B093D7051092FA012A
:106FA0001092F9011092FC011092FD011092FE0165
:106FB0001092FF0110929C0210929D0210929E026C
:106FC00010929F021092C6051092C5050E94611A88
:106FD000872D9927EDE0CDB7DEB70C94BE7AA3E1FB
:106FE000B0E0E5EFF7E30C949D7A8091EE0290918A
:106FF000EF022091060230910702821B930B9093BF
:10700000500880934F08809110029091110297FDD3
:1070100007969C0153E0359527955A95E1F73093F3
:107020000D0820930C0880910E0290910F0297FD9D
:10703000079643E0959587954A95E1F79093FE076B
:107040008093FD0730931908209318089093100837
:1070500080930F0880914A0890914B08AC01440F2F
:10706000551F480F591F2091020230910302C90198
:10707000880F991F880F991F820F931F820F931FEC
:10708000480F591F57FF02C04D5F5F4F55954795F9
:107090005595479550934B0840934A0880915A085C
:1070A00090915B08AC01440F551F480F591F209168
:1070B000040230910502C901880F991F880F991F9A
:1070C000820F931F820F931F480F591F57FF02C053
:1070D0004D5F5F4F559547955595479550935B0884
:1070E00040935A082091020230910302C901880F8F
:1070F000991F880F991F820F931F820F931F9C0166
:10710000442737FD4095542F8091CC029091CD02B9
:10711000A091CE02B091CF02820F931FA41FB51F82
:107120008093CC029093CD02A093CE02B093CF0275
:107130002091040230910502C901880F991F880F20
:10714000991F820F931F820F931F9C01442737FDC5
:107150004095542F8091C8029091C902A091CA0213
:10716000B091CB02820F931FA41FB51F8093C8025A
:107170009093C902A093CA02B093CB0280912208D7
:10718000909123082091020230910302820F931FF5
:10719000909323088093220880915208909153087D
:1071A0002091040230910502820F931F909353089F
:1071B000809352088091E4029091E50201969093A9
:1071C000E5028093E4028091D2059091D30520914D
:1071D000E2023091E302821B930B9C01442737FDAE
:1071E0004095542F8091C4029091C502A091C6028F
:1071F000B091C702820F931FA41FB51F8093C402D2
:107200009093C502A093C602B093C7028FEC8093FF
:107210007A00109214012091B4023091B50240918D
:10722000B6025091B70229873A874B875C87295469
:107230003B46414050402CF028E43BE641E050E022
:107240000DC089859A85AB85BC85885B9449AE4F16
:10725000BF4F4CF428EB34E94EEF5FEF2D833E83B4
:107260004F83588708C089859A85AB85BC858D83F7
:107270009E83AF83B8872091BC023091BD024091BC
:10728000BE025091BF022D873E874F87588B2954ED
:107290003B46414050402CF028E43BE641E050E0C2
:1072A0000DC08D859E85AF85B889885B9449AE4FAA
:1072B000BF4F4CF428EB34E94EEF5FEF29833A835C
:1072C0004B835C8308C08D859E85AF85B889898393
:1072D0009A83AB83BC83A0914F08B0915008BB8BBD
:1072E000AA8BFD01CF01AA2797FDA095BA2FA090E8
:1072F000AC02B090AD02C090AE02D090AF02A80E2A
:10730000B91ECA1EDB1EA092AC02B092AD02C092A2
:10731000AE02D092AF02E0905608F090570800916C
:10732000580810915908E80EF91E0A1F1B1FE09219
:107330005608F09257080093580810935908F09196
:107340006502F98BFF2309F098C1809164028823BC
:1073500009F093C18091460886FF8FC18091FD0797
:107360009091FE07AA2797FDA095BA2FBC01CD01E9
:1073700029813A814B815C810E940E7A9B01AC018C
:1073800097FF04C02150384F4F4F5F4F6BE055952A
:107390004795379527956A95D1F780916501682EB5
:1073A000772488249924CA01B901A40193010E9479
:1073B0000E7ADC01CB018093FE029093FF02A09332
:1073C0000003B0930103B7FF04C08150904FAF4F4B
:1073D000BF4F1C012D013CE05594479437942794EE
:1073E0003A95D1F72092FE023092FF0240920003BC
:1073F0005092010380910C0890910D08AA2797FDE7
:10740000A095BA2FBC01CD012D813E814F815885B9
:107410000E940E7A97FF04C06150784F8F4F9F4FA4
:107420002BE095958795779567952A95D1F7A401D7
:1074300093010E940E7ADC01CB01809302039093AA
:107440000303A0930403B0930503B7FF04C0815066
:10745000904FAF4FBF4F9C01AD018CE055954795C4
:10746000379527958A95D1F720930203309303032C
:1074700040930403509305038091FE029091FF0214
:107480009093F5078093F407809102039091030392
:107490009093F9078093F807221933094409550995
:1074A0002093020330930303409304035093050396
:1074B000E20EF31E041F151FE0925608F0925708C3
:1074C0000093580810935908809164018823B1F4FF
:1074D00057FF04C02F5F3F4F4F4F5F4F5595479564
:1074E00037952795A21AB30AC40AD50AA092AC020E
:1074F000B092AD02C092AE02D092AF022A893B890F
:1075000079010027F7FC0095102F809102039091DC
:107510000303A0910403B0910503E80EF91E0A1FAE
:107520001B1FC801B70129813A814B815C810E94F0
:107530000E7A9B01AC0197FF04C02150384F4F4F8A
:107540005F4FBBE05595479537952795BA95D1F78D
:1075500080916601A82EBB24CC24DD24CA01B90188
:10756000A60195010E940E7ADC01CB018093F60200
:107570009093F702A093F802B093F902B7FF04C00A
:107580008150904FAF4FBF4F3C014D01ACE09594FF
:10759000879477946794AA95D1F76092F6027092D7
:1075A000F7028092F8029092F902C801B7012D818A
:1075B0003E814F8158850E940E7A97FF04C061502A
:1075C000784F8F4F9F4FFBE09595879577956795FF
:1075D000FA95D1F7A60195010E940E7ADC01CB0144
:1075E0008093FA029093FB02A093FC02B093FD02F9
:1075F000B7FF04C08150904FAF4FBF4FAC01BD01EA
:10760000ECE07595679557954795EA95D1F74093C6
:10761000FA025093FB026093FC027093FD022A89E8
:107620003B8937FF03C0309521953F4F2134310509
:10763000E4F1D401C30197FE07C0B095A0959095E1
:1076400081959F4FAF4FBF4F81389105A105B1057F
:1076500084F4DB01CA0177FF07C0B095A09590952F
:1076600081959F4FAF4FBF4F81389105A105B1055F
:10767000E4F081E08093980218C01092F90710920C
:10768000F8071092F5071092F4071092FA02109280
:10769000FB021092FC021092FD021092F602109270
:1076A000F7021092F8021092F9028091FA0290917A
:1076B000FB02A091FC02B091FD02BC01CD0124E6C9
:1076C00030E040E050E00E94827AE090F602F090D4
:1076D000F702E21AF30AF0920B08E0920A0880918E
:1076E000F6029091F702A091F802B091F902BC0164
:1076F000CD0124E630E040E050E00E94827ADA01D9
:10770000C9012091FA023091FB028C01021B130B7C
:10771000109300080093FF0780913E0190913F0174
:10772000A0914001B0914101BC01CD0128E631E0BA
:1077300040E050E00E940E7A2091560830915708A0
:10774000409158085091590826173707480759079C
:1077500064F0261B370B480B590B209356083093C7
:107760005708409358085093590820915608309173
:107770005708409158085091590857FF0CC0260FE0
:10778000371F481F591F20935608309357084093BE
:107790005808509359086091FD077091FE076E0DCF
:1077A0007F1D9B01442737FD4095542F8091B002E7
:1077B0009091B102A091B202B091B302820F931FD7
:1077C000A41FB51F8093B0029093B102A093B202A0
:1077D000B093B30280916A0290916B02681B790B9F
:1077E000CB01AA2797FDA095BA2F29853A854B850D
:1077F0005C85820F931FA41FB51F8093B4029093E2
:10780000B502A093B602B093B702C0908001D090A9
:107810008101E0908201F0908301C816D906EA0642
:10782000FB06C4F488EA91E6A0E0B0E08C199D095B
:10783000AE09BF098093B4029093B502A093B6023B
:10784000B093B7028093B0029093B102A093B202BA
:10785000B093B30222273327A9012C193D094E0901
:107860005F098091B4029091B502A091B602B091E7
:10787000B70282179307A407B507B4F4D701C6016E
:10788000885A9146A040B0408093B4029093B502CC
:10789000A093B602B093B7028093B0029093B10266
:1078A000A093B202B093B30260910C0870910D08DE
:1078B000600F711F9B01442737FD4095542F809125
:1078C000B8029091B902A091BA02B091BB02820FA6
:1078D000931FA41FB51F8093B8029093B902A09381
:1078E000BA02B093BB028091680290916902681B52
:1078F000790BCB01AA2797FDA095BA2F2D853E8540
:107900004F855889820F931FA41FB51F8093BC0217
:107910009093BD02A093BE02B093BF02E090840199
:10792000F09085010091860110918701E816F90613
:107930000A071B07C4F488EA91E6A0E0B0E08E19BC
:107940009F09A00BB10B8093BC029093BD02A09342
:10795000BE02B093BF028093B8029093B902A09385
:10796000BA02B093BB0222273327A9012E193F097F
:10797000400B510B8091BC029091BD02A091BE02C0
:10798000B091BF0282179307A407B507B4F4D801DA
:10799000C701885A9146A040B0408093BC029093A2
:1079A000BD02A093BE02B093BF028093B802909331
:1079B000B902A093BA02B093BB028091AC0290913D
:1079C000AD02A091AE02B091AF028093C00290933D
:1079D000C102A093C202B093C3028091BC029091F5
:1079E000BD02A091BE02B091BF028093DC029093D1
:1079F000DD02A093DE02B093DF028091B402909189
:107A0000B502A091B602B091B7028093D4029093D0
:107A1000D502A093D602B093D7028091B80290917C
:107A2000B902A091BA02B091BB028093D8029093A0
:107A3000D902A093DA02B093DB028091B002909158
:107A4000B102A091B202B091B3028093D0029093A0
:107A5000D102A093D202B093D302809120019091E1
:107A6000210197FD079633E0959587953A95E1F7C3
:107A700090930D0880930C0880911E0190911F0136
:107A800097FD079623E0959587952A95E1F79093C2
:107A9000FE078093FD0780910A0290910B020F97D9
:107AA00034F488E19CEF90930D0880930C0880914A
:107AB0000A0290910B02079734F480E398EF9093B9
:107AC0000D0880930C08209102012A30A9F48091BE
:107AD0000A0290910B02835F934034F088EE93E0AA
:107AE00090930D0880930C0880910A0290910B02EC
:107AF0008A5F9340DCF014C080910A0290910B02DF
:107B0000815D974034F088EE93E090930D08809368
:107B10000C0880910A0290910B02805E974034F02D
:107B200080ED97E090930D0880930C0880910802F7
:107B3000909109020F9734F488E19CEF9093FE072F
:107B40008093FD078091080290910902079734F411
:107B500080E398EF9093FE078093FD072A30A9F405
:107B60008091080290910902835F934034F088EE7F
:107B700093E09093FE078093FD0780910802909117
:107B800009028A5F9340DCF014C080910802909152
:107B90000902815D974034F088EE93E09093FE07F0
:107BA0008093FD078091080290910902805E9740C2
:107BB00034F080ED97E09093FE078093FD0760918D
:107BC0007301662309F4AFC0409120015091210157
:107BD0008091060390910703481B590B50930D03A6
:107BE00040930C032091200130912101280F391F6F
:107BF00037FF02C02F5F3F4F35952795309307031E
:107C000020930603413851051CF080E890E005C040
:107C100040585F4F34F480E89FEF90930D038093BA
:107C20000C0340911E0150911F0180910803909117
:107C30000903481B590B50930B0340930A032091EF
:107C40001E0130911F01280F391F37FF02C02F5F1F
:107C50003F4F35952795309309032093080341380A
:107C600051051CF080E890E005C040585F4F34F4A7
:107C700080E89FEF90930B0380930A03462F5527CC
:107C800080910C0390910D03849FB001859F700D2E
:107C9000949F700D11249B0177FF02C0215F3F4F1D
:107CA000B4E035952795BA95E1F780910C0890914D
:107CB0000D08820F931F90930D0880930C088091FC
:107CC0000A0390910B03849FD001859FB00D949F70
:107CD000B00D1124AD019D01B7FF02C0215F3F4FE0
:107CE000A4E035952795AA95E1F78091FD0790913D
:107CF000FE07820F931F9093FE078093FD078091EC
:107D0000200190912101860F971F9093210180936C
:107D1000200180911E0190911F01840F951F909367
:107D20001F0180931E0100910F081091100880918F
:107D3000F4079091F507101611065CF59C0197FF6A
:107D400004C022273327281B390BC901AA2797FD16
:107D5000A095BA2F20916401332744275527BC01F1
:107D6000CD010E940E7A9B01AC0197FF04C0215CFB
:107D70003F4F4F4F5F4FF6E0559547953795279505
:107D8000FA95D1F780910A0890910B08820F931F02
:107D900027C097FF03C0909581959F4FAA2797FD15
:107DA000A095BA2F20916401332744275527BC01A1
:107DB000CD010E940E7A9B01AC0197FF04C0215CAB
:107DC0003F4F4F4F5F4FE6E05595479537952795C5
:107DD000EA95D1F780910A0890910B08821B930BCA
:107DE00090930B0880930A08E0901808F090190807
:107DF0008091F8079091F9071E141F045CF59C010F
:107E000097FF04C022273327281B390BC901AA2753
:107E100097FDA095BA2F2091640133274427552759
:107E2000BC01CD010E940E7A9B01AC0197FF04C0FA
:107E3000215C3F4F4F4F5F4F76E055954795379503
:107E400027957A95D1F78091FF0790910008820FCE
:107E5000931F27C097FF03C0909581959F4FAA2736
:107E600097FDA095BA2F2091640133274427552709
:107E7000BC01CD010E940E7A9B01AC0197FF04C0AA
:107E8000215C3F4F4F4F5F4F66E0559547953795C3
:107E900027956A95D1F78091FF0790910008821B82
:107EA000930B909300088093FF078091460887FF0B
:107EB00044C0B989BB2309F040C080916402882383
:107EC000E1F5E1E0EE16E1E0FE064CF080910C08F1
:107ED00090910D088E0D9F1D805091400DC0F0E0D7
:107EE000EF16FFEFFF0664F480910C0890910D08E7
:107EF0008E0D9F1D80509F4F90930D0880930C080E
:107F000021E0013012074CF08091FD079091FE07AF
:107F1000800F911F805091400CC03FEF003013073D
:107F200064F48091FD079091FE07800F911F8050AF
:107F30009F4F9093FE078093FD07E2E1CD5E0C9486
:107F4000B97A80918102882329F5809149028C7F3A
:107F500080934902809148028F7D80934802ACEA69
:107F6000B3E0E7E0F7E09BE08091C101882309F4EA
:107F70008C938D91818312829150389697FFF4CF24
:107F80008091C101882359F08091C1018150809373
:107F9000C10105C0809149028160809349028091AE
:107FA0003202882319F0109232020895809334022D
:107FB00080933602809130028E7F8093300285EA72
:107FC0008093BC000895882319F480E090E0089520
:107FD000E82FFF27EE0FFF1FE859F84F80819181AE
:107FE00081589F4F8F3F910521F01CF08FEF90E05B
:107FF00004C097FF02C080E090E099270895CF93D6
:10800000DF93A3E8B2E0C7E3D6E057E08991E82F19
:10801000FF27EE0FFF1FE859F84F0190F081E02D88
:10802000E158FF4FEF3FF10521F01CF0EFEFF0E0DA
:1080300004C0F7FF02C0E0E0F0E0893111F4EC93F6
:108040001BC04C91242F3327E217F307A9F0CF016F
:10805000821B930B97FD039695958795959587952C
:10806000242F280F2C93822F9927E817F90714F44F
:10807000215001C02F5F2C935150119657FFC6CF4E
:1080800080914106883F38F0EFEFF0E0E81BF109FE
:10809000ED57FD4F8081809378018091780188238E
:1080A00029F0843618F084E68093780180914306A5
:1080B000883F38F0EFEFF0E0E81BF109ED57FD4F96
:1080C00080818093770180917701882329F084361D
:1080D00018F084E68093770180915006883F38F04D
:1080E000EFEFF0E0E81BF109ED57FD4F8081809341
:1080F0007201809172018B3010F48AE002C08F3FD0
:1081000011F48093720180917D06883F38F0EFEF83
:10811000F0E0E81BF109ED57FD4F808180932408C2
:1081200080912408863010F485E002C08F3F11F45E
:108130008093240880917F06883F38F0EFEFF0E0CD
:10814000E81BF109ED57FD4F808180934D08809128
:108150004D08863010F485E002C08F3F11F4809303
:108160004D0880916A06873F19F4429905C006C000
:10817000863F31F4439B02C08CE815C086E413C0EF
:10818000883F38F0EFEFF0E0E81BF109ED57FD4FC5
:1081900080818093210880912108893110F488E141
:1081A00002C08F3F11F48093210880916B06873FB6
:1081B00019F4429905C006C0863F31F4439B02C0C2
:1081C0008CE815C086E413C0883F38F0EFEFF0E08C
:1081D000E81BF109ED57FD4F80818093FA078091EC
:1081E000FA07893110F488E102C08F3F11F48093BF
:1081F000FA0780916C06883F38F0EFEFF0E0E81B5B
:10820000F109ED57FD4F808180932A0880912A085B
:10821000893110F488E102C08F3F11F480932A085D
:10822000809142060E94E33F80935F028091450661
:10823000883F38F0EFEFF0E0E81BF109ED57FD4F14
:1082400080818093760180914706883F38F0EFEF78
:10825000F0E0E81BF109ED57FD4F80818093740138
:1082600080914F06883F38F0EFEFF0E0E81BF1090E
:10827000ED57FD4F80818093750180915106883FB5
:1082800038F0EFEFF0E0E81BF109ED57FD4F80818A
:108290008093710180915206883F38F0EFEFF0E053
:1082A000E81BF109ED57FD4F8081809373018091A8
:1082B0005306883F38F0EFEFF0E0E81BF109ED5787
:1082C000FD4F80818093700180915406883F38F083
:1082D000EFEFF0E0E81BF109ED57FD4F808180934F
:1082E0006F0180915A06883F38F0EFEFF0E0E81B0D
:1082F000F109ED57FD4F808180936D0180915B0600
:10830000883F38F0EFEFF0E0E81BF109ED57FD4F43
:10831000808180935E0280915C06883F38F0EFEFA9
:10832000F0E0E81BF109ED57FD4F808180935D027D
:1083300080915D06883F38F0EFEFF0E0E81BF1092F
:10834000ED57FD4F808180935C0280915E06883FEF
:1083500038F0EFEFF0E0E81BF109ED57FD4F8081B9
:1083600080935B0280917806883F38F0EFEFF0E071
:10837000E81BF109ED57FD4F808180935A028091EF
:108380007906883F38F0EFEFF0E0E81BF109ED5790
:10839000FD4F80818093590280917A06883F38F0A2
:1083A000EFEFF0E0E81BF109ED57FD4F808180937E
:1083B000580280917B06883F38F0EFEFF0E0E81B31
:1083C000F109ED57FD4F80818093570280915F0640
:1083D000883F38F0EFEFF0E0E81BF109ED57FD4F73
:1083E000808180936B0180916306883F38F0EFEFC6
:1083F000F0E0E81BF109ED57FD4F808180936A01A1
:1084000080916006883F38F0EFEFF0E0E81BF1095B
:10841000ED57FD4F80818093690180916406883F0C
:1084200038F0EFEFF0E0E81BF109ED57FD4F8081E8
:108430008093680180916D06883F38F0EFEFF0E09F
:10844000E81BF109ED57FD4F808180936701809112
:108450007006883F38F0EFEFF0E0E81BF109ED57C8
:10846000FD4F80818093660180917106883F38F0CE
:10847000EFEFF0E0E81BF109ED57FD4F80818093AD
:10848000650180917206883F38F0EFEFF0E0E81B5D
:10849000F109ED57FD4F80818093640180919A0628
:1084A000883F38F0EFEFF0E0E81BF109ED57FD4FA2
:1084B00080818093090890915B03992321F080913A
:1084C0000908981720F080910908882311F49093E7
:1084D000090880913F06809346088091A206809308
:1084E000290880917706883F38F0EFEFF0E0E81B2D
:1084F000F109ED57FD4F80818093630180919306D0
:10850000883F38F0EFEFF0E0E81BF109ED57FD4F41
:10851000808180935D0880916D01282F33272F5F24
:108520003F4F8CE398E2B9010E944D7A70937A0133
:108530006093790180914D0680934E0880914C069E
:1085400080931108E0919506EE23D9F181E08093A4
:108550005602FF27EE0FFF1FE859F84F80819181E7
:10856000805C9F4F14F41092560280917B01209101
:1085700056028217B1F0833088F4222319F08CED73
:1085800095E002C088EC90E09093E4018093E301D1
:1085900085E080936C0220937B0103C0815080931F
:1085A0007B0180919D0890919E0897FF0FC080915C
:1085B0005602882359F08091A70380688093A7030F
:1085C00005C0E09356028AE080937B0180919D086C
:1085D00090919E0897FF1DC0809181028823C9F069
:1085E000809156028823A9F080910A0190910B0195
:1085F0008F5F9F4F71F488E99AE39093E401809331
:10860000E30180E094EA90930B0180930A011092B9
:10861000560280915602882321F0809148028160A1
:1086200003C0809148028E7F80934802DF91CF91F2
:108630000895A7E1B0E0EFE1F3E40C949D7A0E9485
:10864000EF3780914902992784719070892B91F5B9
:108650008091A30682FF27C08091660290916702F5
:108660000097F1F002E088359007D4F49C0197FF61
:1086700002C02D5F3F4F3595279535952795809101
:1086800057069927289FA001299F500D389F500D0C
:108690001124CA0164E670E00E944D7ACB0106C045
:1086A0008DE290E003C0809157069927909347028E
:1086B00080934602209144023091450255E72033D1
:1086C000350759F410928D0210928C028091110896
:1086D0009927909347028093460260918C02709193
:1086E0008D027A8369838091110899270A96681709
:1086F000790714F49A83898380918202843608F082
:108700006AC08091480282FD66C0809122039091E8
:108710002303009731F00197909323038093220362
:108720000BC01092810290934B0280934A02809179
:1087300049028D7E80934902809102018A3011F0B6
:10874000843110F0289A01C0289880914A029091B3
:108750004B02895E9340E0F18091E1088536C0F1DB
:1087600080914602909147029A83898380914902C1
:1087700080618093490280913306A82FBB27AA0FFE
:10878000BB1FFD01E255F84F118210828091340623
:10879000282F3327220F331FC9018255984FFC0120
:1087A00011821082A859B84F11961C921E92285916
:1087B000384FD90111961C921E9280913606E82FEF
:1087C000FF27EE0FFF1FE859F84F1182108251C4A6
:1087D000109281024EC4809182028D3808F41FC429
:1087E000809149028F7E809349029091580682E3DE
:1087F000989FC00111249093230380932203E98161
:10880000FA81B9978CF080918102882369F0809178
:108810004A0290914B02FFEF8F3F9F0729F001968C
:1088200090934B0280934A0220914A0230914B026E
:108830002F3F310509F030F51092A4021092A502E5
:108840001092A6021092A7021092A0021092A1020A
:108850001092A2021092A30210920E0310920F0324
:1088600010921003109211031092AC021092AD02FC
:108870001092AE021092AF02809148028062809303
:1088800048024DC0809149028260809349028091E4
:10889000480285FF44C08091EF019091F001A091C2
:1088A000F101B091F20187399105A105B1058CF470
:1088B00080917C0290917D02A0917E02B0917F0216
:1088C000825A9E4FAF4FBF4F24F08091460880FDE3
:1088D00005C0809148028F71809348021092A402D3
:1088E0001092A5021092A6021092A7021092A00266
:1088F0001092A1021092A2021092A3021092AC0256
:108900001092AD021092AE021092AF02295E334077
:1089100030F088EE93E090934B0280934A0280916E
:108920003506E82FFF27EE0FFF1FE859F84F80812B
:108930009181813591050CF434C12091810222236B
:1089400009F02FC180913606E82FFF27EE0FFF1F99
:10895000E859F84F808191818C3491050CF4FFC067
:10896000809124038F5F80932403893C08F419C10C
:108970002093240310924B0210924A023091330646
:10898000E32FFF27EE0FFF1FE859F84F80819181F9
:1089900087349105B4F480913406E82FFF27EE0F59
:1089A000FF1FE859F84F808191810190F081E02DFF
:1089B000F7FF03C0F095E195FF4FE734F1050CF4A4
:1089C00078C041E020913406A22FBB27AA0FBB1F1D
:1089D000A859B84F8D919C9111978734910544F017
:1089E000E32FFF27EE0FFF1FE859F84F8081918199
:1089F0008D919C918734910574F080913306E82F16
:108A0000FF27EE0FFF1FE859F84F808191818734CF
:108A100091050CF042E0E22FFF27EE0FFF1FE8590F
:108A2000F84F808191818634910574F480913306EA
:108A3000E82FFF27EE0FFF1FE859F84F8081918143
:108A4000873491050CF043E0E22FFF27EE0FFF1F64
:108A5000E859F84F808191818A5B9F4F74F480912F
:108A60003306E82FFF27EE0FFF1FE859F84F8081EC
:108A70009181873491050CF044E0E22FFF27EE0F3F
:108A8000FF1FE859F84F808191818A5B9F4F74F4F2
:108A900080913306E82FFF27EE0FFF1FE859F84FAC
:108AA00080819181863491050CF445E0842F0E94E9
:108AB000C72A80913406E82FFF27EE0FFF1FE859E1
:108AC000F84F808191810190F081E02DF7FF03C084
:108AD000F095E195FF4F7E97CCF480913306E82F17
:108AE000FF27EE0FFF1FE859F84F808191818A5BC5
:108AF0009F4F64F481E08093C20310926D0288EE70
:108B000093E09093E4018093E3014BC080910001D6
:108B10000E94742A80E00E943406809159060E94C7
:108B20009C758091460880FF10C08091180190913B
:108B30001901875B934038F48091180190911901D5
:108B40008E5E924010F40E94991A81E00E94DE34F9
:108B500080936D0281E08093E101579A19C0808172
:108B60009181855B9F4FDCF4809124038F5F80931C
:108B70002403893CB0F020938102209324031092B7
:108B80004B0210924A0282E00E94DE3480936D0212
:108B900068E770E0809100010E94FA3302C02093E0
:108BA000240380913506E82FFF27EE0FFF1FE859B9
:108BB000F84F808191818C599F4F0CF029C22091F0
:108BC0009606E22FFF27EF77F070EE0FFF1FE255BA
:108BD000F84F80819181069714F084E606C0808169
:108BE00091818B5F9F4F1CF48CE9809327038091C8
:108BF0008102E0913606882309F058C1FF27EE0F65
:108C0000FF1FE859F84F808191818C599F4F9CF448
:108C10008091A30683FD0BC0E22FFF27EE0FFF1FFD
:108C2000E859F84F80819181855B9F4FDCF08091FE
:108C300096068823B9F08091A30683FF34C1809102
:108C40009606E82FFF27EE0FFF1FE859F84F8081A7
:108C50009181875F9F4F0CF426C180912703843652
:108C600009F021C180916D02882329F08091490289
:108C700088608093490280911A0190911B01A09114
:108C80001C01B0911D018093D4059093D505A0934C
:108C9000D605B093D7051092EF011092F001109213
:108CA000F1011092F20110927C0210927D0210925A
:108CB0007E0210927F021092FC011092FD01109230
:108CC000FE011092FF0180913306E82FFF27EE0F7F
:108CD000FF1FE859F84F808191818D599F4FACF467
:108CE00080913406E82FFF27EE0FFF1FE859F84F59
:108CF000808191810190F081E02DF7FF03C0F09514
:108D0000E195FF4FE436F10534F48091960688230F
:108D100011F480932503809125038F5F80932503B1
:108D20008E3F08F458C180914F089091500897FFEA
:108D300003C0909581959F4F8197B4F480910C0862
:108D400090910D0897FF03C0909581959F4F45978F
:108D50005CF48091FD079091FE0797FF03C090950A
:108D600081959F4F459714F010926D021092250344
:108D70008091A703882309F093C080916D02882316
:108D800009F48EC080916003882309F089C081E0D6
:108D900090E090934B0280934A0281E0809381029D
:108DA00010920E0310920F031092100310921103F1
:108DB0001092AC021092AD021092AE021092AF026D
:108DC0001092A8021092A9021092AA021092AB026D
:108DD00080914E06E82EFF240027112780914A0833
:108DE00090914B089C01442737FD4095542FC801B2
:108DF000B7010E940E7ADC01CB018093BC029093F4
:108E0000BD02A093BE02B093BF0280915A08909118
:108E10005B089C01442737FD4095542FC801B701DA
:108E20000E940E7ADC01CB018093B4029093B502CC
:108E3000A093B602B093B7028091DC029091DD025C
:108E4000A091DE02B091DF028093B8029093B90244
:108E5000A093BA02B093BB028091D4029091D50244
:108E6000A091D602B091D7028093B0029093B10244
:108E7000A093B202B093B3021092A4021092A50282
:108E80001092A6021092A7021092A0021092A102C4
:108E90001092A2021092A30284E680936C029BC0FF
:108EA0008CED95E091C01092250395C0FF27EE0F41
:108EB000FF1FE859F84F80819181853691059CF01C
:108EC0008091A30683FD0BC0E22FFF27EE0FFF1F4B
:108ED000E859F84F80819181855B9F4FDCF080914C
:108EE00096068823B9F08091A30683FF72C0809113
:108EF0009606E82FFF27EE0FFF1FE859F84F8081F5
:108F000091818E5C9F4F0CF064C0809127038C3957
:108F100009F05FC080913306E82FFF27EE0FFF1F97
:108F2000E859F84F808191818D599F4FACF4809121
:108F30003406E82FFF27EE0FFF1FE859F84F808116
:108F400091810190F081E02DF7FF03C0F095E1954C
:108F5000FF4FE436F1053CF480919606882319F41E
:108F60008093260318C01092A4021092A5021092BA
:108F7000A6021092A7021092A0021092A1021092D3
:108F8000A2021092A30210929302109292021092E7
:108F9000910210929002809126038F5F80932603A6
:108FA0008B3F70F0109281021092260310924B02B8
:108FB00010924A02809148028F71809348020BC040
:108FC000843649F48CEA9DE09093E4018093E301B8
:108FD00002C010922603209144023091450273E0B2
:108FE000283E370708F045C08091F9019091FA01B9
:108FF0008B569F4F1CF02F5F3F4F05C02115310549
:10900000C1F121503040309345022093440231C0D9
:109010001092270310924502109244022AC02E5E3D
:10902000324038F1809165089091660880599140EE
:1090300000F580917C0290917D02A0917E02B0911A
:109040007F028C5D9540A040B0409CF480E395E7A2
:10905000909345028093440280914A0290914B0282
:109060008A5E934030F089EE93E090934B028093B8
:109070004A0280913C01815080933C0180913C01E7
:109080008F3F21F08091490284FFDFC30E94FF3FA0
:10909000B090490680913003909131039C01220FDA
:1090A000331F280F391FC0903306AC2DBB27AA0FE2
:1090B000BB1FFD01E859F84F4B2D55278081918149
:1090C000849FB001859F700D949F700D1124260F11
:1090D000371F37FF02C02D5F3F4FB9017595679568
:1090E00075956795A255B84F80914A06082F1127AC
:1090F0008D919C91809FD001819FB00D909FB00D6C
:1091000011246A0F7B1F70933103609330038091A9
:109110003203909133039C01220F331F280F391F14
:10912000D0903406AD2DBB27AA0FBB1FFD01E85917
:10913000F84F80819181849FF001859FF00D949F6D
:10914000F00D11242E0F3F1F37FF02C02D5F3F4F40
:10915000A9015595479555954795A255B84F8D91BD
:109160009C91809F7001819FF00C909FF00C1124C6
:109170004E0D5F1D5093330340933203809156028E
:10918000882309F448C0CB0177FD0396DC01B5952F
:10919000A795B595A795CA0157FD0396FC01F595CE
:1091A000E795F595E79580919E01682F772767FDF4
:1091B00070956A9F90016B9F300D7A9F300D11243E
:1091C00080916203482F552747FD50954E9FC0015F
:1091D0004F9F900D5E9F900D1124280F391F37FF70
:1091E00002C0295F3F4F03E0359527950A95E1F7C7
:1091F00030939302209392026E9F90016F9F300DE7
:109200007E9F300D11244A9FC0014B9F900D5A9FA5
:10921000900D11243FC080919406E82FFF27EC5B4E
:10922000FE4F868180939E01908190936203A82FC8
:10923000BB27A7FDB095A69F9001A79F300DB69FB5
:10924000300D1124E92FFF27E7FDF095E49FC001C1
:10925000E59F900DF49F900D1124280F391F37FFC3
:1092600002C0295F3F4F13E0359527951A95E1F726
:109270003093930220939202A49F9001A59F300DFA
:10928000B49F300D1124E69FC001E79F900DF69F1B
:10929000900D1124281B390B37FF02C0295F3F4F67
:1092A00043E0359527954A95E1F730939102209355
:1092B000900280913606E82FFF27EE0FFF1FE85936
:1092C000F84F80819181909581959F4F90938F0267
:1092D00080938E028530910514F0049705C00FEF3E
:1092E0008C3F900734F4049690938F0280938E0203
:1092F00004C010928F0210928E02809144029091CD
:1093000045028150924078F18091920290919302AF
:1093100097FD079623E0959587952A95E1F7909319
:10932000930280939202809190029091910297FD16
:10933000079603E0959587950A95E1F7909391023A
:10934000809390021092A4021092A5021092A6029D
:109350001092A7021092A0021092A1021092A202F3
:109360001092A30243C080914E03882309F43EC0AB
:10937000282F3327809192029091930297FD0796B0
:1093800013E0959587951A95E1F7289FA001299FED
:10939000500D389F500D1124CA0157FD0F96B4E0AF
:1093A00095958795BA95E1F79093930280939202F1
:1093B000809190029091910297FD0796A3E0959578
:1093C0008795AA95E1F7289FB001299F700D389FD6
:1093D000700D1124CB0177FD0F96F4E095958795DC
:1093E000FA95E1F790939102809390028090920217
:1093F000909093028091510390915203881A990A98
:1094000090929302809292020091900210919102A8
:1094100080914F0390915003081B190B10939102F8
:109420000093900280913506E82FFF27EE0FFF1F73
:10943000E859F84FE080F1808FE790E0E80EF91EE0
:10944000F0928D02E0928C02809172019927AA27F6
:1094500097FDA095BA2FBC01CD010E948279DC0155
:10946000CB0120E030E040E251E4BC01CD010E949C
:10947000F078DC01CB01BC01CD010E945479DC0104
:10948000CB01809354088091710180932B088091C7
:1094900070019927AA2797FDA095BA2FBC01CD018D
:1094A0000E948279DC01CB0120E030E040E251E40F
:1094B000BC01CD010E94F078DC01CB01BC01CD01E3
:1094C0000E945479DC01CB018093040880916F01E4
:1094D00080931A088091CE0380FF59C080915D0867
:1094E000813808F454C08091C703992787FD90956F
:1094F0002B2D3327829FD001839FB00D929FB00DFB
:1095000011248A0E9B1E9092930280929202809167
:10951000C803992787FD9095829FF001839FF00DE6
:10952000929FF00D11240E0F1F1F109391020093B4
:1095300090028091C903282F332727FD3095809111
:109540008E0290918F02820F931F90938F028093CF
:109550008E028091CB03282F332727FD30958091F1
:1095600044069927289F8001299F100D389F100DD0
:10957000112410934301009342018091CA0399275B
:109580008E159F0524F490938D0280938C02809118
:109590008C0290918D0297FF04C010928D02109260
:1095A0008C028091460882FF02C010922B084091E5
:1095B000920250919302CA0157FD03969C01359582
:1095C00027953595279537FF03C0309521953F4F57
:1095D00080914E0290914F0282179307B4F4CA0112
:1095E00057FF03C0909581959F4F97FD03969595E2
:1095F00087959595879590934F0280934E02853677
:10960000910544F084E690E001C0019790934F02E9
:1096100080934E024091900250919102CA0157FDF1
:1096200003969C01359527953595279537FF03C0FF
:10963000309521953F4F80914C0290914D028217B9
:109640009307B4F4CA0157FF03C0909581959F4FCB
:1096500097FD0396959587959595879590934D02DF
:1096600080934C028536910544F084E690E001C079
:10967000019790934D0280934C028091490284FFA0
:1096800008C010924F0210924E0210924D0210929A
:109690004C02ED2DFF27EE0FFF1FE859F84F4091C8
:1096A0006E06242F3327808191812817390744F4CF
:1096B0008091A00682FF04C081E08093630213C002
:1096C000ED2DFF27EE0FFF1FE859F84F842F992744
:1096D00020916F06821B910920813181281739075B
:1096E00014F41092630240913406E42FFF27EE0F2A
:1096F000FF1FE859F84F50916E06852F99272227B2
:109700003327281B390B808191818217930744F4FA
:109710008091A00683FF04C081E08093620216C09E
:1097200080916202882391F0E42FFF27EE0FFF1F44
:10973000E859F84F80916F069927851B9109208180
:1097400031818217930714F410926202EC2DFF27E7
:10975000EE0FFF1FE859F84F40916E06242F332774
:10976000808191812817390744F48091A00680FFF9
:1097700004C081E08093600217C08091600288235A
:1097800099F0EC2DFF27EE0FFF1FE859F84F842FBB
:10979000992720916F06821B91092081318128171A
:1097A000390714F41092600240913306E42FFF272A
:1097B000EE0FFF1FE859F84F50916E06852F99273D
:1097C00022273327281B390B808191818217930729
:1097D00044F48091A00681FF04C081E0809361027F
:1097E00016C080916102882391F0E42FFF27EE0FCD
:1097F000FF1FE859F84F80916F069927851B910943
:10980000208131818217930714F4109261028091B4
:109810006302882319F480916202811181E08093B0
:10982000640280916002882321F480916102882380
:1098300051F081E0809365021092640210926302FD
:109840001092620202C080936502809164028823B4
:1098500021F480916502882369F080916D06992733
:1098600029813A818217930714F49A83898381E0CE
:10987000809398028091480299279C01247030704F
:1098800082FF2DC080915103909152039095819554
:109890009F4F909393028093920280914F039091F7
:1098A0005003909581959F4F9093910280939002E1
:1098B00080917E0190917F0190938D0280938C0224
:1098C000809146088B778B668093460880912908A3
:1098D0008C7B8093290888EC80935F021EC0809166
:1098E000490284FF1AC030938F0220938E02309376
:1098F00093022093920230939102209390029AE572
:109900009093540888E780932B08909304088093E1
:109910001A08109264021092650280911D089091BD
:109920001E08A0911F08B09120082091DC02309100
:10993000DD024091DE025091DF02820F931FA41FCF
:10994000B51F80931D0890931E08A0931F08B09325
:1099500020088091250890912608A0912708B091B1
:109960002808E090D402F090D5020091D602109120
:10997000D702EB82FC820D831E838E0D9F1DA01FDC
:10998000B11F8093250890932608A0932708B093D1
:1099900028088091120890911308A0911408B091A2
:1099A0001508E090D802F090D9020091DA021091E7
:1099B000DB02EF82F88609871A878E0D9F1DA01F94
:1099C000B11F8093120890931308A0931408B093CA
:1099D00015088091050890910608A0910708B0919C
:1099E0000808E090D002F090D1020091D2021091CC
:1099F000D302EB86FC860D871E878E0D9F1DA01F50
:109A0000B11F8093050890930608A0930708B093B0
:109A10000808F0906502FF86FF2029F48091640217
:109A2000882309F460C01092CC021092CD021092EB
:109A3000CE021092CF021092C8021092C902109268
:109A4000CA021092CB0210921D0810921E081092AA
:109A50001F081092200810922508109226081092D4
:109A600027081092280810921208109213081092DA
:109A7000140810921508109205081092060810920A
:109A80000708109208088091BC029091BD02A09135
:109A9000BE02B091BF028093B8029093B902A09326
:109AA000BA02B093BB028091B4029091B502A0912A
:109AB000B602B091B7028093B0029093B102A09326
:109AC000B202B093B3021092F8011092F701109213
:109AD00069021092680210926B0210926A020F855E
:109AE000002309F0D0C180916402882309F0CBC122
:109AF0008091D2059091D305815092402CF48091B1
:109B00008102882309F4BFC19090D608A0904E0628
:109B100020904A0830904B0840905A0850905B08BB
:109B200019140CF0BBC0BB24CC24DD24CA01B9013C
:109B3000A60195010E94827A79018A0180919F088D
:109B40009091A008281A390AC101AA2797FDA0956B
:109B5000BA2FE81AF90A0A0B1B0B6B817C818D81E5
:109B60009E81A60195010E94827A59016A01809125
:109B7000A1089091A208481A590AC201AA2797FD84
:109B8000A095BA2FA81AB90ACA0ADB0A292C3324CD
:109B900027FC3094432C532CC801B701A20191013A
:109BA0000E940E7A97FF04C061507E4F8F4F9F4FE7
:109BB0003B014C0109E095948794779467940A954A
:109BC000D1F7C601B501A20191010E940E7A97FF5B
:109BD00004C061507E4F8F4F9F4F5B016C0119E0B5
:109BE000D594C794B794A7941A95D1F780914E0253
:109BF00090914F02813491053CF480914C029091F8
:109C00004D0281349105D4F0D401C30197FE03C005
:109C10000196A11DB11D3C014D0195948794779447
:109C20006794D601C501D7FE03C00196A11DB11DE1
:109C30005C016D01D594C794B794A7948091D8081E
:109C4000282F332727FD3095432F532F261537050F
:109C50004805590514F439014A01992787FD909563
:109C6000909581959F4FAA2797FDA095BA2F6816CA
:109C700079068A069B0614F43C014D012A153B0522
:109C80004C055D0514F459016A01A816B906CA0607
:109C9000DB060CF0D0C05C016D01CDC0EA2CFF24C6
:109CA00000271127CA01B901A80197010E94827AF1
:109CB00039014A01C101AA2797FDA095BA2F681A58
:109CC000790A8A0A9B0A6B817C818D819E81A80119
:109CD00097010E94827A59016A01C201AA2797FD61
:109CE000A095BA2FA81AB90ACA0ADB0AD401C3017F
:109CF00097FE03C00F96A11DB11D3C014D01F4E07C
:109D00009594879477946794FA95D1F7D601C50115
:109D1000D7FE03C00F96A11DB11D5C016D01E4E0EB
:109D2000D594C794B794A794EA95D1F780914E0241
:109D300090914F02813491053CF480914C029091B6
:109D40004D0281349105A4F0C401B30123E030E059
:109D500040E050E00E94827A39014A01C601B50113
:109D600023E030E040E050E00E94827A59016A012D
:109D700080913606E82FFF27EE0FFF1FE859F84FB6
:109D8000808191810190F081E02DF7FF03C0F09573
:109D9000E195FF4F7A97A4F0C401B30123E030E0CE
:109DA00040E050E00E94827A39014A01C601B501C3
:109DB00023E030E040E050E00E94827A59016A01DD
:109DC00089E180938A0121E2621671048104910481
:109DD0002CF070E2672E712C812C912C30EE6316E2
:109DE0003FEF73063FEF83063FEF930644F460EEC8
:109DF000662E6FEF762E6FEF862E6FEF962E41E276
:109E0000A416B104C104D1042CF050E2A52EB12C4B
:109E1000C12CD12C50EEA5165FEFB5065FEFC5063D
:109E20005FEFD50644F440EEA42E4FEFB42E4FEF73
:109E3000C42E4FEFD42E8091BC029091BD02A09110
:109E4000BE02B091BF0286199709A809B90980938B
:109E5000BC029093BD02A093BE02B093BF0280915A
:109E6000B4029091B502A091B602B091B7028A19DE
:109E70009B09AC09BD098093B4029093B502A093ED
:109E8000B602B093B7028091F7019091F8018F3F2D
:109E9000910509F008F4C4C56F85662309F04EC525
:109EA00080916402882309F049C580919802882333
:109EB00009F044C570917606788B772309F43EC586
:109EC00080911D0890911E08A0911F08B091200854
:109ED000B7FF04C081509F4FAF4FBF4FE92EFA2EFE
:109EE0000B2F112707FD1A95E0921D08F0921E080E
:109EF00000931F0810932008809125089091260850
:109F0000A0912708B0912808B7FF04C081509F4F47
:109F1000AF4FBF4F892F9A2FAB2FBB27A7FDBA9505
:109F2000898B9A8BAB8BBC8B8093250890932608EA
:109F3000A0932708B093280880914E06A82EBB2432
:109F4000CC24DD242091CC023091CD024091CE0270
:109F50005091CF02C601B5010E940E7A97FF04C04E
:109F600061507F4F8F4F9F4F672E782E892E9924F7
:109F700087FC9A946092CC027092CD028092CE02BD
:109F80009092CF022091C8023091C9024091CA023A
:109F90005091CB02C601B5010E940E7A97FF04C012
:109FA00061507F4F8F4F9F4F272E382E492E5524BB
:109FB00047FC5A942092C8023092C9024092CA02C9
:109FC0005092CB028091C4029091C502A091C6022A
:109FD000B091C702B7FF04C081509F4FAF4FBF4F32
:109FE000892F9A2FAB2FBB27A7FDBA958093C40268
:109FF0009093C502A093C602B093C702D801C701CF
:10A0000086199709A809B90980931A0390931B032D
:10A01000A0931C03B0931D0320917506E22EFF242C
:10A0200000271127BC01CD01A80197010E94827A67
:10A0300059016A01209328033093290340932A038E
:10A0400050932B0389899A89AB89BC89821993091A
:10A05000A409B50980931E0390931F03A0932003C6
:10A06000B0932103BC01CD01A80197010E94827A1F
:10A0700020932C0330932D0340932E0350932F03F2
:10A08000D601C501D7FE04C081509F4FAF4FBF4FCF
:10A09000892F9A2FAB2FBB27A7FDBA959093690202
:10A0A0008093680257FF04C021503F4F4F4F5F4FCE
:10A0B000BB2757FDBA95A52F942F832F90936B0242
:10A0C00080936A0280914E0290914F0281349105F3
:10A0D000DCF480914C0290914D0281349105A4F4FE
:10A0E00080913606E82FFF27EE0FFF1FE859F84F43
:10A0F000808191810190F081E02DF7FF03C0F09500
:10A10000E195FF4F7A97E4F08091D6088F3FC1F434
:10A11000809168029091690297FD019695958795C7
:10A12000909369028093680280916A0290916B0219
:10A1300097FD01969595879590936B0280936A029F
:10A140008091120890911308A0911408B0911508FD
:10A15000B7FF04C081509F4FAF4FBF4F892F9A2F39
:10A16000AB2FBB27A7FDBA958093120890931308D5
:10A17000A0931408B09315088091050890910608E3
:10A18000A0910708B0910808B7FF04C081509F4F05
:10A19000AF4FBF4F892F9A2FAB2FBB27A7FDBA9583
:10A1A0008093050890930608A0930708B0930808C9
:10A1B0008091DC029091DD02A091DE02B091DF027D
:10A1C0002F81388549855A85281B390B4A0B5B0B33
:10A1D00020931203309313034093140350931503F9
:10A1E0008091D4029091D502A091D602B091D7026D
:10A1F000EB84FC840D851E85E81AF90A0A0B1B0BFB
:10A20000E0921603F09217030093180310931903BA
:10A2100020931A0330931B0340931C0350931D0398
:10A22000E0921E03F0921F0300932003109321037A
:10A230008091B8029091B902A091BA02B091BB028C
:10A24000821B930BA40BB50B8093B8029093B902B9
:10A25000A093BA02B093BB028091B0029091B10278
:10A26000A091B202B091B3028E199F09A00BB10B5D
:10A270008093B0029093B102A093B202B093B30264
:10A2800088898823E1F02091960230919702213845
:10A2900031054CF08091EE029091EF02019690937F
:10A2A000EF028093EE0220583F4F4CF48091EE0273
:10A2B0009091EF0201979093EF028093EE0210923B
:10A2C00097021092960281E090E09093350380937C
:10A2D0003403E0901A03F0901B0300911C031091CB
:10A2E0001D03D801C70117FF07C088279927DC0184
:10A2F0008E199F09A00BB10B81509240A040B04035
:10A3000034F084E090E0909335038093340380919F
:10A310003A0390913B03A0913C03B0913D032091FF
:10A320001D0830911E0840911F0850912008821B83
:10A33000930BA40BB50B815E914BAF4FBF4F8F5367
:10A340009C49A040B04028F08091D70889310CF496
:10A35000FFC021E0E21620E1F20620E0020720E043
:10A3600012070CF473C080913603882309F46AC085
:10A37000D801C70117FF07C088279927DC018E196C
:10A380009F09A00BB10B9C01AD01B7FF04C0215088
:10A390003E4F4F4F5F4FF9E05595479537952795BD
:10A3A000FA95D1F78091340390913503820F931F72
:10A3B0009093350380933403D801C70117FF03C07E
:10A3C0000796A11DB11DE3E0B595A79597958795D3
:10A3D000EA95D1F78093280390932903A0932A0349
:10A3E000B0932B0389589341A040B04064F088E8B3
:10A3F00093E1A0E0B0E08093280390932903A09319
:10A400002A03B0932B032091280330912903409114
:10A410002A0350912B0357FF04C021503F4F4F4F49
:10A420005F4F232F342F452F552747FD5A95809195
:10A43000680290916902820F931F90936902809342
:10A44000680206C081E08093360302C01092360392
:10A4500040E0E41640EFF4064FEF04074FEF140717
:10A460000CF073C080913703882309F46AC0D801C7
:10A47000C70117FF07C088279927DC018E199F099C
:10A48000A00BB10B9C01AD01B7FF04C021503E4FA2
:10A490004F4F5F4F69E055954795379527956A95DA
:10A4A000D1F78091340390913503820F931F9093DD
:10A4B000350380933403D801C70117FF03C0079603
:10A4C000A11DB11D23E0B595A795979587952A9570
:10A4D000D1F78093280390932903A0932A03B09384
:10A4E0002B0388579C4EAF4FBF4F64F488E79CEE18
:10A4F000AFEFBFEF8093280390932903A0932A0323
:10A50000B0932B03209128033091290340912A0313
:10A5100050912B0357FF04C021503F4F4F4F5F4FC7
:10A52000232F342F452F552747FD5A9580916802D8
:10A5300090916902820F931F909369028093680241
:10A5400011C081E0809337030DC0109237030AC019
:10A55000109235031092340384E690E090938901C1
:10A56000809388016889262F332780913403909146
:10A5700035032817390724F4309335032093340327
:10A580001091D708112379F0212F332727FD30951B
:10A5900080913403909135032817390724F43093C0
:10A5A00035032093340340911A0350911B036091AB
:10A5B0001C0370911D03413851056105710574F04C
:10A5C0008091F2029091F30220913403309135038F
:10A5D000820F931F9093F3028093F20240585F4FD3
:10A5E0006F4F7F4F74F48091F2029091F3022091AB
:10A5F000340330913503821B930B9093F3028093C5
:10A60000F20281E090E09093350380933403C09090
:10A610001E03D0901F03E0902003F0902103D70188
:10A62000C601F7FE07C088279927DC018C199D0910
:10A63000AE09BF0981509240A040B04034F084E0A0
:10A6400090E0909335038093340380913E03909182
:10A650003F03A0914003B091410320912508309120
:10A6600026084091270850912808821B930BA40BC1
:10A67000B50B815E914BAF4FBF4F8F539C49A040AC
:10A68000B04018F019310CF4FFC001E0C01600E131
:10A69000D00600E0E00600E0F0060CF473C0809104
:10A6A0003803882309F46AC0D701C601F7FE07C042
:10A6B00088279927DC018C199D09AE09BF099C01E7
:10A6C000AD01B7FF04C021503E4F4F4F5F4F09E02F
:10A6D00055954795379527950A95D1F7809134037D
:10A6E00090913503820F931F909335038093340329
:10A6F000D701C601F7FE03C00796A11DB11D13E0E7
:10A70000B595A795979587951A95D1F780932C03C2
:10A7100090932D03A0932E03B0932F038958934158
:10A72000A040B04064F088E893E1A0E0B0E08093FE
:10A730002C0390932D03A0932E03B0932F0320910D
:10A740002C0330912D0340912E0350912F0357FF7E
:10A7500004C021503F4F4F4F5F4F232F342F452FC1
:10A76000552747FD5A9580916A0290916B02820F9E
:10A77000931F90936B0280936A0206C081E08093DE
:10A78000380302C01092380320E0C21620EFD20630
:10A790002FEFE2062FEFF2060CF073C08091390321
:10A7A000882309F46AC0D701C601F7FE07C08827CD
:10A7B0009927DC018C199D09AE09BF099C01AD01E7
:10A7C000B7FF04C021503E4F4F4F5F4FE9E0559512
:10A7D000479537952795EA95D1F780913403909165
:10A7E0003503820F931F9093350380933403D70171
:10A7F000C601F7FE03C00796A11DB11D73E0B59514
:10A80000A795979587957A95D1F780932C03909388
:10A810002D03A0932E03B0932F0388579C4EAF4F68
:10A82000BF4F64F488E79CEEAFEFBFEF80932C033B
:10A8300090932D03A0932E03B0932F0320912C030C
:10A8400030912D0340912E0350912F0357FF04C0E8
:10A8500021503F4F4F4F5F4F232F342F452F552708
:10A8600047FD5A9580916A0290916B02820F931F67
:10A8700090936B0280936A0211C081E08093390348
:10A880000DC0109239030AC01092350310923403A0
:10A8900084E690E090938901809388014889242F71
:10A8A000332780913403909135032817390724F416
:10A8B00030933503209334038091D708882379F0AF
:10A8C000282F332727FD309580913403909135034D
:10A8D0002817390724F4309335032093340340912B
:10A8E0001E0350911F036091200370912103413892
:10A8F00051056105710574F08091F0029091F102AB
:10A900002091340330913503820F931F9093F1020D
:10A910008093F00240585F4F6F4F7F4FCCF480918F
:10A92000F0029091F1022091340330913503821BA3
:10A93000930B9093F1028093F0020AC010926B0285
:10A9400010926A02109269021092680210929802A4
:10A9500080912B08882341F410926B0210926A02B6
:10A96000109269021092680280911D0890911E0851
:10A97000A0911F08B091200880933A0390933B0365
:10A98000A0933C03B0933D03809125089091260845
:10A99000A0912708B091280880933E0390933F032D
:10A9A000A0934003B09341031092CC021092CD02C9
:10A9B0001092CE021092CF021092C8021092C902D9
:10A9C0001092CA021092CB021092C4021092C502D9
:10A9D0001092C6021092C70210921D0810921E0813
:10A9E00010921F0810922008109225081092260835
:10A9F000109227081092280810921208109213083B
:10AA0000109214081092150810920508109206086A
:10AA100010920708109208081092F8011092F7019E
:10AA2000E0908E02F0908F02C701F7FE04C08827E5
:10AA300099278E199F0904973CF08091460884FD60
:10AA400003C082E380936C0210914B06A12EBB24BD
:10AA5000CC24DD24B701882777FD8095982F9701B6
:10AA6000F7FE04C0222733272E193F09442737FD5C
:10AA70004095542F0E940E7A9B01AC01C601B5018E
:10AA80000E940E7A97FF04C061507E4F8F4F9F4FF8
:10AA900059E095958795779567955A95D1F79B01DC
:10AAA000812F99278E9DD0018F9DB00D9E9DB00D59
:10AAB0001124CD01B7FD03969595879595958795BA
:10AAC000280F391F80914402909145028150924095
:10AAD00010F020E030E080916E0290916F02280F1C
:10AAE000391F442737FD4095542F20930E03309390
:10AAF0000F0340931003509311038091AC02909187
:10AB0000AD02A091AE02B091AF02821B930BA40BD9
:10AB1000B50B8093AC029093AD02A093AE02B093BC
:10AB2000AF028155934CA040B04064F080E593ECB7
:10AB3000A0E0B0E08093AC029093AD02A093AE028F
:10AB4000B093AF028091AC029091AD02A091AE02A1
:10AB5000B091AF02805B9C43AF4FBF4F64F480EB7A
:10AB60009CE3AFEFBFEF8093AC029093AD02A09354
:10AB7000AE02B093AF0200918C0110918D0117FDD0
:10AB8000FCC08091460883FFF8C080918B01815002
:10AB900080938B01882309F0F4C08DE080938B01B2
:10ABA0008091DC029091DD02A091DE02B091DF0283
:10ABB000B7FF04C081509E4FAF4FBF4F39E0B595EE
:10ABC000A795979587953A95D1F77C0197FF04C093
:10ABD000F094E194F108F3948091D4029091D5021D
:10ABE000A091D602B091D702B7FF04C081509E4F0A
:10ABF000AF4FBF4F29E0B595A795979587952A95B3
:10AC0000D1F79C0197FF03C0309521953F4FE21685
:10AC1000F3060CF47901B701F7FE02C0695F7F4FBC
:10AC20002B0183E0559447948A95E1F722E030E0C8
:10AC3000420E531E60905608709057088090580836
:10AC40009090590820913E0130913F014091400180
:10AC500050914101C401B3010E94827A59016A01F5
:10AC60003093030820930208021B130BC801845E73
:10AC70009D4F68E671E00E944D7A9C01245B304054
:10AC80008091880190918901009731F0019790930C
:10AC90008901809388011BC049E1E416F104BCF4EA
:10ACA0008091960290919702820F931F9093970242
:10ACB0008093960280916C02882349F081508093A2
:10ACC0006C02882321F4B0929B02A0929A02809198
:10ACD000880190918901892BF9F480918A01992743
:10ACE000289FB001299F700D389F700D1124CB0152
:10ACF000B2010E944D7ACB01AA2797FDA095BA2FE9
:10AD0000680E791E8A1E9B1E609256087092570824
:10AD1000809258089092590880916C02882369F5B6
:10AD200080919A0290919B02209102083091030831
:10AD3000821B930B845E9D4F68E671E00E944D7A02
:10AD40009C01245B30408091750186959927289F4E
:10AD5000D001299FB00D389FB00D11249D01B7FF80
:10AD600002C0215F3F4F04E0359527950A95E1F732
:10AD700030936F0220936E0204C010926F02109203
:10AD80006E0280919802882381F01092A0021092A6
:10AD9000A1021092A2021092A3021092A402109299
:10ADA000A5021092A6021092A702F0906502FF2061
:10ADB000F1F480912B08282F3327442755278091C1
:10ADC000DC029091DD02A091DE02B091DF02BC01B5
:10ADD000CD010E940E7ADC01CB01BC01CD0128EF30
:10ADE0003AE240E050E00E94827A390102C06624D3
:10ADF0007724E0906402EE20F1F480912B08282F54
:10AE00003327442755278091D4029091D502A091F1
:10AE1000D602B091D702BC01CD010E940E7ADC01AE
:10AE2000CB01BC01CD0128EF3AE240E050E00E94A6
:10AE3000827A290102C0442455248091FF07909111
:10AE40000008893C91051CF088EC90E005C088530F
:10AE50009F4F34F488E39FEF909300088093FF079F
:10AE600080910A0890910B08893C91051CF088ECB0
:10AE700090E005C088539F4F34F488E39FEF909390
:10AE80000B0880930A0880910C0890910D08AA275E
:10AE900097FDA095BA2F20915408A22EBB24CC2454
:10AEA000DD24BC01CD01A60195010E940E7A9B0113
:10AEB000AC018091FF0790910008AA2797FDA0950B
:10AEC000BA2F17E0880F991FAA1FBB1F1A95D1F739
:10AED000280F391F4A1F5B1F57FF04C0215C3F4FDB
:10AEE0004F4F5F4FA6E05595479537952795AA9503
:10AEF000D1F78301020F131F10930D0800930C0864
:10AF00008091FD079091FE07AA2797FDA095BA2F83
:10AF1000BC01CD01A60195010E940E7A9B01AC01F6
:10AF200080910A0890910B08AA2797FDA095BA2F47
:10AF3000F7E0880F991FAA1FBB1FFA95D1F7280FBA
:10AF4000391F4A1F5B1F57FF04C0215C3F4F4F4F03
:10AF50005F4FE6E05595479537952795EA95D1F7E8
:10AF60004201820E931E9092FE078092FD0780910F
:10AF70004F0890915008880F991FAA2797FDA09518
:10AF8000BA2F20910408332744275527BC01CD014F
:10AF90000E940E7A5B016C0197FF08C02FE330E03E
:10AFA00040E050E0A20EB31EC41ED51E76E0D5943C
:10AFB000C794B794A7947A95D1F780911A08282F4F
:10AFC0003327442755278091C0029091C102A09158
:10AFD000C202B091C302BC01CD010E940E7ADC0115
:10AFE000CB01BC01CD0120EF35E540E050E00E94EF
:10AFF000827AB501620F731F7093500860934F08F7
:10B000000150104134F080E090E190930D0880935E
:10B010000C0880910C0890910D088050904F34F4EA
:10B0200080E090EF90930D0880930C0851E0851616
:10B0300050E1950634F080E090E19093FE07809314
:10B04000FD078091FD079091FE078050904F34F4EA
:10B0500080E090EF9093FE078093FD076150704170
:10B0600034F080E090E19093500880934F088091F5
:10B070004F08909150088050904F34F480E090EF4A
:10B080009093500880934F0880910101482F5527D5
:10B0900080912201909123014817590794F420913F
:10B0A00022013091230109811A81049FC001059F6B
:10B0B000900D149F900D1124B9010E94397A7A8362
:10B0C000698329813A81220F331F220F331F3A836C
:10B0D00029838091460880FD02C00C94CC60EE204C
:10B0E00011F00C94CC60FF2011F00C94CC60809196
:10B0F000A70399278F779070009711F00C94CC607C
:10B100004C012091F4023091F5022115310509F02E
:10B1100044C080911801909119018959934058F0C9
:10B1200087B5853F20F48091FB01815011C081E0FB
:10B1300080934D0353C0809118019091190184367A
:10B14000910530F587B58B30F8F08091FB018F5F6A
:10B150008093FB019AE08902900111248091DE0521
:10B16000821B87BD87B5809588BD8CE291E0909366
:10B17000E4018093E3018EE591E09093F5028093E2
:10B18000F4020E94611A2AC081E080934C0326C019
:10B19000F0924C03F0924D0321C09093FA018093FA
:10B1A000F90180917C0290917D02A0917E02B09184
:10B1B0007F0254E0880F991FAA1FBB1F5A95D1F731
:10B1C0008093FC019093FD01A093FE01B093FF01D9
:10B1D000215030403093F5022093F40280914608CC
:10B1E00020915F0281FF25C02233E8F480918E0117
:10B1F000815080938E018F3FE1F5109299028091EA
:10B200007C0290917D02A0917E02B0917F0280939A
:10B21000780290937902A0937A02B0937B0281E046
:10B2200080938E0126C0273420F188EC80938E0114
:10B230001DC08091420190914301820F911D209188
:10B2400044063327829FA001839F500D929F500D8B
:10B250001124CA01AA2797FDA095BA2F80937802DE
:10B2600090937902A0937A02B0937B0281E080935D
:10B2700099028091DC029091DD02A091DE02B091F2
:10B28000DF02E0903E01F0903F01009140011091FB
:10B290004101BC01CD01A80197010E94827A5901A8
:10B2A0006A018091D4029091D502A091D602B0910A
:10B2B000D702BC01CD01A80197010E94827AB90191
:10B2C000C5010E9437789093170880931608CC9791
:10B2D00034F08CE390E090931708809316088091E7
:10B2E0001608909117080E94246D90931708809378
:10B2F000160880E280933D01109277021092760248
:10B3000080919902882309F4ABC58091490299275D
:10B310009C012071307084FDA3C580914802826039
:10B320008093480270912908872F992741E0C42E05
:10B33000D12CC822D92280FD04C08091460881FD0D
:10B3400010C0E980FA803093430320934203309386
:10B3500077022093760280914902806C80934902A3
:10B36000DFC28091490281FFAEC200917E0110913F
:10B370007F01C8010F96A0908C02B0908D028A15B3
:10B380009B050CF06EC080914C03882309F069C0C6
:10B390008091440390914503459784F08091EF019B
:10B3A0009091F001A091F101B091F20180937802A7
:10B3B00090937902A0937A02B0937B028091490224
:10B3C00087FF15C0809149028F7780934902809151
:10B3D000EF019091F001A091F101B091F201809301
:10B3E000780290937902A0937A02B0937B028091C5
:10B3F0004902806480934902E0900908EE20F1F050
:10B400008091780290917902A0917A02B0917B02AA
:10B41000BC01CD0124E630E040E050E00E94827A99
:10B420008E2D9927AA27BB2782179307A407B50754
:10B430002CF4D0927702C092760210C0C501801B16
:10B44000910B0F9797FF03C0909581959F4F909315
:10B450007702809376028BE280933D011092700216
:10B4600034C1C8010F97A816B906C4F520914D0341
:10B470002223A1F58091490286FF15C080914902DF
:10B480008F7B809349028091EF019091F001A09110
:10B49000F101B091F2018093780290937902A09328
:10B4A0007A02B0937B0280914902806880934902BE
:10B4B000C501801B910B0F9697FF03C09095819556
:10B4C0009F4F909581959F4F90937702809376023E
:10B4D0008DE280933D0120937002F7C08DE380934D
:10B4E0003D0160917102662371F1209172023091E9
:10B4F000730240917402509175028091780290918C
:10B500007902A0917A02B0917B0282179307A40777
:10B51000B507CCF480914902806480934902862F5C
:10B52000992790937702809376028AE08093700245
:10B530008EE580933D018091490287FFC6C08091CE
:10B5400049028F7733C0662309F443C02091720209
:10B55000309173024091740250917502809178028B
:10B5600090917902A0917A02B0917B022817390755
:10B570004A075B0774F5809149028068809349020D
:10B58000862F9927909581959F4F9093770280936E
:10B59000760286EF8093700286E780933D0180916A
:10B5A000490286FF92C0809149028F7B80934902B5
:10B5B0008091EF019091F001A091F101B091F20121
:10B5C0008093780290937902A0937A02B0937B02E1
:10B5D0007CC080914902807C09F477C08091700220
:10B5E000882309F04CC08091EF019091F001A09167
:10B5F000F101B091F201885C9040A040B0402091F0
:10B6000078023091790240917A0250917B02821740
:10B610009307A407B5076CF08091EF019091F001BA
:10B62000A091F101B091F201885C9040A040B0403F
:10B630001DC08091EF019091F001A091F101B091B6
:10B64000F20188539F4FAF4FBF4F281739074A0762
:10B650005B07BCF08091EF019091F001A091F101A6
:10B66000B091F20188539F4FAF4FBF4F8093780244
:10B6700090937902A0937A02B0937B0202C0109259
:10B680007002809149028F738093490210924303A4
:10B690001092420371FF06C084EF91E09093E401A1
:10B6A0008093E30180918002882379F480917C0269
:10B6B00090917D02A0917E02B0917F02C397A10577
:10B6C000B1051CF081E0809380026091420370918B
:10B6D00043038091760290917702680F791F7093EF
:10B6E000430360934203CB0177FF04C08827992767
:10B6F000861B970B855F91400CF4CEC04091700281
:10B70000442389F180917202909173022091780212
:10B7100030917902821B930B0996439748F48091EC
:10B72000720290917302A0917402B091750212C0DE
:10B73000242F332727FD3095432F532F80917802F4
:10B7400090917902A0917A02B0917B02820F931FAF
:10B75000A41FB51F8093780290937902A0937A0278
:10B76000B0937B0224C080914406209178023091EE
:10B77000790240917A0250917B021616170644F422
:10B7800063E00E942D7A280F311D411D511D07C015
:10B7900063E00E942D7A281B310941095109209349
:10B7A00078023093790240937A0250937B02109290
:10B7B000430310924203E0907C02F0907D020091DE
:10B7C0007E0210917F02D801C70180509440A040B2
:10B7D000B040209178023091790240917A025091E4
:10B7E0007B0282179307A407B5075CF4D801C70151
:10B7F00080509C4FAF4FBF4F281739074A075B0750
:10B8000044F08093780290937902A0937A02B093E7
:10B810007B028091290881FF06C084E690E0909326
:10B82000E4018093E301809148068823A9F5809183
:10B830007102882389F5409166025091670257FF93
:10B8400002C04D5F5F4F559547955595479580913F
:10B85000220190912301209101013327489FB001DB
:10B86000499F700D589F700D1124CB01B9010E94A2
:10B870004D7A70937F0160937E01663471051CF4EC
:10B8800086E490E005C06739710534F086E990E000
:10B8900090937F0180937E018091F4029091F50254
:10B8A000892BD1F18091EF019091F001A091F101EC
:10B8B000B091F2018093780290937902A0937A027A
:10B8C000B0937B0229C080917C0290917D02A0916F
:10B8D0007E02B0917F0280599140A040B040809399
:10B8E000780290937902A0937A02B0937B028091C0
:10B8F0004806882311F0992702C088E790E09093CA
:10B900007F0180937E0189819A8190936702809361
:10B9100066028EE280933D01E0906602F09067023D
:10B920008091EF019091F001A091F101B091F201AD
:10B93000209178023091790240917A0250917B02F5
:10B94000281739074A075B0724F08091290880FDF2
:10B95000D3C280914102882309F0CEC28091F402C3
:10B960009091F502892B49F0E0906602F090670211
:10B970001092450310924403E1C08091EF01909131
:10B98000F001A091F101B091F201821B930BA40B85
:10B99000B50B8093120390931303A0931403B093F9
:10B9A00015038230E0E89E07EFEFAE07EFEFBE072A
:10B9B0002CF481E090E8AFEFBFEF09C08F5F9F47A5
:10B9C000A040B04064F08FEF9FE7A0E0B0E080932C
:10B9D000120390931303A0931403B0931503809163
:10B9E0001203909113039093450380934403809135
:10B9F0007701282F332744275527809112039091F0
:10BA00001303A0911403B0911503BC01CD010E9452
:10BA10000E7A97FF04C0615E7F4F8F4F9F4F25E0E6
:10BA200095958795779567952A95D1F76093120339
:10BA300070931303809314039093150365300EEFF6
:10BA400070070FEF80070FEF90072CF484E09EEF54
:10BA5000AFEFBFEF09C0605074408040904064F089
:10BA600080E094E0A0E0B0E0809312039093130391
:10BA7000A0931403B09315038090120390901303C6
:10BA80002091F9013091FA0137FF02C0295F3F4F41
:10BA900003E0359527950A95E1F74FEF22383407F3
:10BAA0001CF421E83FEF05C02038310514F020E8F0
:10BAB00030E0C901AA2797FDA095BA2F20917801FF
:10BAC000332744275527BC01CD010E940E7A97FFEA
:10BAD00004C06D5F7F4F8F4F9F4F12E09595879504
:10BAE000779567951A95D1F79B015FEF61307507E0
:10BAF0001CF420E03FEF06C06F3F710519F014F011
:10BB000020E031E080914902807C49F0C90137FD95
:10BB100003969C0135952795359527950DC0809105
:10BB2000290880FF09C0C90137FD07969C01A3E0E1
:10BB300035952795AA95E1F7820E931E20917601FF
:10BB4000222309F454C060919C0270919D0280915F
:10BB50009E0290919F0297FF04C061587F4F8F4FC4
:10BB60009F4FF7E09595879577956795FA95D1F76B
:10BB70003327442755270E940E7A97FF04C0615E41
:10BB80007F4F8F4F9F4FE5E0959587957795679508
:10BB9000EA95D1F760931203709313038093140313
:10BBA000909315036138AFEF7A07AFEF8A07AFEFD5
:10BBB0009A072CF480E89FEFAFEFBFEF0AC06F3F0A
:10BBC00071058105910569F064F080E091E0A0E0E5
:10BBD000B0E08093120390931303A0931403B093E7
:10BBE00015038091120390911303880E991E809182
:10BBF0007401282F33278091DA08992787FD9095C3
:10BC0000289FF001299FF00D389FF00D11249F010E
:10BC1000F7FF02C021583F4F220F232F221F330B63
:10BC2000FFEF21383F071CF420E83FEF06C02F3F0D
:10BC3000310519F014F020E031E0280D391DC9015B
:10BC4000AA2797FDA095BA2F00916602109167026E
:10BC50009801442737FD4095542FBC01CD010E9427
:10BC60000E7A97FF04C061507E4F8F4F9F4F59E06F
:10BC700095958795779567955A95D1F7E61AF70ABE
:10BC80008091760290917702892B09F064C010169A
:10BC900011060CF060C02091440330914503C901A6
:10BCA00037FF03C0309521953F4F2D33310540F4C8
:10BCB00080919402909195028E159F0574F526C08F
:10BCC0002C53304045E0369527954A95E1F72031D1
:10BCD000310510F02FE030E0409194025091950230
:10BCE00018161906E4F480E190E0821B930B489F3C
:10BCF0009001499F300D589F300D1124B4E03695C6
:10BD00002795BA95E1F72E153F0520F580917C0126
:10BD100090917D01E816F906F4F07C011CC0205FCB
:10BD20003F4F80917C0190917D01829FB001839F64
:10BD3000700D929F700D11249B01A4E036952795FC
:10BD4000AA95E1F74E155F0514F07A0104C0E216DA
:10BD5000F30608F07901C701AA2797FDA095BA2F2D
:10BD6000FDE0880F991FAA1FBB1FFA95D1F72091FC
:10BD7000160830911708442737FD4095542FBC0111
:10BD8000CD010E94827A20931603309317034093CB
:10BD9000180350931903E0901603F0901703809155
:10BDA0004603909147039C01220F331F280F391F30
:10BDB0002E0D3F1D37FF02C02D5F3F4FA901559546
:10BDC0004795559547955093470340934603809177
:10BDD0004006282F3327220F331F220F331F24172B
:10BDE00035076CF480914E08282F3327220F331F1C
:10BDF000220F331F205530404217530724F0309351
:10BE00004703209346038091290880FF14C0809146
:10BE1000460390914703A981BA818A179B0724F0B2
:10BE2000B0934703A0934603E0914603F091470384
:10BE3000FA83E98361C029813A81201B310B37FFE6
:10BE400002C02D5F3F4F3595279535952795E0909A
:10BE50004603F0904703E20EF31EFA82E9824CC0DB
:10BE600080914806882301F560916602709167020F
:10BE700077FF02C06D5F7F4F7595679575956795E4
:10BE8000409122015091230180910101282F3327F5
:10BE9000649FC001659F900D749F900D1124B9019E
:10BEA0000E944D7ACB0101C0992790937F01809326
:10BEB0007E0180917E0190917F01873491051CF471
:10BEC00086E490E005C08639910534F086E990E07B
:10BED00090937F0180937E0109811A81109347031B
:10BEE0000093460380914902806C809349028091BF
:10BEF00048028D7F809348028091490299279C01D6
:10BF00002270307081FF39C18091480390914903BC
:10BF1000A0914A03B0914B030097A105B10521F010
:10BF2000809180028130B9F480916602909167021D
:10BF3000AA2797FDA095BA2F1EE0880F991FAA1F68
:10BF4000BB1F1A95D1F78093480390934903A093A0
:10BF50004A03B0934B0380918002813019F482E050
:10BF60008093800229813A8179010027F7FC0095AE
:10BF7000102F80911608909117089C01442737FDD7
:10BF80004095542FC801B7010E940E7ADC01CB0105
:10BF90008093160390931703A0931803B09319038B
:10BFA000B7FF04C08150904EAF4FBF4F7C018D0151
:10BFB000ADE015950795F794E794AA95D1F7E0922F
:10BFC0001603F0921703009318031093190360915E
:10BFD0004A0270914B023FE0603A730750F580913E
:10BFE000480390914903A0914A03B0914B039C01EF
:10BFF000AD01FAE05695479537952795FA95D1F713
:10C00000821B930BA40BB50BA8019701E4E0220F50
:10C01000331F441F551FEA95D1F7820F931FA41FAA
:10C02000B51F8093480390934903A0934A03B093AC
:10C030004B0360547F4118F5809148039091490368
:10C04000A0914A03B0914B039C01AD016CE0569561
:10C050004795379527956A95D1F7821B930BA40BCB
:10C06000B50BA8019701F2E0220F331F441F551FA3
:10C07000FA95D1F7820F931FA41FB51F41C080917D
:10C08000F9019091FA018091F9019091FA0197FFDD
:10C0900003C0909581959F4F84369105CCF5809192
:10C0A000EF019091F001A091F101B091F2019C019A
:10C0B0008091780290917902281B390B37FF03C0D9
:10C0C000309521953F4F2F3F310509F00CF58091B8
:10C0D000480390914903A0914A03B0914B039C01FE
:10C0E000AD01EEE05695479537952795EA95D1F73E
:10C0F000821B930BA40BB50B8E0D9F1DA01FB11FB0
:10C100008093480390934903A0934A03B0934B0351
:10C110008091480390914903A0914A03B0914B0349
:10C120007EE0B695A795979587957A95D1F79093E8
:10C1300067028093660240914606442399F0552792
:10C140009C01BA010E944D7AC901861B970B9093FE
:10C15000950280939402260F371F30937D01209320
:10C160007C011FC010929502109294028FEF93E011
:10C1700090937D0180937C0114C0109280021092F4
:10C1800048031092490310924A0310924B033093D4
:10C1900067022093660205C080914902806C8093FB
:10C1A000490280915C0381FF37C089819A8197FDA4
:10C1B00003969595879595958795209146023091A0
:10C1C00047022817390760F4809166029091670250
:10C1D000892B31F0220F331F220F331F3A8329831B
:10C1E0008091EF019091F001A091F101B091F201E5
:10C1F0008093780290937902A0937A02B0937B02A5
:10C2000088E99AE39093E4018093E30180E09EE063
:10C2100090930B0180930A0120911108822F992796
:10C22000880F991F880F991F889669817A818617D0
:10C23000970714F09A83898370914E087D8B872F1E
:10C240009927880F991F880F991F80559040A981C1
:10C25000BA818A179B0714F49A83898380913102EB
:10C26000882341F48091E1088F3F21F4809160039D
:10C270008823E9F080914A0290914B020297C0977F
:10C28000B0F4E981FA811E161F068CF481E090E07B
:10C2900090934B0280934A02E22EFF24EE0CFF1C87
:10C2A000EE0CFF1C8701085D1F4F1A83098329814B
:10C2B0003A8130939C0520939B0580910E039091C9
:10C2C0000F03A0911003B091110312E0880F991F82
:10C2D000AA1FBB1F1A95D1F700914F081091500863
:10C2E000081B190B213A31058CF0C90137FD019665
:10C2F00095958795801791070CF48C019095819501
:10C300009F4F081719076CF48C010BC001351105FC
:10C3100014F000E510E03FEF003B130714F400EBCE
:10C320001FEF4D89242F3327220F331F220F331F76
:10C33000C90169817A81861B970B801791070CF4DC
:10C340008C0189819A81821B930B081719070CF4C1
:10C350008C0180910C0890910D086091920270916F
:10C360009302861B970B90931C0880931B08D09018
:10C370002B082091A4023091A5024091A602509171
:10C38000A702DD2041F0661A770AC301AA2797FDAC
:10C39000A095BA2F04C0AA2797FDA095BA2F280F01
:10C3A000391F4A1F5B1F2093A4023093A5024093BC
:10C3B000A6025093A7028091A4029091A502A09199
:10C3C000A602B091A70281509A4FA040B04064F0FD
:10C3D00080E09AEFA0E0B0E08093A4029093A502E1
:10C3E000A093A602B093A7028091A4029091A50207
:10C3F000A091A602B091A70280509640AF4FBF4FC8
:10C4000064F480E096E0AFEFBFEF8093A4029093D6
:10C41000A502A093A602B093A702C0905506209152
:10C420001B0830911C0878E0E72EEC1498F08C2D56
:10C430009927829FA001839F500D929F500D112438
:10C44000CA0157FD07967C0163E0F594E7946A956D
:10C45000E1F712C08C2D86959927829FB001839FAA
:10C46000700D929F700D1124CB0177FD03967C0116
:10C47000F594E794F594E794A0907901B0907A014F
:10C480009501442737FD4095542F8091A402909147
:10C49000A502A091A602B091A702BC01CD010E9405
:10C4A000827AE20EF31E90906301692D7727882728
:10C4B0009927980117FF04C022273327201B310B2F
:10C4C00037FF02C02F5F3F4F35952795A981BA816D
:10C4D0002A0F3B1F442737FD4095542F0E940E7AA8
:10C4E00097FF04C0615C7F4F8F4F9F4F26E095956B
:10C4F0008795779567952A95D1F79B016E157F05EE
:10C500000CF47B01309521953F4FE216F3060CF4B5
:10C5100079018091FD079091FE07609190027091E2
:10C520009102861B970B9093FC078093FB07209149
:10C53000A0023091A1024091A2025091A302DD20FD
:10C5400041F0461A570AC201AA2797FDA095BA2FB3
:10C5500004C0AA2797FDA095BA2F280F391F4A1F9C
:10C560005B1F2093A0023093A1024093A20250933C
:10C57000A3028091A0029091A102A091A202B09189
:10C58000A30281509A4FA040B04064F080E09AEF3F
:10C59000A0E0B0E08093A0029093A102A093A20239
:10C5A000B093A3028091A0029091A102A091A20257
:10C5B000B091A30280509640AF4FBF4F64F480E02B
:10C5C00096E0AFEFBFEF8093A0029093A102A093FB
:10C5D000A202B093A3022091FB073091FC0748E030
:10C5E0004C1598F08C2D9927829FB001839F700D78
:10C5F000929F700D1124CB0177FD07966C0193E09B
:10C60000D594C7949A95E1F712C0C6948C2D9927BA
:10C61000829FD001839FB00D929FB00D1124CD0158
:10C62000B7FD03966C01D594C794D594C794950132
:10C63000442737FD4095542F8091A0029091A1028C
:10C64000A091A202B091A302BC01CD010E94827A06
:10C65000C20ED31E692D772788279927980117FFC7
:10C6600004C022273327201B310B37FF02C02F5F66
:10C670003F4F35952795E981FA812E0F3F1F4427BB
:10C6800037FD4095542F0E940E7A97FF04C0615CDD
:10C690007F4F8F4F9F4FA6E095958795779567952C
:10C6A000AA95D1F79B016C157D050CF46B013095B3
:10C6B00021953F4FC216D3060CF4690180911108F1
:10C6C000282E332450909706F7E08F2EF7E09F2E08
:10C6D000EEEBAE2EE6E0BE2E7BE0472E6CE2662E41
:10C6E00068E0762ED5012C9112160CF029C1203469
:10C6F00029F4E981FA81FF8BEE8B1FC049815A81B1
:10C70000CA01AA2797FDA095BA2F332727FD309598
:10C71000432F532FBC01CD010E940E7A97FF04C016
:10C72000615C7F4F8F4F9F4F56E09595879577952A
:10C7300067955A95D1F77F8B6E8BF5012181203457
:10C7400039F42E893F892E0D3F1D3F8B2E8B2AC039
:10C75000203C39F44E895F894E195F095F8B4E8BFF
:10C7600021C0C701AA2797FDA095BA2F332727FD1F
:10C770003095432F532FBC01CD010E940E7A97FFB5
:10C7800004C0615C7F4F8F4F9F4F46E09595879522
:10C79000779567954A95D1F7AE89BF89A60FB71FE0
:10C7A000BF8BAE8BF5012281203439F42E893F896D
:10C7B0002C0D3D1D3F8B2E8B2AC0203C39F44E8919
:10C7C0005F894C195D095F8B4E8B21C0C601AA277A
:10C7D00097FDA095BA2F332727FD3095432F532F70
:10C7E000BC01CD010E940E7A97FF04C0615C7F4FAF
:10C7F0008F4F9F4F36E095958795779567953A953A
:10C80000D1F7AE89BF89A60FB71FBF8BAE8BF501DD
:10C810002381203439F42E893F89200F311F3F8B2B
:10C820002E8B2AC0203C39F44E895F89401B510B66
:10C830005F8B4E8B21C0C801AA2797FDA095BA2F08
:10C84000332727FD3095432F532FBC01CD010E9484
:10C850000E7A97FF04C0615C7F4F8F4F9F4F26E099
:10C8600095958795779567952A95D1F7AE89BF8974
:10C87000A60FB71FBF8BAE8BF301808191812E89EC
:10C880003F898217930764F4B901680F791F77FF16
:10C8900002C06F5F7F4F759567957F8B6E8B1DC054
:10C8A000552049F44E895F89440F551F481B590B89
:10C8B0005F8B4E8B12C051E0551578F4252D332730
:10C8C0006E897F89861B970BB9010E944D7AAE89CC
:10C8D000BF89A60FB71FBF8BAE8BC101880F991FF1
:10C8E000880F991FEE89FF898E179F0764F4FD89D1
:10C8F0008F2F9927880F991F880F991F2E893F899D
:10C900002817390714F09F8B8E8B8E899F8997FD8E
:10C9100003969595879595958795F4018183880F62
:10C92000991F880F991F2E893F89281B390BC90130
:10C93000880F8283EE89FF89D301ED93FC9303C0B6
:10C94000F401118212824A9422E030E0620E731EDA
:10C9500044E050E0A40EB51E68E070E0860E971E1D
:10C9600047FEC0CEE2E1C95E0C94B97A84B1806A18
:10C9700084B93D9A82E58CBD1DBC459A81E08093C7
:10C9800060088AEA8093710883E8809372088AE0DD
:10C9900080937308109275081092740810927708AB
:10C9A000109276081092D908109295080895309147
:10C9B0006008332309F070C00DB407FE6DC083E03A
:10C9C0008093E201459A2EB58091630399278130C7
:10C9D000910589F0823091051CF4892B21F03EC02D
:10C9E0000297B9F03BC03093940820936403213838
:10C9F000A9F581E008C0253549F480916403820FD0
:10CA00008093640382E08093630328C030936303C0
:10CA100025C080919408E82FFF27EA54F74F208320
:10CA20008F5F80939408909164038032A0F029175F
:10CA300069F480E2A6EBB8E0E6E9F8E00D90019237
:10CA40008A95E1F781E08093950802C030939508BC
:10CA50001092630303C0920F9093640320917008B7
:10CA60002232A0F445980000000000000000E09190
:10CA70006908F0916A08E20FF11D80818EBD8091F6
:10CA800092089081890F8093920803C081E080937F
:10CA900060082F5F209370080895EF92FF920F9324
:10CAA0001F9380914E069927880F991F880F991F11
:10CAB0007C010027F7FC0095102F8091DC029091FB
:10CAC000DD02A091DE02B091DF02BC01CD01A80120
:10CAD00097010E94827A30937508209374088091A0
:10CAE000D4029091D502A091D602B091D702BC0198
:10CAF000CD01A80197010E94827A30937708209394
:10CB00007608209156083091570840915808509166
:10CB10005908DA01C90173E0880F991FAA1FBB1FCA
:10CB20007A95D1F7820F931FA41FB51F820F931F11
:10CB3000A41FB51F20913E0130913F01409140015B
:10CB400050914101BC01CD010E94827A30937D0851
:10CB500020937C088091EE029091EF0220910602D2
:10CB600030910702821B930B909383088093820875
:10CB7000E091E402F091E50280912208909123086F
:10CB8000BF010E944D7ACB019B01220F331F220F60
:10CB9000331F280F391F280F391F37FF02C02D5FA1
:10CBA0003F4F3595279535952795309379082093F4
:10CBB00078088091520890915308BF010E944D7AE5
:10CBC0009B01220F331F220F331F260F371F260F03
:10CBD000371F37FF02C02D5F3F4F3595279535959D
:10CBE000279530937B0820937A081092E5021092E3
:10CBF000E402109223081092220810925308109217
:10CC00005208809173089927AA27BB27FC013A97FD
:10CC1000E830F10508F016C2E758FF4F0C94D47ABB
:10CC200080915E028093860880915D0280938708E0
:10CC300080915C028093880880915B0280938908D0
:10CC400080915A0280938A088091590280938B08C0
:10CC50008091580280938C088091570280938D08B0
:10CC60008091490280938E0880914902837F80934E
:10CC700049028091000180938F08809198068093EB
:10CC8000900880914802809391084299DBC180917D
:10CC90004802877F80934802D5C18091DB0890913C
:10CCA000DC0890938708809386088091DF08909134
:10CCB000E0089093890880938808809122019091E0
:10CCC000230180938A08809183060E94E33F80932A
:10CCD0008B0880913D0180938C089091650390931F
:10CCE0008D08E92FFF2713E0EE0FFF1F1A95E1F7DC
:10CCF000E95FF84F868180938E08838180938F0847
:10CD00008781809390088581809391089F5F90939D
:10CD10006503E92FFF27EE0FFF1FEE0FFF1FEF54F4
:10CD2000F94F8585882309F08DC1992309F48AC1BB
:10CD3000892F992701966CE070E00E944D7A9C0142
:10CD4000982FE82FFF27EE0FFF1FEE0FFF1FEF5466
:10CD5000F94F8585882311F4222351F72093650329
:10CD600071C180910101809386088091840680932F
:10CD70008708809185068093880880918606809335
:10CD800089088091870680938A0880918B0680931A
:10CD90008B0880918C0680938C0880918D068093FF
:10CDA0008D088091900680938E0880918E068093E6
:10CDB0008F0880918F06809390088091910640C1E2
:10CDC00080918206809386081092870880919F0642
:10CDD0008093880837C1F89480913506E82FFF27A3
:10CDE000EE0FFF1FE859F84F0190F081E02DE03879
:10CDF000F1051CF0EFE7F0E006C02FEFE138F20795
:10CE000014F4E1E8FFEFE093860880913606E82FFE
:10CE1000FF27EE0FFF1FE859F84F0190F081E02D3A
:10CE2000E038F1051CF0EFE7F0E006C07FEFE138F5
:10CE3000F70714F4E1E8FFEFE093870880913406E8
:10CE4000E82FFF27EE0FFF1FE859F84F0190F08100
:10CE5000E02DE038F1051CF0EFE7F0E006C08FEFC1
:10CE6000E138F80714F4E1E8FFEFE09388088091D7
:10CE70003306E82FFF27EE0FFF1FE859F84F019008
:10CE8000F081E02DE038F1051CF0EFE7F0E006C09E
:10CE90002FEFE138F20714F4E1E8FFEF7894E09324
:10CEA00089088091830280938A088091840280930C
:10CEB0008B088091850280938C08809186028093F4
:10CEC0008D088091870280938E08809188028093DC
:10CED0008F08809189028093900880918A02B0C067
:10CEE0008091C203863018F01092C20385E08093CF
:10CEF0008608809192068093870880917C029091A9
:10CF00007D02A0917E02B0917F02BC01CD0125E09F
:10CF100030E040E050E00E94827A3093890820930C
:10CF200088088091780290917902A0917A02B0915C
:10CF30007B02BC01CD0125E030E040E050E00E94E2
:10CF4000827A30938B0820938A0880918806809398
:10CF50008C088091890680938D0880918A06809341
:10CF60008E088091820280938F088091660380935F
:10CF7000900880919B0590919C0597FD039695954F
:10CF80008795959587955CC082E08093860810927E
:10CF9000870885E08093880888E3809389088091DA
:10CFA000020180938A088091A70380938B08909157
:10CFB000A80390938C088F778093A7039071909328
:10CFC000A80310928D088091460880938E08809166
:10CFD000290880938F08809194068093900880910F
:10CFE000A3062EC080916706809386088091A106D3
:10CFF0008093870880916B018093880880916006F8
:10D00000809389088091610680938A0880916206E6
:10D0100080938B0880916A0180938C0880916406CC
:10D0200080938D088091650680938E0880916606B6
:10D0300080938F088091E108809390088091C505C6
:10D040008093910880919508882309F451C16091DB
:10D05000960880919F01681719F08AEF80939D01CF
:10D0600060939F0181E080938B01409197085091DC
:10D070009808CA0181509E4F8F5F9340B0F4209171
:10D08000990830919A08C90181509E4F8F5F934053
:10D0900060F480913F0685FF08C05093520340938F
:10D0A00051033093500320934F0380919D0890913A
:10D0B0009E0821E08936920724F490938D01809395
:10D0C0008C012091A7083091A8088091E3019091EC
:10D0D000E4018217930740F48091B601882321F47C
:10D0E0003093E4012093E301862F99278836910538
:10D0F00009F468C08936910524F48736910551F00A
:10D10000FFC08936910509F496C08B36910509F464
:10D11000E2C0F6C08091A9088093D6088091AA0841
:10D120008093D8088091AB088093D7088091AC0891
:10D1300080938A018091AD088093DA088091AE08CF
:10D1400080939E018091AF08809362038091B00824
:10D1500080934E03809156028823F9F02091B10804
:10D160003091B20837FD19C030939B0220939A0288
:10D1700090916906992389F08FE0989FC00111244E
:10D18000281B390BC90188599E4F68E671E00E943F
:10D190004D7A90939B0280939A022091590330918B
:10D1A0005A038091B3089091B408280F391F37FFB4
:10D1B00002C02F5F3F4F3595279530935A03209338
:10D1C00059039EC08091A90880936B088091AA089A
:10D1D00080936C088091AB0880936D088091AC08B7
:10D1E00080936E088091AD0880936F0880918B05C5
:10D1F0009091AE08892B80938B0590918C0593704C
:10D200008091AF088C70982B90938C058091B0081A
:10D21000809360038091B10880938F018091B20860
:10D220008093D9088091B30880935C038091B408FF
:10D2300080935B0365C08091A90880936108809109
:10D24000AA08809362088091AB088093630880915C
:10D25000AC08809364088091AD089091AE089093DB
:10D260006608809365088091AF089091B00890930C
:10D270006808809367088091B108992787FD909589
:10D280009093A3078093A2078091B20880937102C4
:10D290008091B3089091B4089C01442737FD4095D4
:10D2A000542FDA01C90163E0880F991FAA1FBB1F21
:10D2B0006A95D1F7820F931FA41FB51F820F931F8A
:10D2C000A41FB51F8093720290937302A0937402FF
:10D2D000B093750215C08091A90880935F03809177
:10D2E000AA0880935E038091AB0880935D0308C019
:10D2F00010925203109251031092500310924F0358
:10D300001F910F91FF90EF900895809160088823FE
:10D3100019F480E090E00895459881E798E09093B3
:10D320006A088093690890916103E92FFF27E0570D
:10D33000FE4F9F5F909361038081809373089D30BF
:10D3400010F010926103109260080E944D6581E018
:10D350008093700880917108809392088EBD81E05F
:10D3600090E0089587B18C6087B9429843981092F5
:10D37000680380E88093A101109267038093A00165
:10D3800008958091A2079091A30781589F4F39F08B
:10D390008091A2079091A307815880937203809196
:10D3A0006D03815080936D038F3F09F052C189E076
:10D3B00080936D0380914902992780739070892B27
:10D3C00021F48091A80380FF1DC0809180068823EE
:10D3D00051F080917003882319F484E080936803EE
:10D3E00081E080937003809181068823B9F0809159
:10D3F0007103882319F484E08093670381E08093AC
:10D4000071030CC0109270031092710380917C061E
:10D4100080936E0380917E0680936F0380917003EA
:10D42000882309F082C08091A006282F332724FF8B
:10D4300007C080918102882319F425FD8FC090C018
:10D4400090917D06983F48F0809124088D3D28F00A
:10D4500080916E0388236CF00AC0983F78F0809129
:10D460002408853059F480916E0387FF02C04298EA
:10D4700001C0429A81E08093A10154C08091680369
:10D480008150809368038F3F09F06BC08091A306A1
:10D4900085FF2FC090917203892F86958093680332
:10D4A000992361F49093660380916E0387FF02C015
:10D4B000429801C0429A1092A10153C081E080932A
:10D4C00066038091A10190916E03882349F48093B3
:10D4D000720380E88093A10199230CF441C03EC0FF
:10D4E000982311F0429A01C0429886958093A10139
:10D4F00038C0809124088695809368038091A101AB
:10D50000813021F41092720380E801C086958093E7
:10D51000A1018091A10190916E03892311F0429A9B
:10D5200001C04298109266031CC08091680381502C
:10D53000809368038F3FA9F489E08093680380910A
:10D54000A101813011F480E801C086958093A1018A
:10D550008091A10190918006892311F0429A01C027
:10D56000429880917103882309F043C09091A006EE
:10D5700097FF07C080918102882319F496FD52C05D
:10D5800053C090917F06983F48F080914D088D3DA3
:10D5900028F080916F0388236CF00AC0983F78F0E0
:10D5A00080914D08853059F480916F0387FF02C048
:10D5B000439801C0439A81E08093A00136C08091D6
:10D5C00067038150809367038F3F79F580914D0801
:10D5D0008695809367038091A001813011F480E8E3
:10D5E00001C086958093A0018091A00190916F0366
:10D5F00017C0809167038150809367038F3FA9F420
:10D6000089E0809367038091A001813011F480E864
:10D6100001C086958093A0018091A0019091810620
:10D62000892311F0439A01C04398429B05C0809121
:10D630004802886080934802439B06C0809148025C
:10D640008061809348020895809148028F7E809384
:10D65000480208954FB724E130E0F8948091C90062
:10D660008F778093C9008091C9008F7B8093C90018
:10D670008091C9008F7D8093C900832F9927809363
:10D68000CD002093CC008091C80082608093C800B8
:10D6900080E18093C9008091CA008F778093CA008F
:10D6A0008091CA008F7B8093CA008091CA008F7DD1
:10D6B0008093CA008091CA008F7E8093CA008091B7
:10D6C000CA00877F8093CA008091C9008B7F8093B6
:10D6D000C9008091CA0084608093CA008091CA000A
:10D6E00082608093CA008091C80087FF03C0809148
:10D6F000CE00F9CF8091C90080688093C9004FBFE8
:10D700000895EF92FF920F931F93CF93DF93482FCB
:10D7100000E010E08091A201813061F41092A2013A
:10D7200084E4809373031092750310927403109233
:10D73000760339C180917303882319F421E030E026
:10D7400001C0980190917403992371F4232B11F077
:10D7500081E010C084E480937303909375039093E9
:10D7600074039093760308C1913069F4232B09F078
:10D77000F9C082E080937403809175038F5F80937A
:10D78000750383E0F7C09230D1F4232B09F0EAC08F
:10D7900083E08093730340937603909175039230F6
:10D7A00039F41092770347FF03C081E08093770339
:10D7B00083E0809374039F5F90937503DDC0933083
:10D7C00009F0D0C0232B09F0CDC09093730382E001
:10D7D00080937403809175038F5F8093750320910C
:10D7E0007603822F9927782F6627842F9927682B15
:10D7F000792B80915906813049F47370CB018050A8
:10D80000924063E070E00E944D7A17C0823061F46C
:10D810007770CB018050944066E070E00E944D7AB2
:10D820002695269526950BC0737068567140CB01DE
:10D8300077FD0196BC017595679526952695022F73
:10D8400011270F7010700F5F1F4F0D30110508F07A
:10D8500082C07801E00EF11EF701E859F84F80818F
:10D8600091819B01281B390BC90137FF03C090959B
:10D8700081959F4F069704F5E0919B06EE2351F0AA
:10D88000FF27EE0FFF1FE859F84F80819181843602
:10D89000910594F480918202883C30F48091820258
:10D8A000865F8093820208C088EC80938202809118
:10D8B0006F008F7D80936F00F701E859F84F8081EA
:10D8C00091819C01220F331F280F391F260F371F0C
:10D8D00037FF02C02D5F3F4FE901D595C795D5951C
:10D8E000C795CB0101968C179D0714F4219706C0AC
:10D8F00061507040C617D7070CF4219680918202C0
:10D90000843BD0F0F701E859F84F80819181FE0106
:10D91000E81BF90BCF0163E070E00E944D7ACB0168
:10D92000880F991F860F971F2EEA37E0E20EF31E2D
:10D93000F7019183808307C02EEA37E0E20EF31EE1
:10D94000F70111821082000F111F0859184FF801BA
:10D95000D183C08311C00231110570F081E0809342
:10D96000A2010AC081E08093A20110927503109277
:10D97000770384E48093730380917503803198F07A
:10D9800080917703882331F48091A201882311F4D8
:10D9900080933C01109275031092770310927403E8
:10D9A00084E480937303E6E0CDB7DEB70C94C57AC8
:10D9B000CF93FC0197FF05C0CFEFF095E195FF4FA6
:10D9C00001C0C1E028E631E0CF01B9010E944D7AE3
:10D9D000FC018B35910554F08B5590408A359105AB
:10D9E00038F484EB90E08E1B9F0BFC0141E00DC0EE
:10D9F000CF01855B90408A35910518F4E45BF040D7
:10DA000003C02E1B3F0BF9014FEFEE0FFF1FE55A2E
:10DA1000F74F259134918C2F992787FD9095289F5A
:10DA2000B001299F700D389F700D1124842F992704
:10DA300087FD9095689FA001699F500D789F500DBC
:10DA40001124CA01CF9108952AE530E0281B390B33
:10DA5000C9010E94D86C0895CF93DF9380E00E94A3
:10DA6000327180912201909123016AE070E00E945E
:10DA70004D7A9F938F9380912201909123016AE0C8
:10DA800070E00E944D7A7F936F938FE299E09F93AD
:10DA90008F93C5E2D1E7DF93CF93E0918E03F091AE
:10DAA0008F0309952DB73EB7285F3F4F2DBF80915B
:10DAB0009D01882361F186E00E94327180918F017F
:10DAC00099279F938F9380916508909166086AE0EB
:10DAD00070E00E94397A7F936F938FED90E09F936F
:10DAE0008F9380910208909103089F938F9388E30E
:10DAF00099E09F938F93DF93CF93E0918E03F09102
:10DB00008F0309958DB79EB70C968DBF12C086E026
:10DB10000E94327186E499E09F938F93DF93CF93B5
:10DB2000E0918E03F0918F0309950F900F900F9065
:10DB30000F90809160038823F9F086E00E94327193
:10DB40008091600399279F938F938DE499E09F9331
:10DB50008F93DF93CF93E0918E03F0918F0309951C
:10DB60002DB73EB72A5F3F4F2DBF8091810288239A
:10DB700019F083E58093AE0180E10E9432718091BB
:10DB8000B0019091B1016CE370E00E94397A9F93EB
:10DB90008F938091B0019091B1016CE370E00E948D
:10DBA000397A7F936F938091DF089091E0089F937B
:10DBB0008F9389E599E09F938F93C5E2D1E7DF9337
:10DBC000CF93E0918E03F0918F03099580914608E1
:10DBD0002DB73EB7265F3F4F2DBF80FF29C08AE19A
:10DBE0000E94327180913D0199279F938F9380917C
:10DBF0007C0290917D02A0917E02B0917F02BC01D7
:10DC0000CD0124E630E040E050E00E94827A3F936C
:10DC10002F9386E699E09F938F93DF93CF93E091C4
:10DC20008E03F0918F0309958DB79EB708968DBF2F
:10DC3000DF91CF910895CF93DF9380E00E943271FE
:10DC400080912607992787FD90959F938F938091C8
:10DC50001E07992787FD90959F938F9380911607B4
:10DC6000992787FD90959F938F9380910E07992711
:10DC700087FD90959F938F938DE699E09F938F9367
:10DC8000C5E2D1E7DF93CF93E0918E03F0918F034C
:10DC9000099580E10E9432712DB73EB7245F3F4F56
:10DCA0002DBF80914607992787FD90959F938F936D
:10DCB00080913E07992787FD90959F938F93809140
:10DCC0003607992787FD90959F938F9380912E0714
:10DCD000992787FD90959F938F938DE799E09F9368
:10DCE0008F93DF93CF93E0918E03F0918F0309958B
:10DCF000809131062DB73EB7245F3F4F2DBF853051
:10DD000098F480E10E9432718DE899E09F938F939F
:10DD1000DF93CF93E0918E03F0918F0309950F90DD
:10DD20000F900F900F9018C08730B0F488E10E94D8
:10DD300032718FED90E09F938F938EE999E09F93DE
:10DD40008F93DF93CF93E0918E03F0918F0309952A
:10DD50008DB79EB706968DBFDF91CF9108950F9333
:10DD60001F9380E00E9432712AE030E08091DB084E
:10DD70009091DC08B9010E94397A9F938F9380912A
:10DD8000DB089091DC08B9010E94397A7F936F9388
:10DD90008091220190912301B9010E944D7A9F93B5
:10DDA0008F938091220190912301B9010E944D7AB5
:10DDB0007F936F9387EA99E09F938F9305E211E732
:10DDC0001F930F93E0918E03F0918F03099580E1EB
:10DDD0000E9432718DB79EB70C968DBF8091DF087F
:10DDE0009091E0089F938F938091DD089091DE08D9
:10DDF0009F938F9389EB99E09F938F931F930F933A
:10DE0000E0918E03F0918F0309958DB79EB7089628
:10DE10008DBF1F910F910895EF92FF920F931F9363
:10DE200080E00E9432718FEDE82EF12CFF92EF928C
:10DE300080918C0190918D019F938F9380915F03CE
:10DE400099279F938F9385EC99E09F938F9305E299
:10DE500011E71F930F93E0918E03F0918F030995C3
:10DE600080E10E9432718DB79EB70A968DBF809176
:10DE70005D0399279F938F93FF92EF9280915E03AA
:10DE800099279F938F9388ED99E09F938F931F938A
:10DE90000F93E0918E03F0918F0309958DB79EB794
:10DEA0000A968DBF1F910F91FF90EF9008950F93E9
:10DEB0001F93CF93DF9380919D01C5E2D1E7882323
:10DEC00009F47DC080E00E94327180916208992738
:10DED0009F938F938091640899279F938F938BEEE4
:10DEE00099E09F938F938E01DF93CF93E0918E0300
:10DEF000F0918F0309958DB79EB708968DBF8091DD
:10DF00006308833031F48CE00E9432718AEF99E02B
:10DF100005C08CE00E9432718FEF99E09F938F9340
:10DF2000DF93CF93E0918E03F0918F0309950F90CB
:10DF30000F900F900F908091610881FF12C08CE0CC
:10DF40000E94327184E09AE09F938F931F930F9306
:10DF5000E0918E03F0918F0309950F900F900F9031
:10DF60000F9080E10E94327180918F0199279F93D9
:10DF70008F938FED90E09F938F938091670890919E
:10DF800068089F938F9380916508909166086AE076
:10DF900070E00E94397A7F936F9389E09AE09F93B3
:10DFA0008F9385E291E79F938F93E0918E03F09199
:10DFB0008F0309958DB79EB70C968DBF12C082E076
:10DFC0000E9432718CE19AE09F938F93DF93CF93FD
:10DFD000E0918E03F0918F0309950F900F900F90B1
:10DFE0000F90DF91CF911F910F910895CF93C82F7C
:10DFF000209178032093790399278F329105E1F0DE
:10E00000803391051CF44F9779F027C08F34910528
:10E01000D9F08F38910509F586E0289FF001112489
:10E02000EF5EF64F849117C086E0289FF00111241F
:10E03000EE5EF64F84910FC086E0289FF001112418
:10E04000ED5EF64F849107C086E0289FF001112411
:10E05000EC5EF64F849180937803909178038091E1
:10E0600079039813C0E08091A301282F33278F5F95
:10E070008093A30120FF0FC00E9438719091780314
:10E0800086E0989FF0011124EB5EF64F25913491C4
:10E090008C2FF901099580E090E0CF9108951092BE
:10E0A000DC081092DB081092E0081092DF08109252
:10E0B000DE081092DD081092E1088AE090E00E94EC
:10E0C000DF1590937B0380937A030895CF93DF93BA
:10E0D00080917A0390917B030E94E815882309F4CC
:10E0E000AFC080917A0390917B030A9690937B0353
:10E0F00080937A03E0E0F0E09F0190E05FEFA7E01B
:10E10000B7E04BE0ED018B8187FF0BC09F5F8D81F6
:10E11000E80FF11D8981280F311D8E81851708F4C4
:10E12000582F4150189647FFEDCF5093E108232B0D
:10E1300041F52091800330918103409182035091F9
:10E140008303BB27A52F942F832F90937F03809366
:10E150007E03AA27BB27281B390B4A0B5B0BCF0179
:10E16000AA27BB27280F391F4A1F5B1F2093800354
:10E17000309381034093820350938303E5E0F0E002
:10E1800013C020917E0330917F032E173F0718F4B0
:10E19000E21BF30B02C0E0E0F0E0892F9927880F23
:10E1A000991FE80FF91F3596F093DC08E093DB0820
:10E1B000EF3FF10578F480912201909123018E9F29
:10E1C00090018F9F300D9E9F300D1124C90164E690
:10E1D00070E013C0CF01969587959695879520910D
:10E1E000220130912301289FA001299F500D389FC3
:10E1F000500D1124CA0169E170E00E94397A7093D0
:10E20000DE086093DD0820917C0330917D032E0FA2
:10E210003F1F30937D0320937C035EE0213135075F
:10E2200078F08091DF089091E00801969093E008E3
:10E230008093DF0820513E4030937D0320937C0380
:10E24000DF91CF91089508950895909187039332B7
:10E2500040F4E92FFF27EE51F74F80839F5F9093A3
:10E2600087030895833218F48D5F809387030895A0
:10E2700090E2E5EEF8E08FE19193815087FFFCCFCB
:10E280000895CF93CFB723E031E0F8948091C9008F
:10E290008F778093C9008091C9008F7B8093C900DC
:10E2A0008091C9008F7D8093C900832F9927809327
:10E2B000CD002093CC008091C80082608093C8007C
:10E2C00088E18093C9008091CA008F778093CA004B
:10E2D0008091CA008F7B8093CA008091CA008062BF
:10E2E0008093CA008091CA0080618093CA008091A7
:10E2F000CA0088608093CA008091C90084608093BE
:10E30000C9008091CA0084608093CA008091CA00CD
:10E3100082608093CA008091C80087FF03C080910B
:10E32000CE00F9CF8091C90080688093C9008091A8
:10E33000C90080648093C9000E943871CFBFCF911B
:10E340000895282F99278F709070892B31F420958C
:10E3500080918603822B8093860308958091AA0181
:10E36000882309F44BC08091490285FD04C0809147
:10E37000AE01882381F082E98093E20883E28093F2
:10E38000E3088091AE01882309F485E58093E408D1
:10E390001092AE0102C08093E2088091AB018F30F1
:10E3A00071F4809186030E94F66F882341F081E921
:10E3B0008093E2088093E30881E38093E40810925D
:10E3C000AA018091C80085FFFCCF8091C9008F7E93
:10E3D0008093C9008091C9008E7F8093C90080918D
:10E3E000E208882311F48EEF01C08EE78093CE00FF
:10E3F000809186038093AB011092860308951F924B
:10E400000F920FB60F9211248F939F93EF93FF9368
:10E410009091AA01992309F040C080918803882334
:10E4200061F48091E208882311F483E003C081390C
:10E4300099F481E0809388030FC0833099F4809130
:10E44000E208882349F09093E2088091C9008E7F0A
:10E450008093C9008EEF1EC08091C90081608093B7
:10E46000C9000EC0833261F48091C9008E7F809311
:10E47000C9008FEF8093CE0081E08093AA0118C07D
:10E4800080918803E82FFF27EE51F74F8F5F80932D
:10E49000880380818093CE000BC010928803109275
:10E4A000890310928A038091C90080618093C9001A
:10E4B000FF91EF919F918F910F900FBE0F901F9042
:10E4C0001895EF92FF920F931F93CF93DF937C01E8
:10E4D0008B01EA01452B39F0F80181918F01F70199
:10E4E00009952197C9F7E6E0CDB7DEB70C94C57A58
:10E4F000EF92FF920F931F93CF93DF937C018B01D9
:10E50000EA01452B41F0F8010F5F1F4F8491F7019D
:10E5100009952197C1F7E6E0CDB7DEB70C94C57A2F
:10E520000F931F93CF938C01C62F161634F480E2FD
:10E53000F8010995C1501C16D4F3CF911F910F918A
:10E5400008950F931F93CF938C01C62F161634F4A2
:10E5500080E3F8010995C1501C16D4F3CF911F91A7
:10E560000F910895A5E3B0E0E8EBF2E70C949D7AF3
:10E570002E96EEADFFAD2E978824992454018091FC
:10E580008503882321F42C961FAE1EAE2C97AEE493
:10E590004A2E512C4C0E5D1E6F01B60105C015327E
:10E5A00039F00894C11CD11CF60114911123B9F75C
:10E5B000A601461B570B31F02C968EAD9FAD2C97C4
:10E5C0000E947872112309F46AC20894C11CD11CFC
:10E5D000FF24FDA6FCA67FEFE72EF9A6F60108941E
:10E5E000C11CD11C1491153721F0812F806288370E
:10E5F000B1F4F0FE0AC0F20124E030E0420E531EF6
:10E6000080809180A280B3800AC0F20142E050E095
:10E61000440E551E808191814C01AA24BB241032E6
:10E6200021F489A58823D1F61DC0133219F458E0CE
:10E63000F52AD4CF1A3211F01D3291F41A3259F45E
:10E64000F20182E090E0480E591EE081ECA7EE2333
:10E650002CF6E195ECA790E1F92AAFEDFA22BECFB6
:10E660001B3211F419A7BACF1E32C1F5F601089476
:10E67000C11CD11C14911A3279F4F20122E030E06D
:10E68000420E531E408151813FEF4F3F530714F418
:10E690004FEF5FEFE42EA2CF40E050E0812F805398
:10E6A0008A30A0F4CA0163E0880F991F6A95E1F7E8
:10E6B000840F951F480F591F410F511D4053504063
:10E6C000F6010894C11CD11C1491E8CF8FEF4F3F85
:10E6D000580714F44FEF5FEFE42E85CF103329F481
:10E6E000F4FC7CCF90E2F92A79CF812F81538930D5
:10E6F000D8F440E050E0CA0133E0880F991F3A9502
:10E70000E1F7840F951F480F591F410F511D4053CA
:10E710005040F6010894C11CD11C1491812F8053E4
:10E720008A3048F34CA75FCF183619F4A4E0FA2AD0
:10E7300055CF1C3619F4B1E0FB2A50CF133661F4E3
:10E740003E010894611C711CF20122E030E0420E8F
:10E75000531E808189833CC1143421F0143611F09A
:10E76000193651F5143411F431E0F32AF0FE0AC0E1
:10E77000F20144E050E0440E551E80809180A2805A
:10E78000B3800CC0F20182E090E0480E591E8081F7
:10E7900091814C01AA2497FCA094BA2CB7FE0AC020
:10E7A000B094A09490948094811C911CA11CB11CE5
:10E7B0008DE289A70AE06FC01F3411F01F3631F4D3
:10E7C0001F3411F491E0F92A08E064C0103779F49D
:10E7D000F201A2E0B0E04A0E5B1E808191814C0103
:10E7E000AA24BB2400E1B0E4FB2A18E753C0133786
:10E7F000C1F5F20122E030E0420E531E60807180CC
:10E800006114710489F43E010894611C711C88E252
:10E8100089838EE6F301818385E78B838CE68C8385
:10E820008D8389E28E831F82E7FC13C08E2D99278A
:10E8300087FD9095AC0160E070E0C3010E946A78AA
:10E84000009729F0382E3618E3140CF0C3C03E2C84
:10E85000C1C0F30101900020E9F731973E2E361830
:10E86000B9C0153511F0153731F4153511F4F1E053
:10E87000FF2A0AE00FC0183519F0183709F0A0C0B8
:10E8800000E1F3FE07C081149104A104B10411F06A
:10E8900020E4F22A19A6EDA6E7FC02C03FEDF32220
:10E8A00029E2622E712C6C0E7D1E81149104A1044C
:10E8B000B10421F44DA5442309F47BC0802F99278E
:10E8C000AA27BB278EA79FA7A8ABB9AB202E3324BE
:10E8D00090E0891690E0990691E0A90690E0B906CB
:10E8E00048F0C501B4012EA53FA548A959A90E9429
:10E8F000607A17C0AFEF8A169104A104B10449F001
:10E9000040F0C401B1010E94397A9B014427552788
:10E9100008C0882D602F0E942D7A282F3327442786
:10E9200055272AAB3BAB4CAB5DAB0A3059F48AA9F7
:10E93000880F880F880F9AA9990F890F382D381BD7
:10E94000832F10C0003139F48AA98295807F482D29
:10E95000481B842F07C08AA9880F880F880F582D5D
:10E96000581B852F90E02EA53FA548A959A98216CE
:10E970009306A406B50608F091E08AA89BA8ACA867
:10E98000BDA88A3010F4805D04C0895A183509F496
:10E990008F7DD3018E933D01992309F099CF0830E3
:10E9A00041F4F3FE06C0803321F080E3FD01829341
:10E9B0003F01CE010196382E3618F8E23F0E0BC00B
:10E9C000112309F46CC03E010894611C711C198369
:10E9D00091E0392E19A6032D2DA4231827FC2224FB
:10E9E00089A5882311F00F5F02C0F6FC0E5F020DAF
:10E9F000EF2CFF24C70180739070892B49F48CA5FC
:10EA0000801B682F2C968EAD9FAD2C970E94907224
:10EA100089A5882331F041E050E0BE01675D7F4F5A
:10EA20000AC0E6FE0EC080E38AA71BA742E050E0C2
:10EA3000BE01665D7F4F2C968EAD9FAD2C970E94D8
:10EA40006172C70180739070809749F48CA5801B18
:10EA5000682F2C968EAD9FAD2C970E94A172622DCF
:10EA60002C968EAD9FAD2C970E94A172832D992775
:10EA700087FD9095AC01B3012C968EAD9FAD2C9780
:10EA80000E946172E4FE89CD2CA5201B2CA7622F69
:10EA90002C968EAD9FAD2C970E9490727ECDE2E1B8
:10EAA000CB5C0C94B97A2FB740E0F894E0E0F0E04A
:10EAB00081E2809357009491E2E0F0E08093570068
:10EAC0003491E4E0F0E08093570084912FBF9E31B1
:10EAD00099F4363941F4893011F441E00DC08A309F
:10EAE00059F442E009C0373939F4863011F443E073
:10EAF00003C0853009F444E0842F992708959FB717
:10EB0000F8948091C900877F8093C9008091C900E3
:10EB10008F7E8093C9008091C9008F778093C90050
:10EB20008091C9008F7B8093C9008091C9008F7D3F
:10EB30008093C9009FBF08951F93CF93DF93182F31
:10EB400080918503882309F4A0C08091A90118173A
:10EB500009F49BC080918403882321F40E9453759B
:10EB60008093840382ED91E090933B0180933A017E
:10EB700088EC9AE09F938F93C2E0D2E1DF93CF932A
:10EB8000E0918E03F0918F0309950F900F900F90F5
:10EB90000F90812F992784309105F1F085309105F0
:10EBA0001CF4892B51F00CC086309105D9F08630C9
:10EBB0009105ACF0089741F12AC084EC9AE002C0BC
:10EBC0008BEB9AE09F938F93DF93CF93E0918E032B
:10EBD000F0918F03099527C086EB9AE0F3CF8EEA78
:10EBE0009AE0F0CF86EA9AE09F938F93DF93CF93DA
:10EBF000E0918E03F0918F03099588ED91E0909359
:10EC00003B0180933A010FC081EA9AE0DBCF85EDAA
:10EC10009AE09F938F93DF93CF93E0918E03F091CF
:10EC20008F03099510E00F900F900F900F90809137
:10EC30008403843011F0823099F40E947F75812F13
:10EC40008150833018F40E942A6B1DC0143019F4CF
:10EC50000E94417118C01830B1F40E94237113C092
:10EC6000112389F08BEE9AE09F938F9382E092E1DB
:10EC70009F938F93E0918E03F0918F0309950F90EE
:10EC80000F900F900F901093A901DF91CF911F91DA
:10EC900008950F931F93082F81E08093850340917F
:10ECA000A801E1E5FAE020E030E05FE484919927F3
:10ECB0002F5F3F4F829FB001839F700D929F700D19
:10ECC000112446275150319657FFF0CF4093A801A9
:10ECD000E9E2FAE020E030E057E2849199272F5FE3
:10ECE0003F4F829FB001839F700D929F700D112442
:10ECF00046275150319657FFF0CF4093A80180919D
:10ED00008403882321F40E9453758093840382EB4B
:10ED100092E790938F0380938E038091A8018334B0
:10ED200059F088E190E029E20FB6F894A895809315
:10ED300060000FBE20936000053091F086E09BE0FC
:10ED40009F938F9382E092E19F938F93E0918E0344
:10ED5000F0918F0309950F900F900F900F90EECFC9
:10ED60000E94F40586E690E09F938F931F921F9276
:10ED700082E090E09F938F93809102016AE00E946D
:10ED80002D7A892F99279F938F93809102010E945A
:10ED90002D7A99279F938F9383E29BE09F938F9384
:10EDA00002E012E11F930F93E0918E03F0918F0325
:10EDB000099581E59AE09F938F931F930F93E091BC
:10EDC0008E03F0918F03099589E29AE09F938F93C8
:10EDD0001F930F93E0918E03F0918F0309950E948A
:10EDE000F40583EC8093810080916F0080628093B2
:10EDF0006F008DB79EB746968DBF1F910F910895F6
:10EE0000809199068D3338F08091610887FD03C0A9
:10EE10008CE38093990680914806882331F08055D1
:10EE2000853618F08FE78093480608958091850312
:10EE3000882309F472C080918B03815080938B03E7
:10EE4000882309F059C089E180938B03809199064A
:10EE50008E3338F08091610887FD03C08DE3809385
:10EE6000990680918202823820F580914A02909121
:10EE70004B02805D974020F08091E108843620F4B9
:10EE800010928D0310928C0380918C0390918D03CE
:10EE9000009739F1019790938D0380938C034197EC
:10EEA00028F18091610884FF21C08091480284602C
:10EEB0001BC080918202853BC8F09091990684E145
:10EEC000989FC0011124409620918C0330918D03AE
:10EED0002817390730F42F5F3F4F30938D0320936D
:10EEE0008C03809148028B7F809348028091A80117
:10EEF000833411F0109285038091AC01882321F0B6
:10EF000081508093AC0108958BE48093AC01809193
:10EF1000A901843011F40E94AE7108951F920F92DE
:10EF20000FB60F9211242F933F934F935F936F93DC
:10EF30007F938F939F93AF93BF93EF93FF93209112
:10EF4000CE008091B8018823B1F02093C600809153
:10EF5000B801823029F52F3F19F58FEF94E3ACE02B
:10EF6000B0E0C297A109B109B7FFFBCF8091D103EF
:10EF70008093CE0015C09091A901892F81508330D4
:10EF800020F4822F0E94816B0BC0943021F4822FD9
:10EF90000E94A17105C0983019F4822F0E9424713B
:10EFA000FF91EF91BF91AF919F918F917F916F9161
:10EFB0005F914F913F912F910F900FBE0F901F9037
:10EFC0001895002422273327442751E0BB27EE273A
:10EFD000FF27A0E1660F771F881F991F001C221FC3
:10EFE000331F441F660F771F881F991F001C221FA5
:10EFF000331F441F2AF4050E2B1F3E1F4F1F04C052
:10F00000051A2B0B3E0B4F0B550FBB1FEE1F587FE6
:10F01000556047FD5250AA95E9F6E695B795579584
:10F02000E695B7955795852F9B2F0895222733276F
:10F0300041E0552768E0880F991F221F331F880F72
:10F04000991F221F331F1AF4240F351F02C0241BDF
:10F05000350B440F551F487F456037FD42506A9578
:10F0600051F75695479556954795842F0895AA27A9
:10F0700097FF04C0809590958A1F9A1F77FF04C060
:10F08000609570956A1F7A1F669F9001779FA00117
:10F09000679F300D411D5A1F300D411D5A1F889F1B
:10F0A000F001999F2E0F3F1F401D511D899F300D6C
:10F0B000411D5A1F300D411D5A1FCA01B9011124AB
:10F0C00080CFFB01DC0102C005900D924150504001
:10F0D000D8F70895FC014150504030F001900616D9
:10F0E000D1F73197CF010895882799270895A0E097
:10F0F000B0E0EDE7F8E70C94A57A6C017B01EA013A
:10F10000590121978FEFCF3FD80789F086010894E6
:10F11000C11CD11CC7010894E11CF11CF501099523
:10F12000F80180832197FFEFCF3FDF0779F7EAE00F
:10F13000CDB7DEB70C94C17ACF92DF92EF92FF92F7
:10F140000F931F937C016B01FB010995082FC701E9
:10F150000196F6010995182FC8011F910F91FF9094
:10F16000EF90DF90CF900895A0E0B0E0EAEBF8E7F1
:10F170000C94A77A8C017B01EA01690121978FEF3A
:10F18000CF3FD80771F0F70121917F01C8010F5FD0
:10F190001F4F622FF60109952197FFEFCF3FDF0741
:10F1A00091F7E8E0CDB7DEB70C94C37ACF92DF9247
:10F1B000EF92FF920F931F936C018B017A01FA017A
:10F1C0000995812F9927682FC6010196F7010995A6
:10F1D0001F910F91FF90EF90DF90CF9008955058BE
:10F1E000BB27AA270ED0E0C0D1D030F0D6D020F077
:10F1F00031F49F3F11F41EF4C6C00EF4E095E7FB16
:10F20000BCC0E92FE2D080F3BA1762077307840706
:10F21000950718F071F49EF5FAC00EF4E0950B2EE8
:10F22000BA2FA02D0B01B90190010C01CA01A00158
:10F230001124FF27591B99F0593F50F4503E68F1B3
:10F240001A16F040A22F232F342F4427585FF3CFF4
:10F25000469537952795A795F0405395C9F77EF4C5
:10F260001F16BA0B620B730B840BBAF09150A1F00E
:10F27000FF0FBB1F661F771F881FC2F70EC0BA0F94
:10F28000621F731F841F48F4879577956795B7951C
:10F29000F7959E3F08F0B3CF9395880F08F0992714
:10F2A000EE0F97958795089598D088F09F5790F026
:10F2B000B92F9927B751A0F0D1F0660F771F881F9B
:10F2C000991F1AF0BA95C9F712C0B13081F09FD0DA
:10F2D000B1E008959CC0672F782F8827B85F39F078
:10F2E000B93FCCF3869577956795B395D9F73EF4FA
:10F2F00090958095709561957F4F8F4F9F4F0895A2
:10F30000E89409C097FB3EF49095809570956195BF
:10F310007F4F8F4F9F4F9923A9F0F92F96E9BB2775
:10F320009395F695879577956795B795F111F8CFF1
:10F33000FAF4BB0F11F460FF1BC06F5F7F4F8F4F5C
:10F340009F4F16C0882311F096E911C0772321F052
:10F350009EE8872F762F05C0662371F096E8862FEA
:10F3600070E060E02AF09A95660F771F881FDAF741
:10F37000880F9695879597F9089597F99F6780E884
:10F3800070E060E008959FEF80EC089500240A94F7
:10F390001616170618060906089500240A94121670
:10F3A0001306140605060895092E0394000C11F4A3
:10F3B000882352F0BB0F40F4BF2B11F460FF04C050
:10F3C0006F5F7F4F8F4F9F4F089557FD9058440FA9
:10F3D000551F59F05F3F71F04795880F97FB991FB4
:10F3E00061F09F3F79F08795089512161306140671
:10F3F000551FF2CF4695F1DF08C0161617061806FE
:10F40000991FF1CF86957105610508940895E894D8
:10F41000BB2766277727CB0197F90895629FD00114
:10F42000739FF001829FE00DF11D649FE00DF11DBF
:10F43000929FF00D839FF00D749FF00D659FF00D6E
:10F440009927729FB00DE11DF91F639FB00DE11D5B
:10F45000F91FBD01CF0111240895991B79E004C063
:10F46000991F961708F0961B881F7A95C9F7809503
:10F470000895AA1BBB1B51E107C0AA1FBB1FA617FB
:10F48000B70710F0A61BB70B881F991F5A95A9F74D
:10F4900080959095BC01CD01089597FB092E072614
:10F4A0000AD077FD04D0E5DF06D000201AF470956D
:10F4B00061957F4F0895F6F7909581959F4F089538
:10F4C000A1E21A2EAA1BBB1BFD010DC0AA1FBB1F68
:10F4D000EE1FFF1FA217B307E407F50720F0A21BDA
:10F4E000B30BE40BF50B661F771F881F991F1A9447
:10F4F00069F760957095809590959B01AC01BD0171
:10F50000CF01089597FB092E05260ED057FD04D094
:10F51000D7DF0AD0001C38F45095409530952195DE
:10F520003F4F4F4F5F4F0895F6F790958095709538
:10F5300061957F4F8F4F9F4F08952F923F924F922B
:10F540005F926F927F928F929F92AF92BF92CF9273
:10F55000DF92EF92FF920F931F93CF93DF93CDB77C
:10F56000DEB7CA1BDB0B0FB6F894DEBF0FBECDBFF4
:10F5700009942A88398848885F846E847D848C84C5
:10F580009B84AA84B984C884DF80EE80FD800C81CE
:10F590001B81AA81B981CE0FD11D0FB6F894DEBFB1
:10F5A0000FBECDBFED010895EE0FFF1F0590F49142
:06F5B000E02D0994FFCFDD
:10F5B600035E0A010164FF010020FFFFC01FC01F98
:10F5C6000101F40101737373FF03007D0000C40998
:10F5D600C4096400114167696C6500517561647204
:10F5E6006F000000000000006400D20101200B053E
:10F5F6000000ECFF000204060708080807060402DC
:10F6060000FEFCFAF9F8F8F8F9FAFCFE0002040626
:10F616000708086440415A4655326464640A0296F3
:10F626009696960840403A1030380132FF0378002B
:10F6360090D0030090D0030032002064FFFF6420C6
:10F646000B0A0D0B0E100B0A0C0F0B1110FA20688B
:0EF6560001010101F7FFFCFF70FF010F6400CE
:00000001FF
